:020000040800F2
:1000000000000120117204088D7204087D1A020894
:10001000BD1A02088D7204088D72040800000000E9
:100020000000000000000000000000008D720408C5
:100030008D720408000000008D720408011302088C
:100040008D7204088D7204088D7204088D72040884
:100050008D7204088D720408D91B0208051D020860
:10006000C91C02088D1C0208511C0208C584030823
:10007000B5840308A58403089584030881840308D4
:100080006D840308598403088D7204088D72040876
:100090008D7204088D7204088D720408151C020804
:1000A0008D7204086D6C0308196C03085D6C0308FD
:1000B0004D6C03088D7204083D6C03088D720408B2
:1000C0008D7204088D7204088D7204088D72040804
:1000D0008D7204084D630308416303083563030808
:1000E0009D1B02088D7204088D7204088D7204082D
:1000F000396C03088D720408296C030845840308D1
:100100008D7204088D7204088D7204088D720408C3
:10011000296303081D6303088D7204084BBE0108A0
:10012000318403081D84030809840308F583030848
:10013000E183030800000000000000000000000050
:1001400000000000000000000000000083C801085B
:10015000CD830308B9830308A5830308116303084B
:100160008D7204088D7204088D7204088D72040863
:100170008D7204088D720408000000000000000069
:100180008D7204088D7204088D7204088D72040843
:100190008D7204088D720408000000008D7204083E
:1001A0000000000000000000000000008D72040844
:1001B0008D7204088D720408000000000000000029
:1001C000000000000000000000000000000000002F
:1001D0000000000000000000000000008D72040814
:0801E000606D04000100000045
:1001E800F8210600C22C0120B435012000000000CF
:1001F80024070008031233009C2E01203835012003
:10020800000000002A07000825009600FC330120A2
:10021800923401200000000000000000150070006A
:100228002D320120143301200000000000000000DE
:100238002A006000D82C0120B43201200000000000
:100248004DF503082C0010009E32012028350120AE
:1002580000000000A99C00082B0024008F35012015
:100268006B35012000000000799C000829107800F7
:10027800403101208433012000000000000000000C
:1002880028101000CC350120BC35012000000000EA
:100298000180000814000300A8300120AE320120BC
:1002A800000000005E0700080C106C000A3D0120E9
:1002B800E0450120000000006DE502080E50200115
:1002C800C03B01204C4601200000000075F50308E2
:1002D80013000400804101206C4701200000000049
:1002E80064070008010104003A3B0120704701201F
:1002F800000000000000000000010400323B012063
:10030800744701200000000068070008020103008C
:100318002D3B012078470120000000009DE50208E0
:10032800090201001C4401207C4701200000000054
:100338006C07000801020500423B012080470120AC
:10034800000000006D190108000205008840012026
:100358008847012000000000000000001B02080080
:100368007C4001209047012000000000A102020803
:1003780001200800E4420120984701200000000005
:100388006E0700081900050094430120A0470120CA
:10039800000000007607000837001E006C430120AB
:1003A800A8470120000000007C0700081E00050087
:1003B8005C3E0120C8470120000000009A070008A1
:1003C8001B00F40058360120D0470120000000002F
:1003D800B12601080E0202001E420120C448012075
:1003E80000000000A00700082F001100A045012010
:1003F800C848012000000000A207000805100600F8
:10040800903D0120DC48012000000000B4070008EE
:10041800F5317000E0350120E448012000000000BB
:100428007153010826000E00644901205449012037
:1004380000000000B91101080B201000045301202E
:10044800485F012000000000BA0700081F201C00B8
:10045800904A0120585F012000000000CA070008E8
:1004680005020400E45C0120745F01200000000024
:10047800E607000803010A00B6520120785F012050
:1004880000000000EA0700081A023C009C5F0120F7
:1004980090630120000000005907020827000400AB
:1004A800985F0120CC63012000000000F4070008D9
:1004B8000A020A00746A0120F86A0120000000009C
:1004C800F80700080300010070650120046B012093
:1004D8000000000000000000101002001C65012050
:1004E800086B012000000000020800081600080040
:1004F800306C0120BC6C01200000000004080008DA
:1005080002000C00246C0120E46C012000000000B3
:100518000000000008120C008A6C0120F06C012019
:1005280000000000F1020208F7010600846C0120B7
:10053800FC6C0120000000000C08000810020100FB
:10054800A07501209C750120000000001208000819
:100558000400800038BB01200CBD01200000000011
:1005680000000000F6210C001CBB01208CBD0120FE
:1005780000000000140800082300100004BB01203C
:10058800DCBD012000000000198000080D004C00AF
:1005980064BA0120ECBD01200000000031F502081A
:1005A800FD01240098B1012038BE012000000000A0
:1005B80041FE010818202C0068B101205CBE012012
:1005C800000000002D090208061018004CB1012097
:1005D80088BE012000000000D5F50308FB010100DA
:1005E80048B10120A0BE012000000000790D0208DA
:1005F800FC01090014B00120A4BE01200000000085
:10060800890D02080A402000D8980120B0BE0120B8
:100618000000000020080008340010003CAF012052
:10062800D0BE012000000000A5F503081102080053
:1006380014AF0120E0BE01200000000040080008BF
:10064800121204000CAF0120E8BE012000000000D7
:100658004808000812200D00FCAE0120ECBE012065
:10066800000000004C080008F9010400E4A3012080
:10067800FCBE012000000000BDFE010813020300BB
:10068800E0A3012000BF0120000000005A08000874
:1006980018020200A8A1012004BF012000000000E8
:1006A8000000000017020B009CA1012008BF0120D8
:1006B80000000000AD020208FA01020078A1012042
:1006C80014BF012000000000193C030802020300C7
:1006D8007C9C012018BF01200000000000000000E1
:1006E8000C020300089901201CBF01200000000033
:1006F80029030208FE010900249E012020BF0120D1
:1007080000000000390302081A000E00BCC10120D5
:0C07180028C20120000000005E0800085C
:100724000401F401190000000000000000000000B2
:1007340000000000000000000000000000000000B5
:1007440000000000000000000000000000000000A5
:100754000000000000000000010003000000000091
:1007640048040430900100002900E8036400040AEE
:10077400000100002801000020003200C800D0075A
:100784009600140032002800B00440060005500012
:1007940014000F0008010000010000000000000028
:1007A4000000000000000000000000000000000045
:1007B4002000010100002B21231E64010100000020
:1007C40001000A01290000000000000100000005EA
:1007D400000001020300000000000000000000000F
:1007E400000000000000040101006C16000000007D
:1007F4002003000000004A01B400D60128000005CF
:10080400C40900001901282822010000000000008A
:10081400000000000100000002020000003001009E
:100824000000000064002C01000000000000000033
:100834000000020000019E077D00463220000000F7
:1008440001010101FFFFFFFF000000010000054D51
:10085400424637000000000000007E05EA05B405AA
:080864003200E803D007000098
:10086C00D60101000001010100FFFF00FFFFFFFFA7
:10087C000100000000000100E00101010100000086
:10088C00591B0108000000009401012014200508E8
:10089C00000000000000000000000000000000004C
:1008AC00841505080000000000000000260201204D
:1008BC0004000000C01F05080D000000D143010812
:1008CC00041C012000000000281905080D00000080
:1008DC00F9430108F81B012000000000841A0508E8
:1008EC000800000000000000EC1B012004000000C8
:1008FC00881905080D0000000D1C0108E01B0120E3
:10090C0000000000381A0508030000000D23010840
:10091C00D41B012000000000242005080300000067
:10092C000D230108C81B012000000000CC15050890
:10093C0001000000000000000000000000000000AA
:10094C00000000000E00000000000000000000008D
:10095C00000000001420050800000000000000004A
:10096C0000000000000000008415050800000000D5
:10097C000000000026020120040000006C1F050886
:10098C000300000075240108BC1B012008000000B6
:10099C00881905080D0000000D1C0108E01B012042
:1009AC0000000000381A0508030000000D230108A0
:1009BC00D41B0120000000002420050803000000C7
:1009CC000D230108C81B012000000000CC150508F0
:1009DC00010000000000000000000000000000000A
:1009EC00000000000E0000000000000000000000ED
:1009FC00000000002C200508000000000000000092
:100A0C000000000000000000841505080000000034
:100A1C00000000002602012004000000741F0508DD
:100A2C00030000000D230108101C01200000000031
:100A3C00CC150508010000000000000000000000BB
:100A4C0000000000000000000E000000000000008C
:100A5C00000000000000000020700020702D7200CB
:100A6C00FFFFFFFF0000803F0801000000000000B6
:100A7C000000000078170120FA00000001000000BF
:100A8C0001000000FFFF2D202D2D202D2D2D2D20C0
:100A9C002D2D2D00000000000000000000000000C3
:100AAC000000000000010000FFFFFFFFA01505087B
:100ABC00A8150508C415050800000000000000007A
:100ACC0000000000000000002A13050804000000CC
:100ADC00994101080000000000000000CC15050839
:100AEC0001000000000000000000000000000000F9
:100AFC00000000000E0000000000000000000000DC
:100B0C0000000000624101200100C4090000000047
:100B1C00604101200100C409000000005E41012079
:100B2C000100C409000000005C4101200100C4095F
:100B3C0000000000584101200100C4090000000021
:100B4C005A4101200100C409000000005641012057
:100B5C000100C40900000000544101200100C40937
:100B6C0000000000543B01200100C80001000000FF
:100B7C00523B01203200307532000000503B012006
:100B8C00055A05004D3B012000FF01004F3B0120A1
:100B9C00010000004C0201204B3B01200200000030
:100BAC0014B404084C3B012000FF01004E3B012013
:100BBC00010000004C0201204A3B01200200000011
:100BCC0014B40408403B012080C1803E05000000A5
:100BDC003E3B012080C1803E05000000383B0120D7
:100BEC0080C1803E05000000363B012080C1803E64
:100BFC0005000000303B012000FF01002C3B0120D0
:100C0C000A3201002B3B01200400000040B4040810
:100C1C002A3B01200200000054B40408000000002C
:100C2C000000000054020120905C01209CFF2C016C
:100C3C00000000001A0001200A00000060B4040843
:100C4C00203B0120E0150C17000000001C000120C7
:100C5C000800000090B604081B00012005000000ED
:100C6C0094B50408223B01200200000078B404086B
:100C7C00963D01200100FF7F010000008F3D012007
:100C8C000200000084B40408B33B01200300000000
:100C9C0094B40408B23B01200300000094B404088F
:100CAC00EA3C01200000F40101000000E83C0120B6
:100CBC000000F40101000000E63C01200000F401FA
:100CCC0001000000E43C01200000F40101000000E0
:100CDC00E23C01200000803E01000000E03C0120CD
:100CEC000000803E01000000063D0120E803D00713
:100CFC000A000000043D0120006401000A0000000D
:100D0C00F93C012000640100F83C01200064010062
:100D1C00003D0120006401000A000000FF3C01209E
:100D2C00006401000A000000FE3C01200064010088
:100D3C000A000000033D0120006401000A000000CD
:100D4C00023D0120006401000A000000013D012069
:100D5C00006401000A000000FD3C012000FF0100BE
:100D6C000A000000FC3C012000FF01000A0000000A
:100D7C00FB3C012000FF01000A000000BC3B0120ED
:100D8C000000F40101000000BA3B01200000F40156
:100D9C0001000000B83B01200000F401010000003C
:100DAC00B63B01200000F40101000000B43B01201F
:100DBC000000F40101000000F63C01200064010079
:100DCC00F43C01201400E80301000000F23C012077
:100DDC00E80330750A000000F03C012000C8010057
:100DEC00EF3C012000C80100EE3C012000C80100CE
:100DFC00ED3C0120006401000A000000843D01204C
:100E0C000000D007010000007F3D012000C8010058
:100E1C007E3D012000C801007D3D012000C801007D
:100E2C00823D01200000D007010000007C3D012024
:100E3C0000C801007B3D012000C801007A3D012063
:100E4C0000C80100803D01200000D0070100000017
:100E5C00793D012000C80100783D012000C8010047
:100E6C00773D012000C80100F415050800000000C2
:100E7C00000000000000000000000000A4E90408CD
:100E8C000900000000000000F8020120040000002E
:100E9C00ACE904080900000000000000EC0201208D
:100EAC0004000000481D05080900000000000000B7
:100EBC00E002012004000000DC130508090000001A
:100ECC0000000000D40201200400000004160508F4
:100EDC000900000000000000C8020120040000000E
:100EEC000C1605080900000000000000BC020120DF
:100EFC0004000000141605080900000000000000A2
:100F0C00B0020120040000001C16050809000000B6
:100F1C0000000000A402012004000000CC1505080C
:100F2C0001000000000000000000000000000000B4
:100F3C00000000000E000000000000000000000097
:100F4C00000000001418050800000000000000005C
:100F5C000000000000000000D40705080700000096
:100F6C00000000001C0301200000000024180508EC
:100F7C000800000000000000100301200000000029
:100F8C0030180508080000000000000004030120D0
:100F9C0000000000CC150508010000000000000056
:100FAC000000000000000000000000000E00000027
:100FBC0000000000000000000000000038180508C8
:100FCC000000000000000000000000000000000015
:100FDC00481805080D00000000000000580301200F
:100FEC0000000000501805080D0000000000000073
:100FFC004C030120000000005818050807000000F1
:10100C0000000000440301200000000060180508E7
:10101C000D0000000000000038030120000000005B
:10102C00681805080D000000000000002C030120CA
:10103C000000000070180508070000000000000008
:10104C002403012000000000CC150508010000005D
:10105C000000000000000000000000000000000084
:10106C000E00000000000000000000000000000066
:10107C0078180508000000000000000000000000C7
:10108C0000000000D40705080C0000000000000060
:10109C00563B0120000000008C1805080C000000D5
:1010AC0000000000583B0120000000009C180508BF
:1010BC000C000000000000008E3B0120000000002E
:1010CC00AC1805080C00000000000000823B012059
:1010DC0000000000C01805080C0000000000000013
:1010EC005A3B012000000000CC1805080C00000041
:1010FC00000000005C3B012000000000D418050833
:10110C000C000000000000005E3B0120000000000D
:10111C00E81805080C00000000000000603B0120EE
:10112C0000000000F01805080C0000000000000092
:10113C00623B012000000000F81805080C000000BC
:10114C0000000000A03B0120000000001019050861
:10115C000C00000000000000643B012000000000B7
:10116C001C1905080C00000000000000663B012063
:10117C0000000000B4E904080C00000000000000AE
:10118C00683B012000000000241905080C00000039
:10119C00000000006A3B0120000000003019050827
:1011AC000C000000000000006C3B0120000000005F
:1011BC000C1505080C000000000000006E3B01201F
:1011CC00000000003C1905080C00000000000000A5
:1011DC00703B012000000000481905080C000000BD
:1011EC0000000000723B01200000000054190508AB
:1011FC000C00000000000000863B012000000000F5
:10120C005C1905080C00000000000000843B012064
:10121C0000000000641905080C000000000000002C
:10122C00923B012000000000701905080C00000022
:10123C0000000000943B0120000000007C19050810
:10124C000C000000000000009A3B01200000000090
:10125C00B81605080C00000000000000743B0120CB
:10126C0000000000881905080C00000000000000B8
:10127C007C3B012000000000901905080C000000C8
:10128C0000000000763B0120000000009C190508BE
:10129C000C00000000000000783B01200000000062
:1012AC00A81905080C000000000000007A3B012082
:1012BC0000000000B01905080C0000000000000040
:1012CC007E3B012000000000F40705080C00000024
:1012DC0000000000883B012000000000BC1905083C
:1012EC000C00000000000000803B0120000000000A
:1012FC007B1405080C00000000000000903B01204E
:10130C0000000000C81905080C00000000000000D7
:10131C008A3B012000000000D01905080C000000D9
:10132C00000000008C3B012000000000D8190508CB
:10133C000C00000000000000963B012000000000A3
:10134C00E01905080C00000000000000983B01208B
:10135C0000000000E81905080C0000000000000067
:10136C00AA3B012000000000CC150508010000007C
:10137C000000000000000000000000000000000061
:10138C000E00000000000000000000000000000043
:10139C00F01905080000000000000000000000002B
:1013AC0000000000FC1905080D0000000000000002
:1013BC00B003012000000000041A05080D00000015
:1013CC0000000000A4030120000000000C1A050816
:1013DC0007000000000000009C030120000000003A
:1013EC00181A0508070000000000000094030120F3
:1013FC0000000000241A050809000000000000008D
:10140C008803012000000000301A050809000000C4
:10141C00000000007C030120000000003C1A0508BD
:10142C000900000000000000700301200000000013
:10143C004C1A05080900000000000000640301209C
:10144C0000000000CC1505080100000000000000A1
:10145C000000000000000000000000000E00000072
:10146C00000000000000000000000000601A0508E9
:10147C000000000000000000000000000000000060
:10148C00701A05080500000000000000B13B0120A7
:10149C0000000000CC150508010000000000000051
:1014AC000000000000000000000000000E00000022
:1014BC00000000000000000000000000781A050881
:1014CC000000000000000000000000000000000010
:1014DC00841505080000000000000000DD1E01203E
:1014EC0004000000D81305080D000000FD410108A0
:1014FC000404012000000000C01F05080D000000BE
:10150C00111B0108F8030120000000002819050830
:10151C000D000000F51A0108EC030120000000008A
:10152C00841A05080800000000000000E0030120F8
:10153C0004000000881905080D0000003F1A01087E
:10154C00D4030120000000008C1A050809000000DB
:10155C0000000000C803012004000000381A050830
:10156C00030000000D230108BC0301200000000053
:10157C00CC15050801000000000000000000000070
:10158C0000000000000000000E0000000000000041
:10159C000000000000000000941A05080000000084
:1015AC00000000000000000000000000A41A050864
:1015BC000D000000000000001C04012000000000D1
:1015CC00AC1A05080A00000000000000243E0120AF
:1015DC0000000000B81A05080A0000000000000016
:1015EC002C3E012000000000C01A05080A00000073
:1015FC0000000000343E012000000000C81A05085D
:10160C000800000000000000100401200000000091
:10161C00D01A0508040000008945010800000000EC
:10162C0000000000CC1505080100000000000000BF
:10163C000000000000000000000000000E00000090
:10164C00000000000000000000000000DC1A05088B
:10165C00000000000000000000000000000000007E
:10166C00F01A05080D0000000000000034040120F1
:10167C0000000000001B0508040000007544010870
:10168C000000000000000000081B05080D00000011
:10169C000000000028040120000000001C1B0508AD
:1016AC00040000005144010800000000000000008C
:1016BC00CC1505080100000000000000000000002F
:1016CC0000000000000000000E0000000000000000
:1016DC000000000000000000241B050800000000B2
:1016EC00000000000000000000000000381B05088E
:1016FC0008000000000000007C0401200000000035
:10170C00441B0508080000000000000070040120C4
:10171C0000000000501B050808000000000000003D
:10172C0064040120000000005C1B05080800000098
:10173C00000000005804012000000000681B050890
:10174C0008000000000000004C0401200000000014
:10175C00741B050808000000000000004004012074
:10176C0000000000CC15050801000000000000007E
:10177C000000000000000000000000000E0000004F
:10178C00000000000000000000000000801B0508A5
:10179C000000000000000000FB0101200000000020
:1017AC008C1B05080B000000000000001005012038
:1017BC0000000000981B05080B0000000000000052
:1017CC000405012000000000A41B05080B0000000C
:1017DC0000000000F804012000000000B01B050808
:1017EC000B00000000000000EC04012000000000D1
:1017FC00BC1B05080B00000000000000E0040120E9
:10180C0000000000C81B05080B00000000000000D1
:10181C00D404012000000000D41B05080B000000BC
:10182C0000000000C804012000000000E01B0508B7
:10183C000B00000000000000BC04012000000000B0
:10184C00EC1B05080B00000000000000B004012098
:10185C0000000000F81B0508070000000000000055
:10186C00A804012000000000001C0508070000006F
:10187C0000000000A0040120000000000C1C050862
:10188C000B00000000000000940401200000000088
:10189C00181C050808000000000000008804012046
:1018AC0000000000CC15050801000000000000003D
:1018BC000000000000000000000000000E0000000E
:1018CC00000000000000000000000000241C0508BF
:1018DC0000000000000000000000000000000000FC
:1018EC00381C050808000000000000004C05012011
:1018FC0000000000441C0508080000000000000067
:10190C004005012000000000501C050808000000E4
:10191C000000000034050120000000005C1C0508DC
:10192C000800000000000000280501200000000055
:10193C00681C050808000000000000001C050120C0
:10194C0000000000CC15050801000000000000009C
:10195C000000000000000000000000000E0000006D
:10196C00000000000000000000000000701C0508D2
:10197C000000000000000000F80101200000000041
:10198C00801C05080B0000000000000090050120E1
:10199C00000000008C1C050807000000000000007F
:1019AC008805012000000000981C050807000000B5
:1019BC00000000008005012000000000A41C0508A8
:1019CC000700000000000000780501200000000066
:1019DC00B01C050808000000000000006C05012088
:1019EC0000000000B81C0508080000000000000002
:1019FC006005012000000000C01C05080700000065
:101A0C00000000005805012000000000CC1505085E
:101A1C0001000000000000000000000000000000B9
:101A2C00000000000E00000000000000000000009C
:101A3C0000000000CC1C05080000000000000000A5
:101A4C00F801012000000000D81C05080700000068
:101A5C00000000000006012000000000E01C05084A
:101A6C000700000000000000F80501200000000045
:101A7C00E81C05080700000000000000F00501202C
:101A8C0000000000F01C0508080000000000000029
:101A9C00E405012000000000F81C05080700000008
:101AAC0000000000DC05012000000000001D0508FE
:101ABC000700000000000000D40501200000000019
:101ACC00081D05080700000000000000CC050120DF
:101ADC0000000000101D05080800000000000000B8
:101AEC00C005012000000000181D050807000000BB
:101AFC0000000000B805012000000000201D0508B2
:101B0C000700000000000000B005012000000000EC
:101B1C00281D05080700000000000000A805012092
:101B2C0000000000301D0508080000000000000047
:101B3C009C05012000000000CC15050801000000E8
:101B4C000000000000000000000000000000000089
:101B5C000E0000000000000000000000000000006B
:101B6C0000000000711E010808060120AF3B012097
:101B7C002B000000A4B40408AE3B012000C80100F7
:101B8C00AC3B0120E803D007010000004D414D4261
:101B9C004146373232000000493B0120000301006E
:101BAC00483B012000030100BD1D0108991D0108DF
:101BBC00E4060120591D0108111D01085C070120D4
:101BCC00F91D0108E11D0108100801207D1C010808
:101BDC00311C0108300B0120871E0108214401082B
:101BEC000C0C01207D1A0108000000005C0C012087
:101BFC008925010825210108380D0120AD1E010899
:101C0C0000000000EC0D0120651F0108311F0108C8
:101C1C00780E0120F51F0108412001082C0F01202E
:101C2C00F73C012001060100F51E0108C11E010848
:101C3C006C100120991F0108994401080C11012016
:101C4C0071200108F5440108D4110120EC3C01205D
:101C5C0001030100381D0508000000000000000011
:101C6C000000000000000000441D050808000000F2
:101C7C000000000020130120000000004C1D05088E
:101C8C0007000000000000001813012000000000F5
:101C9C005C1D05080D000000000000000C13012065
:101CAC0000000000681D0508030000000D2301085A
:101CBC000013012000000000CC15050801000000F5
:101CCC000000000000000000000000000000000008
:101CDC000E000000000000000000000000000000EA
:101CEC00701D05080000000000000000000000004E
:101CFC0000000000801D05080A0000000000000024
:101D0C00881D050800000000901D05080A00000051
:101D1C0000000000981D050800000000A01D05082B
:101D2C000A00000000000000863D012000000000B9
:101D3C00A81D05080A000000000000002C1301205B
:101D4C0000000000CC150508010000000000000098
:101D5C000000000000000000000000000E00000069
:101D6C00000000000000000000000000B01D05088D
:101D7C000000000000000000000000000000000057
:101D8C00BC1D0508030000000D2301086013012091
:101D9C0000000000C81D0508030000000D23010809
:101DAC005413012000000000D01D050803000000A2
:101DBC000D2301084813012000000000D81D050860
:101DCC000500000000000000473B0120000000005F
:101DDC00E01D050807000000000000004013012072
:101DEC0000000000EC1D05080700000000000000CA
:101DFC003813012000000000CC150508010000007C
:101E0C0000000000000000000000000000000000C6
:101E1C000E000000000000000000000000000000A8
:101E2C00F81D050800000000000000000000000084
:101E3C000000000027150508030000000D23010811
:101E4C0090130120000000000C1E05080300000088
:101E5C000D2301082000012000000000141E0508BD
:101E6C00030000000D230108841301200000000072
:101E7C001C1E0508030000000D2301087813012027
:101E8C000000000088190508030000000D2301085C
:101E9C006C13012000000000CC15050801000000A7
:101EAC000000000000000000000000000000000026
:101EBC000E00000000000000000000000000000008
:101ECC00281E0508000000000000000000000000B3
:101EDC0000000000381E05080700000051450108ED
:101EEC00EC13012000000000AC19050803000000F1
:101EFC000D230108E013012000000000441E05081A
:101F0C00030000000D230108D41301200000000081
:101F1C004C1E0508030000000D230108C813012006
:101F2C0000000000541E050807000000354501089C
:101F3C00C01301200000000044220508030000002B
:101F4C000D230108B413012000000000601E0508D9
:101F5C00030000000D230108A8130120000000005D
:101F6C006C1E0508030000000D2301089C130120C2
:101F7C0000000000CC150508010000000000000066
:101F8C000000000000000000000000000E00000037
:101F9C00000000000000000000000000411E0108CD
:101FAC00111E0108F4130120F120010800000000AB
:101FBC0080140120ED1C0108C91C01080C1501201E
:101FCC000000000000000000C0150120C92001081D
:101FDC006D45010860160120781E05080000000000
:101FEC00000000000000000000000000841E050836
:101FFC00030000000D2301086C17012000000000F5
:10200C008C1E0508030000000D2301086017012039
:10201C0000000000EC080508030000000D23010877
:10202C005417012000000000981E05080300000052
:10203C000D2301084817012000000000A41E05080C
:10204C00030000000D2301083C17012000000000D4
:10205C00AC1E050802000000DD4501080000000070
:10206C0000000000B41E050802000000DD45010858
:10207C000100000000000000C01E05080200000066
:10208C00DD45010802000000000000000000000017
:10209C000E00000000000000000000000000000026
:1020AC00263B012088136F1701000000283B0120FC
:1020BC0088136F1700000000CC1E050800000000FC
:1020CC00000000000000000000000000DC1E0508FD
:1020DC0008000000000000004C1801200400000063
:1020EC00E81E050808000000000000004018012050
:1020FC0000000000381A0508040000002542010801
:10210C000000000000000000CC15050801000000D4
:10211C0000000000000000000000000000000000B3
:10212C000E00000000000000000000000000000095
:10213C00243B012088136F1701000000D05C0120A4
:10214C0088136F1700000000C11B0108000000007D
:10215C00581801207C4101200100000054B50408EE
:10216C00D25C01200100000060B50408C85C0120AD
:10217C000200000068B50408FEBB0120000000004E
:10218C0000000000FCBB012000000000000000006B
:10219C00FABB01200000000000000000F8BB012089
:1021AC000000000000000000F6BB01200000000051
:1021BC0000000000F4BB0120000000000000000043
:1021CC00181F01200000000000000000233B01202C
:1021DC000200000074B50408241F0508000000006C
:1021EC00000000000000000000000000DC1E0508DC
:1021FC000800000000000000DC18012004000000B2
:10220C00E81E05080800000000000000D01801209E
:10221C0000000000381A050804000000911B01089A
:10222C000000000000000000CC15050801000000B3
:10223C000000000000000000000000000000000092
:10224C000E00000000000000000000000000000074
:10225C00341F050800000000000000000000000012
:10226C0000000000441F05080D0000007543010824
:10227C000C19012004000000501F05080D0000007F
:10228C00E91B010800190120040000005C1F05086F
:10229C000D00000039430108F41801200000000073
:1022AC00681F05080300000095240108E8180120A8
:1022BC0008000000741F0508030000000D2301082E
:1022CC00101C012000000000CC15050801000000C6
:1022DC0000000000000000000000000000000000F2
:1022EC000E000000000000000000000000000000D4
:1022FC00C4150508000000000000000000000000EC
:10230C00000000002A130508040000003D420108EB
:10231C000000000000000000CC15050801000000C2
:10232C0000000000000000000000000000000000A1
:10233C000E00000000000000000000000000000083
:10234C00C81F05080000000000000000000000008D
:10235C0000000000582C05080D00000000000000D3
:10236C006C19012004000000D81F050808000000AB
:10237C00000000006019012004000000E41F0508A3
:10238C0008000000000000005419012004000000A7
:10239C00EC1F05080800000000000000481901208F
:1023AC0004000000F41F05080800000000000000F5
:1023BC003C19012004000000FC1F05080800000067
:1023CC000000000030190120040000000420050862
:1023DC000800000000000000241901200400000087
:1023EC000C2005080800000000000000181901204E
:1023FC0004000000CC1505080100000000000000DE
:10240C000000000000000000000000000E000000B2
:10241C00000000000000000000000000A91B0108E3
:10242C0000000000781901200000000000000000EE
:10243C00F01901200000000000000000901A01209B
:10244C00CE5C01200400000080B50408CC5C0120A7
:10245C00E0150C1700000000CB5C01200800000008
:10246C0090B60408CA5C01200500000094B504086D
:10247C000000000000000000E01A012000C2010072
:10248C00000008001A03000000000000000000001B
:10249C000000000000000000000000000000000030
:1024AC0004030904120100020000004083042A57AF
:1024BC0000020102030100001201000202000040B0
:1024CC0083044057000201020301000012010002C4
:1024DC00EF020140830456320002010203010000A6
:1024EC000A0600020000004001000000090720005D
:1024FC00010104C03209040000020806500507055A
:10250C008102400000070501024000000902200082
:10251C00010104C032090400000208065005070539
:10252C008102400000070501024000000902200062
:10253C00010104C032090400000208065005070519
:10254C008102000200070501020002000A060002D7
:10255C00000000400100000009026400030100C0FB
:10256C0032090400000103000000092111010001DF
:10257C002226000705830308000A080B0102020249
:10258C0001000904010001020201000524001001F0
:10259C000524010002042402020524060102070599
:1025AC0082030800FF09040200020A00000007056C
:1025BC00010240000007058102400000C3B0010881
:1025CC0047A4010815D8010800000000AD960108C9
:1025DC000B970108D99601080000000000000000CC
:1025EC000000000095960108A19601088996010843
:1025FC007D9601080A060002000000400100000060
:10260C0009022200010100E032090400000103016B
:10261C00020009211101000122260007058303088D
:10262C00000A00000A060002000000400100000041
:10263C0009074300020104C0320904000001020230
:10264C0001000524001001052401000104240202EC
:10265C000524060001070582030800FF0904010098
:10266C00020A000000070501024000000705810274
:10267C004000000009024300020100C032090400BE
:10268C0000010202010005240010010524010001D3
:10269C000424020205240600010705820308001029
:1026AC0009040100020A00000007050102000200F3
:1026BC00070581020002000009024300020100C06C
:1026CC00320904000001020201000524001001057A
:1026DC0024010001042402020524060001070582DE
:1026EC000308001009040100020A0000000705019C
:1026FC0002400000070581024000000000FFFF00BF
:10270C0000000000AA5505010000010005010905A3
:10271C00A101A1000501093009310932093309353C
:10272C000934094009381581257F750895088102FF
:10273C00C0C000000921110100012226002D202D0E
:10274C002D202D2D2D2D202D2D2D2D0000000000A8
:10275C00000000000000000000000000AA550B0162
:10276C000000AA5507010000AA550902000000AAA2
:10277C005503009F01000000C0120000FF1FFF1F47
:10278C00245F012000000000301F01200400000025
:10279C00000200051002700B010102FFFF00000097
:1027AC00010000000000803FFF000000000000005E
:1027BC00D46C01200800000000000000C46C012053
:1027CC00080000003996010819960108D5950108F2
:1027DC0000000000C9950108B5950108A1950108F4
:1027EC0000000000000000000000000000000000DD
:1027FC0095950108000000008995010819950108BC
:10280C000D950108C5A30108D9A30108C5940108B9
:10281C00B1A301089BA3010835DB01089D930108B6
:10282C001D9301080593010834C40408050804002D
:10283C000000000094B5040890B6040880B50408A4
:10284C00000000000000000060C4040805080A0035
:10285C000000000094B5040890B6040860B40408A5
:10286C0000000000000000002DB00108FDA30108CD
:10287C0011D60108000000000000000011C801087A
:10288C000DC701080000000000000000000000005F
:10289C007D95010871950108659501085995010808
:1028AC009D4D0308FD3B0308F93B0308F53B03086A
:1028BC00B13F0308F13B0308ED3B030878C604085D
:1028CC0001000000B001000002000000090000003F
:1028DC001000000000600240106002400000000088
:1028EC0000000000000B00000000000000000000D1
:1028FC00000000000060024028600240010000005F
:10290C0000000000060C00000000000000000000A9
:10291C000000000000600240406002400200000025
:10292C0000000000100D000000000000000000007E
:10293C0000000000006002405860024003000000EC
:10294C0000000000160E0000000000000000000057
:10295C0000000000006002407060024004000000B3
:10296C0000000000200F000000000000000000002C
:10297C00000000000060024088600240050000007A
:10298C000000000026100000000000000000000005
:10299C000000000000600240A06002400600000041
:1029AC0000000000301100000000000000000000DA
:1029BC000000000000600240B86002400700000008
:1029CC0000000000362F0000000000000000000096
:1029DC00000000000064024010640240000000008F
:1029EC0000000000003800000000000000000000A3
:1029FC000000000000640240286402400100000056
:102A0C00000000000639000000000000000000007B
:102A1C00000000000064024040640240020000001C
:102A2C0000000000103A0000000000000000000050
:102A3C0000000000006402405864024003000000E3
:102A4C0000000000163B0000000000000000000029
:102A5C0000000000006402407064024004000000AA
:102A6C0000000000203C00000000000000000000FE
:102A7C000000000000640240886402400500000071
:102A8C0000000000264400000000000000000000D0
:102A9C000000000000640240A06402400600000038
:102AAC0000000000304500000000000000000000A5
:102ABC000000000000640240B864024007000000FF
:102ACC00000000003646000000000000000000007E
:102ADC00000000000101000020080508F022050894
:102AEC0000000000B1E50208A0860100040000000F
:102AFC0000000000000000000000000000000000CA
:102B0C000000000000000000000000002008050884
:102B1C00342D05080000000005FE0108E803000044
:102B2C000400000000000000000000000000000095
:102B3C000000000000000000000000000000000089
:102B4C00AC190508C0E9040800000000FD030000F2
:102B5C007D000000060000000000000000000000E6
:102B6C000000000000000000000000000000000059
:102B7C0000000000780705080000000000000000BD
:102B8C00D12A0208E8030000030000000000000046
:102B9C000000000000000000000000000000000029
:102BAC0000000000000000003C2D050800000000A3
:102BBC000000000095F80308102700000300000037
:102BCC0000000000000000000000000000000000F9
:102BDC00000000000000000000000000482D050867
:102BEC000000000081990008793202085F7600002D
:102BFC0005000000000000000000000000000000C4
:102C0C0000000000000000000000000000000000B8
:102C1C00E0090508000000000000000071470208F0
:102C2C001027000001000000000000000000000060
:102C3C000000000000000000000000000000000088
:102C4C00000000004C2D05080000000000000000F2
:102C5C0009FE0108E8030000050000000000000068
:102C6C000000000000000000000000000000000058
:102C7C000000000000000000582D050800000000B6
:102C8C0000000000C9EE0208204E00000300000006
:102C9C000000000000000000000000000000000028
:102CAC00000000000000000000000000682D050876
:102CBC000000000000000000C5EC0208204E0000DF
:102CCC0003000000000000000000000000000000F5
:102CDC0000000000000000000000000000000000E8
:102CEC00782D05080000000000000000A103020878
:102CFC00400D030003000000000000000000000075
:102D0C0000000000000000000000000000000000B7
:102D1C0000000000E40805080000000000000000AE
:102D2C0095F70208102700000100000000000000C9
:102D3C000000000000000000000000000000000087
:102D4C0000000000000000009007050800000000D3
:102D5C00000000003D5E0108102700000300000089
:102D6C000000000000000000000000000000000057
:102D7C00000000000000000000000000B81605086C
:102D8C0000000000000000001DFD0108A86100000B
:102D9C000100000000000000000000000000000026
:102DAC000000000000000000000000000000000017
:102DBC00E80905080000000000000000C94F0208E7
:102DCC00A00F000001000000000000000000000047
:102DDC0000000000000000000000000000000000E7
:102DEC0000000000882D0508000000000000000015
:102DFC00913D0108102700000100000000000000B8
:102E0C0000000000000000000000000000000000B6
:102E1C000000000000000000EC08050800000000A5
:102E2C00000000005D8A01081A410000010000004A
:102E3C000000000000000000000000000000000086
:102E4C00000000000000000000000000480A050817
:102E5C000000000000000000219F01081027000066
:102E6C000100000000000000000000000000000055
:102E7C000000000000000000000000000000000046
:102E8C000423050800000000000000006147010851
:102E9C001A410000010000000000000000000000CA
:102EAC000000000000000000000000000000000016
:102EBC0000000000942D0508000000000000000038
:102ECC0079E60108400D030000000000000000003E
:102EDC0000000000000000000000000000000000E6
:102EEC0000000000000000009C2D05080000000000
:102EFC0000000000D9FC0108400D03000000000098
:102F0C0000000000000000000000000000000000B5
:102F1C00000000000000000000000000A42D0508C7
:102F2C000000000000000000F16B010850C300001D
:102F3C000300000000000000000000000000000082
:102F4C000000000000000000000000000000000075
:102F5C00B02D050800000000000000003DEC020848
:102F6C0040420F00000000000000000000000000C4
:102F7C000000000000000000000000000000000045
:102F8C0000000000BC2D050800000000000000003F
:102F9C003DE7020850C300000000000000000000E4
:102FAC000000000000000000000000000000000015
:102FBC0000000000000000000000803F0000000046
:102FCC0000000000000000000000803F0000000036
:102FDC0000000000000000000000000000000000E5
:102FEC0000000000000000000000000000000000D5
:102FFC00010000000000803F000000000000000005
:10300C00000000000000803F0000000000000000F5
:10301C000000000001000000BC270120000000009F
:10302C000000000000000000000000000000000094
:10303C000000000000000000000000000000000084
:10304C000000000000000000000000000000000074
:10305C000000000000000000000000000000000064
:10306C000000000000000000000000000000000054
:0C307C0000000000000000000000000048
:083088000000803F0000803FC2
:10800000002301228370C270038003714371837166
:10801000C37103724372704700230A2203604360F6
:10802000C381C0F80630C0F80A300280704700BF34
:108030002DE9F84F704CE279237A9A427FD0E279A9
:10804000E379C2EBC202C3EBC30304EB820204EB8D
:10805000830392F82B101E7C8B1E9E422CD0B4F80A
:108060006430664A0133E16812789BB21B2AA4F897
:10807000643067D00025E379614A0133A2FB030233
:10808000520802EB42029B1ADBB2E37100293BD09B
:1080900018F0EAFFD4F89830C01AB0F5FA7F04DB84
:1080A000002345F0040584F89630D4F89030002B76
:1080B00032D12846BDE8F88FE37904F11007C3EB0D
:1080C000C30307EB830361B10022194413F8015B7A
:1080D0002A44994292B2F9D1D3B203EB1222FF2A79
:1080E00038D0B4F86430454A0133E16812789BB265
:1080F0001B2AA4F86430BDD1424B0422B4F86400BA
:1081000000259A805880B6E794F89630002BBFD1AE
:10811000D4F89030002BCCD03B4A1268D31AB3F578
:10812000FA7FC6D994F86630032B02D10023A4F855
:108130008C3000232846C4F89030BDE8F88FE16801
:108140000025A3E72F4B0322B4F8640000259A8092
:10815000588090E7E3791C21012201FB0323FD5C99
:108160001F445DB3954215D1082E3CD0B4F864305D
:10817000224A0133E16812789BB21B2AA4F86430CA
:108180007FF478AF1F4B0622B4F8640000259A8074
:10819000588070E7B4F86430184A0133E168127807
:1081A0009BB21B2AA4F864307FF464AF154B052200
:1081B000B4F8640000259A8058805CE7192EE168C5
:1081C00024D0B4F864300D4A013312789BB21B2AD4
:1081D000A4F864307FF44FAF0A4B0622B4F8640071
:1081E0009A80588047E794F89430002B40F0EA805A
:1081F0001D46E1683FE700BF202801206D9C01205B
:10820000ABAAAAAA709C012058A1012097F803806C
:1082100040F2147CBE7808F03F087A7897F802B0F4
:1082200006F007064FEA4818036997F804A042EAE7
:10823000062048EADB08BA7A97F806904FEA8A0ADD
:1082400097F807E002F01F023D7A09F00F09188045
:108250009601B87B6D00A3F802804FEAC91997F820
:10826000038000F03F020EF07F0E4AEA981897F85C
:1082700005A05001FA790AF0010A4FEA0E1E45EAFC
:10828000D2157A7A48EA8A2802F00302A3F8048019
:1082900097F8058045EA4222FD7A49EA580997F89D
:1082A0000D80ED00A3F8069008F0070897F80690F7
:1082B0005A817A7A4EEA191E46EA9202BE7AA3F8E9
:1082C00008E09A8145EA56127E7B3D7BDA8140EADE
:1082D000D60245EA08251D825A82F87BBD7B97F8B5
:1082E0001080800097F811E0FA7C40EA951008F0C1
:1082F00001080EF00F0E5200BE7C40EA882097F86D
:10830000128097F810904FEACE1E42EAD81297F8E2
:1083100014807D7D4EEA590E06F07F0608F00308B2
:10832000988205F01F05B87D42EA4822A3F816E0BE
:10833000360197F811E0AD015A83C0007A7D46EA14
:108340001E1697F814E040EA52101E8345EA9E0577
:10835000D8839D83F87D10F0010F14BF6546AD25CD
:1083600010F0020F1D8414BF6246AD225A84030729
:108370004ED410F0040F0CBF0125092594F8663087
:10838000032B1AD194F867203B7E04EB42062C4F56
:10839000C3EB8323501CA7FB0323A26EB6F86C70BB
:1083A00000F00F005B09D21B84F86700A6F86C3060
:1083B00013441A09A366A4F88C20224B1B68C4F846
:1083C000903058E67B78102B24D013D86BBB94F8F0
:1083D0009530E168002B7FF44DAE94F89730012B77
:1083E00026D919B10A78303A012A21D9002584F812
:1083F000975040E6303B012B17D857F8010F002566
:10840000E460BA88BB7910492060A280A37132E68B
:108410000325B3E794F895300BB984F89550012300
:10842000E168002584F8963025E6E168002522E61B
:1084300001330122002584F8973084F896201AE64B
:108440001F85EB5158A101202028012038B5044692
:1084500018F00AFE524B002283F89C2093F89D20CE
:10846000012A19D9D3F8A02040F6AC51821A8A42C9
:1084700012DDB3F864204B490132097892B21B290E
:10848000A3F8642005D1484A0121B3F864509180D3
:108490005580002283F89D20E2B27E2A25D093F8F1
:1084A0009D1009B393F89D101B2954D893F8AC1074
:1084B00000296AD0002182F0200283F8AC1093F8E2
:1084C0009D10022901D1012A65D0197A93F89D40A7
:1084D000C1EBC10193F89D0003EB81010130214400
:1084E000C0B2CA7383F89D0038BD93F89D20012A5D
:1084F0002BD91A7A2D490132DC79A1FB02514908A6
:1085000001EB4101521AD2B294420AD093F89D4035
:10851000197A013C1A72C1EBC10103EB810181F8A8
:108520002B4093F8A4203AB10121002283F89C103B
:1085300083F8A420C3F898001A4A12781B2A1ED088
:108540000022C3F8A80083F8AC200122C3F8A000E1
:1085500083F89D2038BD0022124983F89D20B3F88E
:108560006420097801321B2992B2A3F86420BBD1A0
:10857000B3F8641002220C4B59809A8038BDD3F8AE
:10858000A8200949821A0A80DAE77D2A97D10122B8
:1085900083F8AC2038BD012183F8A41095E700BF13
:1085A000202801206D9C0120709C0120ABAAAAAA62
:1085B00003788B4205D9044B03EB4101B1F8B000BD
:1085C00070470020704700BF20280120044B93F81B
:1085D000C80018B10022012083F8C820704700BFEE
:1085E00020280120F0B4C94D05F1CC0295F8EF60C8
:1085F0000244B41E1444A24200F08681013A013CB8
:10860000002341F2210112F8017F83EA07231FB200
:10861000BBB2002FACBF5B0081EA43039BB21F04D7
:1086200054BF5B0081EA43039BB21F0454BF5B004D
:1086300081EA43039BB21F0454BF5B0081EA4303FA
:108640009BB21F0454BF5B0081EA43039BB21F042B
:1086500054BF5B0081EA43039BB21F0454BF5B001D
:1086600081EA43039BB21F0454BF5B0081EA4303CA
:10867000A2429BB2C7D10644B21E013E2A442E44F8
:1086800092F8CC1096F8CC2002EB012292B29A42DA
:1086900001D0F0BC704795F8F020002A00F02F813F
:1086A000431C4FF4AF61012ADBB203F101042B44F8
:1086B0002C4493F8CC6094F8CC3003EB06239BB2A7
:1086C00001FB03F34FEA233303F54873A5F8B030F9
:1086D00000F01581C31C022ADBB203F101042B4414
:1086E0002C4493F8CC6094F8CC3003EB06239BB277
:1086F00001FB03F34FEA233303F54873A5F8B230C7
:1087000000F0FD80431D032ADBB203F101042B447A
:108710002C4493F8CC6094F8CC3003EB06239BB246
:1087200001FB03F34FEA233303F54873A5F8B43094
:1087300000F0E580C31D042ADBB203F101042B44E1
:108740002C4493F8CC6094F8CC3003EB06239BB216
:1087500001FB03F34FEA233303F54873A5F8B63062
:1087600000F0CD8000F10903052ADBB203F101041A
:108770002B442C4493F8CC6094F8CC3003EB0623C4
:108780009BB201FB03F34FEA233303F54873A5F8CB
:10879000B83000F0B48000F10B03062ADBB203F11D
:1087A00001042B442C4493F8CC6094F8CC3003EBB8
:1087B00006239BB201FB03F34FEA233303F548730F
:1087C000A5F8BA3000F09B8000F10D03072ADBB258
:1087D00003F101042B442C4493F8CC6094F8CC3082
:1087E00003EB06239BB201FB03F34FEA233303F5AC
:1087F0004873A5F8BC3000F0828000F10F03082A0E
:10880000DBB203F101042B442C4493F8CC6094F8C0
:10881000CC3003EB06239BB201FB03F34FEA233377
:1088200003F54873A5F8BE3069D000F11103092A99
:10883000DBB203F101042B442C4493F8CC6094F890
:10884000CC3003EB06239BB201FB03F34FEA233347
:1088500003F54873A5F8C03051D000F113030A2A7C
:10886000DBB203F101042B442C4493F8CC6094F860
:10887000CC3003EB06239BB201FB03F34FEA233317
:1088800003F54873A5F8C23039D000F115030B2A5F
:10889000DBB203F101042B442C4493F8CC6094F830
:1088A000CC3003EB06239BB201FB03F34FEA2333E7
:1088B00003F54873A5F8C43021D000F117030C2A42
:1088C000DBB203F101042B442C4493F8CC6094F800
:1088D000CC3003EB06239BB201FB03F34FEA2333B7
:1088E00003F54873A5F8C63009D000F11903DBB2CF
:1088F0005A1C2B44154493F8CC3095F8CC30012306
:1089000085F8C830F0BC70470023B4E62028012069
:1089100070B5594C064618F0A7FBD4F8F430C4F8EB
:10892000F400C01AB0F5FA5F1AD9002384F8F830C1
:1089300084F8F930A12E2FD0A22E00F0948094F864
:10894000F920002594F8EF30A2B1691C6219F6B243
:10895000CDB282F8CC609D4284F8F8500CD070BD46
:1089600094F8F850002DE5D094F8F92094F8EF3001
:10897000002AEAD19D42F2D194F8FA30052B6AD050
:10898000062B03D194F8CD301E2B0ED0002384F893
:10899000F93084F8F83070BD01231B2284F8F930D7
:1089A000134684F8EF200025CFE7691E0022002936
:1089B00048DD10461346234493F8CC30DBB283EAFB
:1089C00002055B08ED0748BF83F08C0383EA52057C
:1089D0005B08EE0748BF83F08C0383EA92055B08CF
:1089E000ED0702D583F08C03DBB283EAD2055B0886
:1089F000EE0702D583F08C03DBB283EA12155B0825
:108A0000ED0702D583F08C03DBB283EA52155B08D5
:108A1000EE0702D583F08C03DBB283EA92155B0884
:108A2000ED0702D583F08C03DBB283EAD2155A0836
:108A3000EB0702D582F08C02D2B20130C0B2814283
:108A40000346B8DC214491F8CC3093429ED10320F8
:108A5000FFF7C8FD9AE70020FFF7C4FD94F8CD307A
:108A60001E2B93D1A1E70123232284F8F93013466A
:108A700084F8EF2097E700BF20280120072905D8B8
:108A8000034B03EB8101B1F8FC00704700207047F5
:108A9000202801201A4B93F81C2132B193F8202191
:108AA0000021A82A83F81C1101D00020704793F8F8
:108AB0003321002AF9D1F4EE046A03F5907103F131
:108AC000F80003F598729FED0F7A10B4CC78B0EEF1
:108AD000476A0B79023103EB04238A4207EE903A8E
:108AE000F8EEE77AA7EEA66AFCEEC67A17EE903AA1
:108AF00040F8043FEAD101205DF8044B704700BF05
:108B0000202801200080BBC310B5044618F0ACFA41
:108B10000F4B41F28832E4B2D3F83811C3F8380170
:108B2000401A904205D9012283F8204183F83C2164
:108B300010BD93F83C219918142A81F8204103D1E3
:108B4000012283F81C2110BD0132D2B2EEE700BF32
:108B500020280120034B03EB4101B1F84001C0087C
:108B6000704700BF20280120724B93F86021002A33
:108B700000F0C280002070B493F86141B3F86251F4
:108B800003EB440183F8600191F8676191F8682173
:108B900042EA0622954202D0002070BC704793F84A
:108BA0006521012A00F0AA80812AF6D10320102C29
:108BB00040F2A68093F86721102493F8681193F887
:108BC000695141EA022193F86A2183F8614142EA3E
:108BD0000522A3F84011A3F8422193F86B11032C4E
:108BE00093F86C2142EA0122A3F84421D5D093F8EE
:108BF0006D11042C93F86E2142EA0122A3F846215C
:108C0000CBD093F86F11052C93F8702142EA012222
:108C1000A3F84821C1D093F87111062C93F8722162
:108C200042EA0122A3F84A21B7D093F87311072C26
:108C300093F8742142EA0122A3F84C21ADD093F8B5
:108C40007511082C93F8762142EA0122A3F84E21EF
:108C5000A3D093F87711092C93F8782142EA0122E6
:108C6000A3F8502199D093F879110A2C93F87A211E
:108C700042EA0122A3F852218FD093F87B110B2CEA
:108C800093F87C2142EA0122A3F8542185D093F87D
:108C90007D110C2C93F87E2142EA0122A3F8562183
:108CA0003FF47BAF93F87F110D2C93F8802142EABB
:108CB0000122A3F858213FF470AF93F881110E2CD4
:108CC00093F8822142EA0122A3F85A213FF465AFCA
:108CD00093F88311102C93F8842142EA0122A3F81F
:108CE0005C217FF45AAF93F8851193F8862142EA0C
:108CF0000122A3F85E2150E700207047104656E796
:108D0000002C3FF44AAF93F86711012C93F86821C7
:108D100042EA0122A3F840213FF43FAF93F86911E2
:108D2000022C93F86A2142EA0122A3F842217FF43F
:108D300054AF32E72028012038B5044618F094F9E2
:108D40004D4AD2F88C31C31AB3F57A6F17D892F81E
:108D50009031C2F88C01BBB1022B21D0242B92F8A8
:108D6000611140F2868001330231DBB2490082F8A2
:108D700090318B421CDB01318B4243D038BD002344
:108D8000C2F88C0182F89031A82CF7D1002592F816
:108D90006111204682F860512B46A2F8625103E02F
:108DA000E0B2014682F86101D51885F86401DAE77E
:108DB000B2F86231E4B283EA042424B2002CA3B2F4
:108DC00027DB5B009BB21C044DD45B009BB21804F4
:108DD00043D45B009BB2190439D45B009BB21D04E1
:108DE0002FD45B009BB21C0425D45B009BB21804FB
:108DF0001BD45B009BB2190411D45B009BB2A2F898
:108E0000623138BD0021012382F8901182F860316F
:108E100038BD41F2210181EA43039BB2D3E741F21D
:108E2000210181EA43039BB2E9E741F2210181EA92
:108E300043039BB2DFE741F2210181EA43039BB286
:108E4000D5E741F2210181EA43039BB2CBE741F22E
:108E5000210181EA43039BB2C1E741F2210181EA8A
:108E600043039BB2B7E741F2210181EA43039BB27E
:108E7000ADE7E0B298E700BF20280120F8B5134D18
:108E800095F8A9210AB90120F8BD114B1C68236887
:108E90005E6A46B1204605F5CA71B047002301203D
:108EA00085F8A931F8BD05F5CA77BE1800E023683A
:108EB0009B68204698470028F9D02368204617F879
:108EC000011B1B689847B742F1D1E7E72028012032
:108ED0000045012003788B4210D9094B03EB810137
:108EE00093F8DC31D1F8AC011BB900F5777080B292
:108EF0007047400800F5777080B2704700207047D7
:108F0000202801202DE9F843D04C18F0ADF8054693
:108F100094F8DD0180B9042294F8A93153B1D4F852
:108F200000323BB1ED1AB5F57A7F03DB0023104622
:108F3000C4F80032BDE8F883002394F8DE1184F809
:108F4000DD31002900F0108194F8E031C04F5BB2B0
:108F500094F8F02113F1630FB8BF97F90030002A9D
:108F60003FD013F1310F80F2C08113F1380F80F23E
:108F7000C18113F13D0F80F2C28113F1420F80F2E3
:108F8000C38113F1450F80F2C48113F1470F80F2C2
:108F9000C58113F1490F80F2C68113F14A0F00F029
:108FA000C78113F14B0F00F0C78113F14C0F00F094
:108FB000C88113F14D0F00F0C88113F15C0F80F2EE
:108FC00024816426D4F8F40104EB820C00FB06F043
:108FD000A04E86FB00E6C017C0EB661080B2CCF84E
:108FE000AC013B7094F8EC7194F8ED3194F8EE011B
:108FF0001B0494F8EF6143EA0763334343EA002319
:1090000003F0F020B0F1E02F00F0A580102794F8D5
:109010000402B2FA82FC94F8E231D4F808624FEA12
:109020005C1C034194F80CE2367803F00F039E4277
:1090300001D90B2B68D994F8E431034103F00F03F5
:109040009E4201D90B2B71D994F8E631034103F00C
:109050000F039E4212D90B2B10D8934202D1BCF1C0
:10906000000F0BD094F8E69104EB830394F8E781AA
:109070000EEA090908EB0928C3F8AC8194F8E83135
:10908000034103F00F030B2B12D89E4210D99A42D2
:1090900002D1BCF1000F0BD094F8E89104EB8303EC
:1090A00094F8E9810EEA090908EB0928C3F8AC81B4
:1090B00094F8EA31034103F00F030B2B02D89E42D0
:1090C00000F2D0800D2F15DD94F8EC31034103F050
:1090D0000F030B2B02D89E4200F2D780102F09D12C
:1090E00094F8EE3143FA00F000F00F00864201D907
:1090F0000B2875D961B394F8E2311B0628D4C4F863
:1091000000520522012007E7934202D1BCF1000F73
:1091100091D094F8E29104EB830394F8E3810EEA92
:10912000090908EB0928C3F8AC8184E7934202D10E
:10913000BCF1000F88D094F8E49104EB830394F819
:10914000E5810EEA090908EB0928C3F8AC817BE741
:1091500005220120E0E694F8E20100063FF556AF53
:109160003D480C27036052E717F07EFF3B4B384920
:10917000A3FB00234A785B0C1AB394F8E00194F83F
:10918000E121D2B2122A18BF012A08D002F0EF0260
:10919000A2F1A202B2FA82F2520902B94A70D4F8DC
:1091A000F81194F8F021A1B18B422BD0591A012962
:1091B00000F0838094F8DE11A4F8FC01C4F8F831C3
:1091C00010E794F8E02194F8E10100EB022080B26E
:1091D000E5E7A4F8FC01C4F8F83194F8DE1101E7E2
:1091E000904202D1BCF1000F84D094F8EE2104EB40
:1091F000800094F8EF3102EA0E0E03EB0E23C0F864
:10920000AC3177E794F8DE11ECE66FF05B0E4FF0CF
:109210000C0C0CF1FF30124E16F9109006EB4C0CB2
:1092200006EB40069CF801C0A3EB090096F801800C
:10923000AEEB0906ACEB080C00FB0CF090FBF6F073
:10924000404440B2002833DA0026BBE62028012043
:10925000000001201F85EB511C1F012083DE1B43F2
:10926000709204089A4203D1BCF1000F3FF42AAF78
:1092700094F8EA9104EB830394F8EB810EEA090970
:1092800008EB0928C3F8AC811CE79A4203D1BCF172
:10929000000F3FF423AF94F8EC9104EB830394F8B0
:1092A000ED810EEA090908EB0928C3F8AC8115E73E
:1092B0006428A8BF6420064684E6002A3FF47AAFFB
:1092C000B4F8FC6104EB8207D4F8F411861BDFF8D4
:1092D00084C0143E01FB06F18CFB01C6C917A1EB4B
:1092E000E60189B2C7F8AC1164E76FF0300E4FF0B9
:1092F000010C8EE76FF0370E4FF0020C89E76FF02C
:109300003C0E4FF0030C84E76FF0410E4FF0040C5D
:109310007FE76FF0440E4FF0050C7AE76FF0460ED2
:109320004FF0060C75E76FF0480E4FF0070C70E732
:109330009E464FF0080C6CE76FF04A0E4FF0090C98
:1093400067E79E464FF00A0C63E79E464FF00B0C12
:109350005FE700BF67666666354B5B68C3F308036B
:1093600070B4CBB9EFF31183B3B9324A324E334DF7
:109370001368AC6811688B42FAD131688C42F7D817
:109380002F4A4FF47A71156801FB05F2141BB4FBE8
:10939000F5F401FB03431EE0EFF31181102383F387
:1093A000128803F1E0239D681A6812F4803F254A71
:1093B00039D1204BC9B21C68136881F31188204A47
:1093C0004FF47A712344146801FB04F2521BB2FB80
:1093D000F4F201FB03231C4A41F28831D2F8104217
:1093E000C2F810321B1B8B420AD9C0B2012382F88B
:1093F000E00182F81432002382F8DD3170BC70473E
:1094000092F814320F2BF9D8591CC0B21344C9B2C8
:1094100083F8E001102982F81412ECD1012370BC0A
:1094200082F8DD317047012414609D68C1E700BFF8
:1094300000ED00E058A1012060A1012010E000E053
:109440005CA1012054A1012020280120036933F8E8
:10945000110000EB8000C01000F55C7080B2704716
:10946000436993F82320002A00F0D3807F4A00212B
:109470002DE9F04F1278DE7D1A2A83F8231006F0CA
:10948000040C06F0080700F0C680BCF1000F40F0A5
:10949000D180002F40F0DE80BC4693F802B016F079
:1094A000010F93F801E093F803900BF0070B0269AA
:1094B000997A4EEA0B2009F03F091C7993F806A02F
:1094C00001F01F0193F807804FEA49191D7A4FEA0E
:1094D000811E93F802B04FEA840410804FEA4505DC
:1094E000987B49EADB090AF00F0A08F07F0800F0D0
:1094F0003F01A2F8029093F805904FEACA1A4FEA8A
:109500004110D97809F001094FEA081844EA91148A
:10951000D97944EA892445EAD115597A948001F031
:1095200003015C7945EA4121DD7A4AEA540A5C7B11
:109530004FEAC505A2F806A004F0070993F806A0B3
:109540005181597A48EA1A189C7A4EEA9101A2F898
:10955000088045EA54151C7B918140F2147E597BAA
:1095600044EA0924D58140EAD10114825182D87B92
:10957000997B93F810A04FEA800093F8118040EA9D
:1095800091100AF0010A08F00F089D7C40EA8A2039
:10959000D97C5C7D4FEAC81893F812904FEA4101DC
:1095A000908205F07F05187C41EAD9194FEA05152C
:1095B000197D48EA5008987D04F01F0401F003016A
:1095C000A2F816804FEAC00093F811804FEA841485
:1095D00049EA412145EA181593F814805B7D15830B
:1095E00014BF7546AD2516F0020F40EA53105183A3
:1095F00044EA98040CBFAD237346D083948315844A
:10960000538427BBBCF1000F0CBF01200920BDE82B
:10961000F08F1046704716491C8C0E80BCF1000F6D
:109620000ED044F002021A8412B277B144F0030261
:109630001A8409E01A8C97B942F002021A842CE7C6
:109640008FB144F001021A8412B24A8025E7032048
:10965000BDE8F08F1A8C42F001021A841DE742F037
:1096600003021A8419E722B2BC46EEE76D9C012082
:10967000709C01203A4B5B68C3F30803F0B42BBB2A
:10968000EFF3118313BB374A374F384E1368B56871
:109690001468A342FAD13C68A542F7D8344A4FF483
:1096A0007A74166804FB06F2551BCA69B5FBF6F519
:1096B00004FB035340F6AC549A1AA2422BDC91F8F7
:1096C00022405CB3182C39D9F0BC7047EFF31184F9
:1096D000102383F3128803F1E0239E681A6812F4C2
:1096E000803F244A26D11F4BE4B21D68136884F3DF
:1096F00011881F4A4FF47A742B44156804FB05F255
:10970000921BB2FBF5F204FB0323CA6940F6AC548A
:109710009A1AA242D3DD002281F822200F28D3D149
:109720000122CB61087081F822200023F0BC81F86F
:1097300023307047012515609E68D4E7631CDBB2B7
:10974000192B81F822300855EFD10B4B01201B78E3
:1097500081F823001A2BB7D1084B9A80B4E700BFD9
:1097600000ED00E058A1012060A1012010E000E020
:109770005CA1012054A101206D9C0120709C01205E
:10978000094BDFED0A6A03EB8101DFED097A91ED08
:10979000867AB8EE477AE7EE267AFCEEE77A17EE9D
:1097A000903A98B2704700BF2028012001F11F3F76
:1097B00000405C44714A92F8583233B192F85E32FC
:1097C0000021162B82F8581201D00020704792F821
:1097D0005D0202282DE9F04140F2CE8002F51774B7
:1097E00002F25E21D323204411F8014F634013F0AD
:1097F000800F4FEA430318BF83F0D503DBB213F0A9
:10980000800F4FEA430318BF83F0D503DBB213F098
:10981000800F4FEA430318BF83F0D503DBB213F088
:10982000800F4FEA430318BF83F0D503DBB213F078
:10983000800F4FEA430318BF83F0D503DBB213F068
:10984000800F4FEA430318BF83F0D503DBB213F058
:10985000800F4FEA430318BF83F0D503DBB213F048
:10986000800F4FEA430318BF83F0D5038842DBB271
:10987000BAD192F87512994202D00020BDE8F08169
:1098800092F86412012092F8683201F00F0192F808
:10989000637203F01F0392F86C42C90192F8705290
:1098A0009B0192F8606241EA570192F8677206F0F4
:1098B000070604F03F0443EA970305F07F0592F89A
:1098C0006B726401C2F830322D0192F85F3244EAC3
:1098D000D704C2F8241243EA062392F86F12B2F8B2
:1098E000608245EA1111C2F81832D2F86052C8F30A
:1098F000CA08D2F86C32B2F864C2C5F38A3EC2F824
:109900003C42C3F38A14D2F86472CCF30A1CC2F846
:109910004812B2F86862C7F3CA37B2F86A52B2F8AE
:109920006E127609D2F87032C5F30A05C1F34A0106
:10993000C2F84042C3F3CA13C2F81C82C2F84412F0
:10994000C2F820E2C2F828C2C2F82C72C2F834620F
:10995000C2F83852C2F84C3292F8743292F873421C
:10996000DB00B2F8721243EA5413C1F38A01C2F861
:109970005432C2F8501281E7D3237AE7202801201D
:10998000F8B5634B0646634C1D68EB0715D594F894
:109990009C3294F89D229A4235D1D4F8A032B34239
:1099A00002D85D4B00221A70D4F8D832F61A002E75
:1099B00022DD012084F8DC02F8BD15F4005543D106
:1099C000D4F8C83204F530709847C7070AD5534910
:1099D000C0F3400310F00A0F94F866208B7023D078
:1099E000052A62D04307D8D5012384F8DD32D4F8A4
:1099F000A032B342D8D8D4E794F8DC020028DBD1F7
:109A000094F8DD02F8BDD4F8A4220020434916449E
:109A100084F89D32404A012388700120C4F8A06276
:109A2000137084F8DC02C7E7D4F8A432052A1E4478
:109A3000C4F8A06251D0420766D4374B01220120FE
:109A40001A7084F8DC02B7E7B4F8A8320BBBB4F89C
:109A5000AA32F3B9B4F8AC32DBB9B4F8AE32C3B958
:109A6000B4F8B032ABB9B4F8B23293B9B4F8B43296
:109A70007BB9B4F8B63263B9B4F8B8324BB9B4F8BC
:109A8000BA3233B9B4F8BC321BB9B4F8BE32002BC9
:109A900083D0D4F8A43200252048012133441E4A43
:109AA0008570C4F8A03211707EE794F86730A26E1A
:109AB00004EB43010133B1F86C7003F00F03A1F81C
:109AC0006C504107A2EB070284F867304FEA12138B
:109AD000A266A4F88C3087D45FE794F8672040F240
:109AE000FF36A36E04EB420101323344B1F86C50EF
:109AF00002F00F02A1F86C605B1B84F867201A0962
:109B0000A366A4F88C2096E7012384F8DD3294E75D
:109B10000CB0012020280120D537012000000120B1
:109B2000002070470020704701207047024B03EB74
:109B30004101B1F8E002704720280120044B93F85E
:109B4000040318B10022012083F80423704700BFEA
:109B500020280120024B03EB8101B1F80803704774
:109B60002028012003788B4205D9044B03EB4101E7
:109B7000B1F8400370470020704700BF2028012043
:109B800038B53A4C054617F06FFAD4F89433C4F858
:109B90009403C01AB0F57A7F1DDD0023282284F8D3
:109BA000983384F89A3384F89B3384F899233D2DB5
:109BB00040D03E2D0ED101222D4B84F89A231A4617
:109BC000C4F89C330123157084F8983394F89923D2
:109BD0009A4220D038BD94F89823002AE7D0531C2D
:109BE000D4F89C13DBB28D54062B84F89833EDD156
:109BF00094F89A33012B25D094F89B33012B25D070
:109C00000023282284F8983384F89A3384F89B330D
:109C100084F8992338BD94F89A33012B1AD094F81C
:109C20009B33012B1AD00022282384F8982384F830
:109C3000993338BD01220F4B84F89B231A46C4F890
:109C40009C33BFE78B78282BD6D8F0E78B78092B8D
:109C5000D6D8ECE7022384F89A33E0E7022384F8AD
:109C60009B3317F001FAC4F8A003DCE72028012099
:109C70008C2B0120802B012030B4002305251E24CD
:109C8000024600E00232032BD4BF0021012100F87C
:109C900013100133042B04D0122B5470F2D130BCBA
:109CA00070475570EEE700BF024B0360436083606E
:109CB000C3607047E803D007024B03EB4101B1F8E2
:109CC000A802704720280120024B03EB4101B1F8A4
:109CD000A80270472028012030B4264C94F89A330B
:109CE000022B02D0002030BC704794F86E53F5B1BF
:109CF000013D04F26D3304F55B70002253FA85F5E3
:109D000010F8013B110A5340854283EA0313DBB28A
:109D10004FEAC30241EA032182EA131383EA0102F4
:109D2000EED122B1002084F89A0330BC7047B4F819
:109D30006C3343F601625BBA9BB2934209D043F69F
:109D40000362934205D00023012084F89A3330BC8B
:109D50007047094AA2F12E0102F12005D0790232A2
:109D60001379AA4203EB0023C3F3CC0321F8023F8B
:109D7000F4D1E8E7202801208C2B0120524B5B68AE
:109D8000C3F3080370B4CBB9EFF31183B3B94F4AEF
:109D90004F4E504D1368AC6811688B42FAD1316850
:109DA0008C42F7D84C4A4FF47A71156801FB05F2E2
:109DB000141BB4FBF5F401FB03431EE0EFF3118128
:109DC000102383F3128803F1E0239D681A6812F4CC
:109DD000803F424A49D13D4BC9B21C68136881F3A8
:109DE00011883D4A4FF47A712344146801FB04F250
:109DF000521BB2FBF4F201FB0323394AD2F8A4133D
:109E0000591AB1F5FA7F19D90021C4B2C2F8A433A6
:109E100082F8A81382F8A913042C34D0A4F12001ED
:109E2000B1FA81F1490971BB552892F8AC3301D1DF
:109E3000002B39D0834216D1002109E092F8A913F2
:109E4000B9B992F8A813C4B2C2F8A4330029E3D078
:109E500092F8AA33013B5018994280F8B0430DD0D4
:109E6000013182F8A81370BC7047012414609D680A
:109E7000B1E7013982F8A91370BC7047012370BCA7
:109E800082F8D0337047002302254FF6FF7082F826
:109E9000AC43194682F8AB3382F8AA43631E82F8BA
:109EA000AD53A2F8AE03D6E7012355251F20A2F833
:109EB000AE1382F8B04382F8AB3382F8AD3382F848
:109EC000AC5382F8AA03CBE700ED00E058A10120D3
:109ED00060A1012010E000E05CA1012054A101205C
:109EE0002028012070B540F201440E4E44EA80045F
:109EF00017F0BAF8054696F8F43306EB8303D3F867
:109F0000D403E3070AD517F091FD640805F1340581
:109F100007D017F0A9F88542FBD8ECE717F080FDD1
:109F2000F3E770BD202801200B49082230B5B1F8B5
:109F3000F5334AF2010580EA03045B0814F0010FCF
:109F400001D06B409BB2013A400812F0FF02F2D1FF
:109F5000A1F8F53330BD00BF20280120F0B5184E20
:109F6000002383B008210446D6F8F80386F89D3014
:109F70000DEB010517F040FAD6F8F8038121E71D33
:109F800017F03AFA8923D6F8F86325F8023D14F859
:109F9000010B3246294615F087FDBC42F7D1BDF8CA
:109FA000063032460021180A50FA83F3C3F1FF034A
:109FB0009BB2D8B2ADF8063015F076FD03B0F0BD17
:109FC0002028012038B50D4C05460146D4F8FC0385
:109FD00017F012FAB4F80004082341F2210280EAD3
:109FE000052010F4004F4FEA400018BF5040013BDD
:109FF00080B2F6D1A4F8000438BD00BF20280120AB
:10A000000FB410B582B00749002004AC54F8042BFB
:10A010002346019419F056FD02B0BDE8104004B08B
:10A02000704700BF91D500082DE9F843304C3C2221
:10A030000021304F204604F108053EF0D3FF2E4AA0
:10A04000397902F11003B2F8602084F824102284D8
:10A05000FE780FCB85E80F00002E3FD0072E3DD0B5
:10A06000012E03D094F82030032B02D00020BDE84D
:10A07000F883224A072122480325136820604FF401
:10A08000807043F002031F4E20831F4813601F4B54
:10A0900060601748597184F8225029F0C9FD4FF4C7
:10A0A0007A72B6F80234A26293B1002506F204492E
:10A0B0004FF02408B6F8023408FB05900135A16A78
:10A0C00000EE103AB8EE400A1AF006FA032DF1D16C
:10A0D000BB7853B184F822300120C8E794F82030CF
:10A0E000032BC6D0002EC1D0BAE70120BFE700BFC6
:10A0F000EC0C002004BB0120C820002020530120CC
:10A10000313C030820280120397F0308000001208A
:10A11000AC4B2DE9F04F2DED068B9B7D85B0012BCF
:10A1200000F04085022BA84B0CBF072200221A70BA
:10A13000A64B1B78132B00F243810122A4499A40BD
:10A140000A4208BF00239F4D0021DFF8B8A2342047
:10A150006A79A04C521A8AF869004FF023008AF8F5
:10A16000621018BF012221708AF865209A4A137084
:10A17000EB799A4A82F8703417F01EF80222984B55
:10A18000DAF81C008AF81020CAF81430002800F011
:10A19000FF841C2200238271C3710D21914C17F0A2
:10A1A00091FBDAF81C0017F041FC06234FF4807194
:10A1B000DAF814008C4FDFF850928C4D8C4E0193DE
:10A1C0002CF080F880226B218A4817F087FE9623B6
:10A1D0004FF01008DFF834E20093D9F80430C3F3ED
:10A1E0000803002B40F0B480EFF31183002B40F004
:10A1F000AF802068AA6823689842FAD133689A42EF
:10A20000F7D8D7F800C04FF47A7101FB0CF39B1A12
:10A21000B3FBFCF301FB00304FF47A7CD9F8043037
:10A22000C3F30803002B74D1EFF31183002B70D11B
:10A230002368A96822689342FAD132689142F7D81C
:10A240003A680CFB02FBABEB0101B1FBF2F10CFB3A
:10A2500003131B1AB3F57A7FE0D3009B013B0093F5
:10A26000BBD1DAF81C201AB1938812681B049361E1
:10A27000DAF8142040F2E93302E0002B00F0898084
:10A280009168013B11F0020F9BB2F6D0F52140F22C
:10A29000E933117301E0002B7BD09168013B11F091
:10A2A000010F9BB2F7D0D36801230DF10F020021FB
:10A2B000DAF814002CF040FFDAF81C0010B1036843
:10A2C00082889A619DF80F30682B00F0A180019B75
:10A2D000013B13F0FF0301937FF479AF9AF86030EC
:10A2E000DAF85C203D49032BC1F8742400F0B680F5
:10A2F00000208AF86B00404A137823B19AF86A303C
:10A30000003318BF0123137005B0BDEC068BBDE808
:10A31000F08FEFF3118188F31288D5F808B02B681D
:10A32000DB0304D50123CEF80030D5F808B023684C
:10A33000C9B2DEF8002081F31188396813440CFBA0
:10A3400001F2A2EB0B02B2FBF1F20CFB032380E75C
:10A35000EFF3118288F31288D5F808C02B68D9036F
:10A3600004D50123CEF80030D5F808C02368D2B256
:10A37000DEF8000082F311884FF47A7239681844CD
:10A3800002FB01F3A3EB0C03B3FBF1F302FB003080
:10A3900042E713498A4209D0184B9A4200F0F982E9
:10A3A00003F580639A427FF47FAF0223144AD821D9
:10A3B00001FB03239A89013292B29A819B8973E748
:10A3C0000023C0E6D8980120F03600206D9C0120C3
:10A3D00048800A0014BB0120E83600202028012014
:10A3E0000030014058A101205CA1012010E000E0F4
:10A3F00060A10120D82000207522012000380040F3
:10A400000C990120C820002000ED00E054A101209B
:10A4100017F006FB8C21DAF814002BF01FF901234A
:10A420000DF10F020021DAF814002CF085FEDAF8A5
:10A430001C0017F0FBFA9DF80F30142BFFF44EAF01
:10A44000182B03D9543B062B3FF648AF0322DAF80A
:10A450005C308AF86020484AC2F87434474A0624BF
:10A46000474D03201368474943F001038AF862000F
:10A47000CAF8001000211360434A444BCAF8042074
:10A48000EA78CAF82030012A414B8AF86B401C71E7
:10A49000A97140F277829FED3F7A01238AF8631019
:10A4A00007EE903A364D013B8AF86620F8EEE77ADF
:10A4B0002A79394C394867EE877A8AF868308AF801
:10A4C0006720FCEEE77AC4ED007A2DF035F82B78A2
:10A4D0000BB18AF862300123314D40F235568AF8CB
:10A4E0006A3031F07BFE24689FED2E0A07EE904A19
:10A4F000F8EE677A80EE270A3DF052FAA5FB0035A8
:10A500009FED296A6D08DFED296A294BB542B7EE48
:10A51000087A284AA8BF35462749AEB207EE906AA6
:10A52000B7081E80F8EE677A9F80730886EE270AC8
:10A530000B8067EEA67AC2ED007A30EE470A3DF056
:10A540002FFA01281D4A4FF00003B8BF0120DFEDAC
:10A550001C4ADFED1C5A10701B499FED1C4ADFEDB1
:10A560001C1A9FED1C2ADFED1C2ADFED1C0A9FED53
:10A570001C1A9FED1C6A42E0202801202053012074
:10A58000D898012039750308953D030890C1793D9D
:10A590000000012000007A44EC270020C8200020A1
:10A5A000ABAAAAAA00247449000034450000003D6B
:10A5B00008000020E4270020E0270020DC270020FE
:10A5C0003C8C4F3EDB0FC93F5C270020DB0F49C0AE
:10A5D00092E741B99730083C15A82ABEDB0FC9BFE6
:10A5E000DB0F4940DB0FC940E4CB1641E4CB16C179
:10A5F0000133F6EE007A202BE1EC017A53D007EE1E
:10A60000903AB8EEE77A27EE247A77EE257AFDEED7
:10A61000E76A16EE902A2032402AE9D8B4EEE57AAD
:10A62000F1EE10FA40F3BF815FED116AF4EEE67AC5
:10A6300037EEC67AF1EE10FAF0EE477AF6DCB4EEB9
:10A64000C47AF1EE10FA40F1B6815FED186AB4EE0B
:10A65000E67A77EE067AF1EE10FAB0EE677AF6D483
:10A66000F4EEE57AF1EE10FA40F3958171EE677A37
:10A6700027EEA75A0133B0EE423AF7EE006A202BDC
:10A6800065EE673AA5EE213A76EEE77AF0EE626A79
:10A69000B6EE007AE3EE056AE3EEA67A67EE877A15
:10A6A000E1EC017AABD1ED4A07EE907A9FEDEC6ACE
:10A6B00004EB440C907FB8EE670AD27F4FEA8C0C13
:10A6C00006EE900A142007EE902AE649F8EEE66AB4
:10A6D000AAF80C05B8EEE77ADFEDE37AE348B7EEC7
:10A6E000001AC6EE261ADFEDE26AE24A1027AAF83F
:10A6F0001035CAF8082502F12803A832DFEDDE8AFA
:10A7000077EEC77A9FEDDD8ACAF81425B0EE414A8C
:10A71000DFEDDB0A67EEA67AAAF80075B0EE603AC4
:10A72000D84FCAF80435C0ED007AA7F55E739FEDE7
:10A73000D65ADFEDD63ADFEDD64A9FEDD62ADFEDC9
:10A74000D62AB1FBF5F06045B1FBF4F238BF6046A4
:10A7500092B2A7F5437405EE900A91FBF5F1F8EE7D
:10A76000655A06EE101AB2FBF6F2FCEEE55AD2B2CA
:10A77000B8EEC66A07EE902A8AF8F922F8EE655A12
:10A78000F8EEE77A26EE286A65EE885A81EE277A97
:10A7900026EE006AFDEEE57A35EEA00A76EE200A96
:10A7A00017EE905AFDEEC07A203517EE900AFDEEB6
:10A7B000E07A203017EE901AFDEEC67A8AEDBF7A65
:10A7C000203117EE902A2032C826402A27F8026B43
:10A7D00000F27281B4EEE36AF1EE10FA40F3068201
:10A7E000F0EE467A9FEDB01ADFEDAE6AF4EEE67A4F
:10A7F00037EEC17AF1EE10FAF0EE477AF6DCB4EEFD
:10A80000E47AF1EE10FA40F1EE819FEDA71ADFED48
:10A81000A76AB4EEE67A77EE017AF1EE10FAB0EEBE
:10A82000677AF6D4F4EEC37AF1EE10FA40F39C8125
:10A8300073EEE77A67EEA76A9FED9D7AB0EE628AC3
:10A84000402927EEA61AA6EE828AA8EE267AE1EE25
:10A85000077A67EEA16A36EE849A34EE661AC4EE81
:10A86000097A66EEA76A21EE271AF1EE669A40F29F
:10A870002E81B0EE457A402DC3ED006A83ED015A7A
:10A88000C3ED029A83ED037A83ED041A83ED065A31
:10A8900083ED055A83ED085A83ED075A00F28E8046
:10A8A000F4EEE35AF1EE10FA40F39481F0EE657A9B
:10A8B0009FED7D1ADFED7B6AF4EEE67A37EEC17A22
:10A8C000F1EE10FAF0EE477AF6DCB4EEE47AF1EE4F
:10A8D00010FA40F17C819FED741ADFED746AB4EEDA
:10A8E000E67A77EE017AF1EE10FAB0EE677AF6D4F6
:10A8F000F4EEC37AF1EE10FA40F32C8173EEE77AAE
:10A9000067EEA76A9FED6A7AF0EE628A9FED631A9E
:10A91000B0EE449A402827EEA68AE6EE828AA8EE98
:10A92000A67AE8EE077AB0EE447AA7EE819AA7EE0F
:10A93000C17AC7EE098A47D9F6EE006AB0EE457AC9
:10A94000B7EE001AC4EE097AC3EDC78A83EDC95A7F
:10A95000243383EDBF5A83EDC25A83EDC15A66EEAC
:10A96000A76A21EE271A67EE277AC3EDBA6AC3ED0C
:10A97000BC6A83EDBB1AC3EDBD7AA3427FF424AF5A
:10A980000120B8E4354B8AF863009B789FED447A48
:10A9900086E501230AE5F4EEE07AF1EE10FA48BF0D
:10A9A00074EE677A64E6B0EE677AB4EEC47AF1EEDC
:10A9B00010FA3FF54AAEF0EE477A51E6F7EE008A1C
:10A9C0004028B0EE689AB7D8F4EEC35AF1EE10FA08
:10A9D00040F3FA80F0EE407A9FED331ADFED316AF2
:10A9E000F4EEE67A37EEC17AF1EE10FAF0EE477A3D
:10A9F000F6DCB4EEE47AF1EE10FA40F1E2809FED7D
:10AA00002A1ADFED2A6AB4EEE67A77EE017AF1EEE1
:10AA100010FAB0EE677AF6D4F4EEC37AF1EE10FADB
:10AA200040F3C58073EEE77A27EEA78A9FED201AE0
:10AA3000B0EE62AAB8EE007A68EE279AA8EE02AAF3
:10AA4000F6EE006AA8EE0A1AE9EE817A34EE671A89
:10AA500027EE877A61EE266A74E700BFD898012056
:10AA60000000484240420F000000C842E827002092
:10AA70000AD7233C8C92040827D4D236E5A6C539E0
:10AA8000DB0FC93F4C27002000000000DB0F4940CE
:10AA9000DB0F49C092E741B99730083CF304353FDA
:10AAA0000000FA42E4CB1641DB0FC940E4CB16C1EB
:10AAB00015A82ABEDB0FC9BFB7EE001A4029F0EE79
:10AAC000459AF0EE456AB0EE419A3FF6D2AEB4EE4A
:10AAD000C36AF1EE10FA40F38380F0EE607A5FED26
:10AAE0000E8A1FED108AF4EEC87A37EEE87AF1EE9E
:10AAF00010FAF0EE477AF6DCB4EEE47AF1EE10FAF2
:10AB00006BD55FED178A1FED178AB4EEC87A77EE22
:10AB1000287AF1EE10FAB0EE677AF6D4F4EEC37A42
:10AB2000F1EE10FA2ADD73EEE77A67EEA78A1FEDE1
:10AB3000208AF0EE62AAB8EE007A27EEA8AAE8EE24
:10AB400082AAAAEEA88AEAEE087A67EE877A87EEEA
:10AB5000897A90E61FED297AF4EEC77AF1EE10FAC1
:10AB600048BF74EEE77ACBE61FED2E7AF4EEC77A93
:10AB7000F1EE10FA48BF74EEE77A5BE61FED337A28
:10AB8000F4EEC77AF1EE10FA48BF74EEE77ACCE73C
:10AB9000142016F011FDCAF81C0000283FF4FDAA8D
:10ABA000FFF7F7BA134B04221A70FFF7C1BA9FEDF3
:10ABB000127AF4EEC77AF1EE10FA48BF74EEE77A33
:10ABC00032E7F0EE477A27E7B0EE407A11E7F0EE91
:10ABD000477A8DE6B0EE657A77E6F0EE477A9DE744
:10ABE000B0EE607A88E7F0EE477A1BE6B0EE467A80
:10ABF00005E600BFF0360020DB0FC9BF38B5384B83
:10AC00005B68C3F30803CBB9EFF31183B3B9354ADB
:10AC1000354D364C1368A06811688B42FAD129680B
:10AC20008842F7D832494FF47A72096802FB01F47E
:10AC3000241AB4FBF1F402FB03441EE0EFF311818C
:10AC4000102383F3128803F1E02398681A6812F442
:10AC5000803F284A22D1234BC9B21D68136881F373
:10AC60001188234A4FF47A742B44116804FB01F2D3
:10AC7000121AB2FBF1F204FB03241F4DD5F89830F1
:10AC8000E31AB3F5FA6F02DD002385F89C3095F8DE
:10AC90009C303BB900230120EB6038BD01201060DF
:10ACA0009868D8E700221549E86814F003FA95F887
:10ACB0009C3073B9124B1B781B2B04D1D5F8783418
:10ACC000104AE31AD3800023C5F878440120EB60D2
:10ACD00038BD0D48FFF742F9002385F89C30E9E7BD
:10ACE00000ED00E058A1012060A1012010E000E08B
:10ACF0005CA1012054A1012020280120BC280120B2
:10AD00006D9C0120709C0120B493040870B582B042
:10AD1000044616F0A9F9974AD2F87C3403F24C4362
:10AD200083420CD392F880344BB1022B40F21F8146
:10AD300092F85D02023098420DDC02B070BD012134
:10AD40000023C2F87C0482F85C4282F8801482F806
:10AD5000583202B070BD591C1344C9B283F85C422A
:10AD6000884282F88014D4BF0123002382F858322D
:10AD7000E3DC92F85E520023162D82F88034DCD09A
:10AD80006B00290692F85D4248BF83F0D503DBB221
:10AD900013F0800F4FEA430318BF83F0D503DBB2F3
:10ADA00013F0800F4FEA430318BF83F0D503DBB2E3
:10ADB00013F0800F4FEA430318BF83F0D503DBB2D3
:10ADC00013F0800F4FEA430318BF83F0D503DBB2C3
:10ADD00013F0800F4FEA430318BF83F0D503DBB2B3
:10ADE00013F0800F4FEA430318BF83F0D503DBB2A3
:10ADF00013F0800F4FEA430318BF83F0D503022CF2
:10AE0000DBB247D95C490C44023111F8016F734041
:10AE100013F0800F4FEA430318BF83F0D503DBB272
:10AE200013F0800F4FEA430318BF83F0D503DBB262
:10AE300013F0800F4FEA430318BF83F0D503DBB252
:10AE400013F0800F4FEA430318BF83F0D503DBB242
:10AE500013F0800F4FEA430318BF83F0D503DBB232
:10AE600013F0800F4FEA430318BF83F0D503DBB222
:10AE700013F0800F4FEA430318BF83F0D503DBB212
:10AE800013F0800F4FEA430318BF83F0D5038C42C1
:10AE9000DBB2BAD1104490F85B1299427FF44DAF07
:10AEA0007A2D2AD022D97C2D27D07D2D7FF445AF55
:10AEB00092F86132042B4AD0052B34D0032B7FF457
:10AEC0003CAF92F8633292F86222202B2B482C4937
:10AED000A8BF2023092AA8BF092280F82A314B7273
:10AEE00080F829210A720CF0DBF826E7282D7FF480
:10AEF00024AF244B01221A701FE7234B1A6E572AE6
:10AF00003FF71BAF2148D118082605684468012087
:10AF1000D654C1F80150C1F805401A6E1C490932D7
:10AF200008701A6609E71B4B1B78EBB1134C012123
:10AF300094F8292104F590703EF054F8164B012145
:10AF4000164A1B6884F82B112D331360F5E6114B5C
:10AF50001B78002B3FF4F1AE002302A9084801F84A
:10AF6000013D09F03BFBE8E60CF09AF8E5E6052028
:10AF7000E1E600BF202801207C2A0120E0370120E3
:10AF8000004401208D44012098440120812A0120A1
:10AF90008E4401208441012058A10120B83D0120A8
:10AFA0002DE9F04FE04C8BB094F8D0332BB94FF033
:10AFB000000A50460BB0BDE8F08F94F8AB33002286
:10AFC00094F8AA03012B84F8D02346D094F8B05308
:10AFD000023D15F0FF0500F0AB8104F56C714FF6F2
:10AFE000FF730D4411F8012B9B1AA9429BB2F9D1B2
:10AFF0001A0A204490F8AF139142D8D190F8AE23AA
:10B00000DBB29A42D3D194F8AC33202B40F0848148
:10B0100094F8AD9309F1020309F1100209F1120A43
:10B0200009F1140B089309F1040309F118080193BD
:10B0300009F10603029309F10803039309F10A03D6
:10B04000049309F10C03059309F10E03069309F12A
:10B050001603079309F11A03B5E094F8AD93204461
:10B06000B4F8AE3309F1020104EB090209F1060656
:10B0700009F1040554FA81F709900296304692F8D6
:10B08000B063019597F8B0C3334492F8B15354FAC2
:10B0900080F6019A6344089109F1080054FA82F29B
:10B0A00003EB052397F8B1C354FA80F592F8B01377
:10B0B00096F8B073194492F8B12395F8B0E301EB18
:10B0C0000C21039009F10A0096F8B183394495F8F0
:10B0D000B1B354FA80F3049001EB022109F10C00A2
:10B0E00093F8B0A309F10E06714454FA80F793F86F
:10B0F000B13354FA86FC01EB082197F8B053069659
:10B1000009F1100251449CF8B06397F8B17354FAF6
:10B1100082FE01EB0B2109F1120A9EF8B08309F1BE
:10B12000140B29449CF8B1C354FA8AF59EF8B1E394
:10B1300001EB0321059095F8B03309F11600314475
:10B1400054FA8BF695F8B15301EB072196F8B073DA
:10B1500096F8B163414409F11808079001EB0C21FE
:10B1600054FA80FC09980B449CF8B0139CF8B1C3C6
:10B1700003EB0E233B4454FA88F703EB052397F8BF
:10B18000B05397F8B173194409F11A0301EB062182
:10B1900054FA83F60D4496F8B0E396F8B16305EBE4
:10B1A0000C2590F8AFC390F8AE030EEB050100EB51
:10B1B0000C2C01EB07211FFA8CFC01EB062189B254
:10B1C0008C457FF4F4AE089954FA82F2A14454FA03
:10B1D00088F854FA81FE019954FA83F354FA81FCF9
:10B1E0000299029254FA8AF254FA81F7039903926F
:10B1F00054FA8BF254FA81F604990492079A54FA9D
:10B2000081F599F8B1B399F8B0A354FA82F9059988
:10B21000CDF814900AEB0B2A9EF8B19354FA81F002
:10B220009EF8B0E306990EEB092ECDF818809CF835
:10B23000B18354FA81F19CF8B0C3C4F80CE30CEB71
:10B24000082B97F8B1E396F8B1C397F8B07396F866
:10B25000B06307EB0E2795F8B1E306EB0C2695F8E3
:10B26000B05390F8B1C390F8B00305EB0E25029AE5
:10B2700091F8B1E300EB0C2091F8B013019001EBD1
:10B280000E2192F8B1C392F8B0230398029102EB19
:10B290000C22049990F8B1E390F8B08391F8B1C30F
:10B2A00091F8B09308EB0E2E0198029909EB0C2C43
:10B2B000C4F82823059AC4F82003C4F8241392F88C
:10B2C000B10392F8B013069A01EB0021C4F808A369
:10B2D00093F8B1034FF0010AC4F81C5393F8B0334C
:10B2E00092F8B15392F8B02303EB00235046C4F810
:10B2F00010B302EB0522C4F81473C4F81863C4F841
:10B300002CE3C4F830C3C4F83413C4F83823C4F8A9
:10B310003C330BB0BDE8F08F04484FF0000A13F047
:10B32000F9FB84F8A90344E620280120D02B012052
:10B33000FF224FF6FF735CE6F8B5284E15F094FE39
:10B34000054600F1FA07344696F8F43306EB83031A
:10B35000D3F8D40316F018FC38BB94F8F43304EB9C
:10B360008303D3F8D40316F00FFC28B315F07CFE4A
:10B37000D4F88834401B9842C4F884042BD805F5CF
:10B38000FA7594F8F43304EB8303D3F8D40316F07E
:10B39000FBFBB0B994F8F43304EB8303D3F8D40384
:10B3A00016F0F2FB90B1002005E015F05DFEB8420A
:10B3B000CAD94FF0FF30F8BD15F056FEB842CCD9CF
:10B3C000F7E715F051FEA842DBD9F2E715F04CFE85
:10B3D000A842DFD9EDE70120EDE700BF20280120DA
:10B3E00038B5002405460470FFF7A6FF431C11D0B2
:10B3F000012803D12B78A040184328700134082C71
:10B40000F2D1054A01202B7892F88C144B4082F837
:10B410008C3438BD0020FCE7202801202DE9F843BA
:10B42000204C0746204D2668A846023695F8F4338E
:10B4300005EB8303D3F8D40316F0A6FB10BB15F07D
:10B4400013FE00F1270615F00FFE8642FBD80025FB
:10B450004FF001092C4698F8F43308EB8303D3F836
:10B46000D40316F091FB18B109FA05F31C43A4B2FA
:10B47000092D06F134060BD015F0F6FD8642FBD8F7
:10B480000135E8E723689E42D0D80020BDE8F88364
:10B4900040F201232340B3F5007FF6D16408012078
:10B4A0003C70F3E758A101202028012037B5FF2385
:10B4B00002AD044605F8013D2846FFF7AFFF00B98D
:10B4C0001CB99DF8070003B030BD013CF4E773B52B
:10B4D0000022204C0144054684F8F52384F8F62325
:10B4E000CEB284F88D2484F88E24FF228DF80720B4
:10B4F0002846FFF793FFF8B115F8010BFEF714FD8E
:10B50000EBB2B342F4D194F88F34EBB11248FFF7A9
:10B5100085FF88B11148FFF781FF68B10DF1070081
:10B52000FFF77CFF40B1B4F8F523B4F88D349A42AC
:10B5300002D0C2238DF807309DF80700A0F1300338
:10B540005842584102B070BD0DF10700FFF766FF89
:10B55000F2E700BF20280120AD2C0120AE2C0120F5
:10B5600070B50D46184C0646013D94F8F433EDB223
:10B5700004EB83030135D3F8D4032DF0EBFF3544FE
:10B58000002384F8F53384F8F6333078FEF7AAFC0C
:10B5900016F8010BFEF7C8FCAE42F6D194F88F34D2
:10B5A0003BB194F8F503FEF79DFC94F8F603FEF723
:10B5B00099FC94F8F433202104EB8304D4F8D403E9
:10B5C000BDE8704016F07EB920280120FE2313B597
:10B5D000ADF80430002304468DF8063003788DF86A
:10B5E000073013B901238DF8063004210DEB01005B
:10B5F000FFF7B6FF0220FFF759FFFF280CD1217893
:10B600006068FFF7ADFF2820FFF750FFA0F130037F
:10B610005842584102B010BD0020FBE737B505463F
:10B6200008461446FFF7D2FF78B10123022101A892
:10B630008DF804508DF80530FFF792FF2046FFF794
:10B6400035FFA0F130035842584103B030BD07B573
:10B650000E4B0268934317D0FF230421ADF804304A
:10B6600043788DF8063083780DEB01008DF80730B4
:10B67000FFF776FF0220FFF719FFA0F130035842D1
:10B68000584103B05DF804FB0120FAE700FFFF001A
:10B6900037B5054608460C46FFF7D9FF60B1237859
:10B6A000022101A88DF804508DF80530FFF758FFEE
:10B6B00021786068FFF70BFF03B030BD10B5064C72
:10B6C000D4F8FC0315F094FE0028F9D0D4F8FC035C
:10B6D000BDE8104015F084BE2028012010B5FFF70A
:10B6E000EDFF0A4A082141F22104B2F8933483EABB
:10B6F00000239BB213F4004F4FEA430318BF63408B
:10B7000001399BB2F6D1A2F8933410BD2028012054
:10B7100038B50B4B0D4603EBC0040A4894F82822B9
:10B7200003EB8203D3F84C1135F07FFB94F82E32F3
:10B730002BB1691C0448BDE8384035F076BB38BDF4
:10B740007092040840DC04081B2E0508F8B50C4C68
:10B750000C4E04F544750C4F206835F07BFB616896
:10B7600011B1304635F061FBA16811B1384635F0B2
:10B770005CFB103435F007FCAC42EDD1F8BD00BFE6
:10B780006895040837DC04083DDC040810B523F094
:10B79000C3FD90B10B480C4C36F07AFA0B4835F0EB
:10B7A00059FBD4F8980416F0A9FCD4F89C0423F0B3
:10B7B000E5FD39F0FFFE29F06BF90548BDE81040C2
:10B7C00036F066BA43DC04082028012063DC040854
:10B7D0006FDC04082DE9F04F002489B083469246BF
:10B7E0000D4626464FF019094FF46178BAF1000F63
:10B7F00022D004EB8403052228460AEB03070793B3
:10B8000039463DF0C7FB3A79B0FA80F6079B19FB41
:10B81000028258461AF8033076090492FA783146C3
:10B8200019FB02820392BA7802927A780093234637
:10B8300001920F4A35F08AFC2B7931460C4A584662
:10B8400019FB03830493EB7819FB03830393AB7811
:10B8500002936B78019315F8053B0093234601345E
:10B8600035F08CFC0A2CC1D109B0BDE8F08F00BFC7
:10B870009CDC04082DE9F04706468CB08946154645
:10B880000024324FC4EBC40309EB03021068918813
:10B8900040F3074892790890ADF824108DF82620DF
:10B8A000B8F1000F4AD0002D4DD02B440AA91868DA
:10B8B0009A889B790A9008A8ADF82C2007228DF869
:10B8C0002E303DF067FB9DF82E30B0FA80FA3A46F4
:10B8D000304606934FEA5A1A9DF92D30514605938A
:10B8E0009DF92C3004939DF82B3003939DF92A3059
:10B8F00002939DF8293001939DF828300093234648
:10B9000035F024FC9DF826303A46514630460693E1
:10B910009DF9253005939DF9243004939DF823303B
:10B92000CDE902839DF8213001939DF820300093EA
:10B930002346013435F022FC102CA3D10CB0BDE815
:10B94000F04735F020BBAA46DCE700BFB2DC0408B4
:10B950002DE9F04F804689B0894616460D461446BB
:10B960000027DFF804B1002E6AD00C2221462846B9
:10B970003DF010FB94F90B30B0FA80FA5A4604936C
:10B98000404694F90A304FEA5A1A03935146B4F9E3
:10B9900008300293B4F906300193B4F904300093EF
:10B9A0003B4635F0D3FB95F90B305A46514640469D
:10B9B00004930C3515F9023C0C34039335F9043C1F
:10B9C000029335F9063C019335F9083C00933B4658
:10B9D000013735F0D3FB082FC5D10024DFF88CA048
:10B9E00025467EB300270123325903FA07FB59F895
:10B9F000043053403BEA030314BF0123002312EA3F
:10BA00000B0F079306D000972B46524607994046E6
:10BA100035F09CFB59F804301BEA030F06D0009761
:10BA20002B4652460799404635F0A8FB01370E2FAA
:10BA3000D9D101350C34082DD3D109B0BDE8F08F30
:10BA4000B246B0E73746012359F80420BB40134201
:10BA500006D000972B4652460121404635F08EFB1A
:10BA600001370E2FEFD1E4E7CFDC0408E7DC040850
:10BA70002DE9F04F064685B0884614468946924621
:10BA80000027002509EB050393F8C0300393002C31
:10BA900065D00AEB0503039A93F8C030D01A324AF6
:10BAA000D0F1000B4BEB000B3046CDE9005359466B
:10BAB0003B4635F04BFB039B59462B4A3046CDE9BC
:10BAC000005301353B4635F059FB062DDAD10137DD
:10BAD00009F106090AF1060A062FD2D108F1E40A93
:10BAE0000025DFF884B01AF8019B002C39D06319C7
:10BAF0005A46304693F8E430A9EB03014F424F41D8
:10BB0000CDE900533946062335F020FB0623164ABB
:10BB100039463046CDE90059013535F02FFB0B2D64
:10BB2000E1D198F8F05074B194F8F0303046EA1A48
:10BB300001930023544200934FF0070354410A4AF3
:10BB4000214635F003FB0023074A21460195009367
:10BB50000723304635F012FB05B0BDE8F08FA34651
:10BB6000A9E72746D2E700BFFCDC04082DE9FF4720
:10BB7000814690460F4614460025DFF85CA0B8F1D8
:10BB8000000F27D00422214638463DF003FAE3781F
:10BB9000B0FA80F6524602934846A378760901939C
:10BBA0003146238800932B4635F0D0FAFB78524675
:10BBB0003146484602930434BB78019337F8043B7E
:10BBC00000932B46013535F0D9FA102DD7D104B0AA
:10BBD000BDE8F0874646E9E710DD04087FB5094B6C
:10BBE000094A0493094B0A4903930A4B0A480293F2
:10BBF0000A4B01930A4B00930A4B35F047FA07B002
:10BC00005DF804FB62DD040822DD040867DD04083A
:10BC10002CDD040871DD040837DD04087ADD040832
:10BC200086DD040803AF0120044B054A05491B6863
:10BC300012680968044835F029BA00BF187AF01F65
:10BC4000147AF01F107AF01F8CDD04082DE9F843F8
:10BC50001424184D35F097F9174835F097FE2D212B
:10BC6000D5F8980416F058FA013CF8D1134D35F088
:10BC70008AF9134E134FDFF854802B7EE11004F045
:10BC80000702384606EB83030131D3F84C9135F0B7
:10BC9000CCF86A7E494642B10B4835F0F7F90134D9
:10BCA0002035102CE9D1BDE8F883404635F0EEF997
:10BCB000F5E700BF20280120A0DD04087420012042
:10BCC00070920408B6DD0408C7DD04089EE5040888
:10BCD00038B50D4618F0DCFB0C4B04461978884249
:10BCE00005D201460A4835F0D1F9204638BD2DB1BC
:10BCF000FF2803D1074835F0C9F9F6E701390648AE
:10BD000035F0A2F94FF0FF34EFE700BFE40C00205C
:10BD1000CEDD0408DFDD0408F2DD04082DE9F04F74
:10BD2000804687B0344C354A2378608802EB830321
:10BD3000D3F84C911BF080FED0E901A30493304B63
:10BD400093F8A03413B9CDF810A09A4608F0400338
:10BD50000026DFF8B8B00593A379002B08BF0123B4
:10BD60009E4206DB0834274B9C42DCD107B0BDE87D
:10BD7000F08F6279237906FB0323049A0136D55CA0
:10BD8000BAF1000F11D1B5FA85F77F090DB305F0AF
:10BD90000F032D095A4639464035029340464B461B
:10BDA000CDE9006535F0EAF9D6E71AF80330EA1A6A
:10BDB00057425741C3B103F00F021B0939464046B1
:10BDC000403302925A46CDE900634B4635F0BEF946
:10BDD000DCE7059B002BBFD100964B460A4A39464B
:10BDE000404635F0CBF9B7E700964B46064A394650
:10BDF000404635F0ABF9C9E79894040870920408FE
:10BE000020280120689504082DDE040817DE0408A8
:10BE100070B5344C344835F01DF894F82530012BBA
:10BE20005AD1324835F0B2FD314E3AF003FA40B102
:10BE3000B6F898502F4835F00DF88DBB2E4835F0E8
:10BE4000A5FD2E4835F006F82D4D94F8293005EB68
:10BE50008303D3F8080635F019F9B6F89410294889
:10BE600034F0E3FF94F826302BBB274835F08EFDE5
:10BE7000264834F0EFFF94F82A3005EB8305D5F817
:10BE8000100635F003F9B6F89610214834F0CDFFCE
:10BE900094F82A309BB91F48BDE8704035F076BD54
:10BEA0004FF47A721C48B5FBF2F102FB115292B2C8
:10BEB00035F0ECF8C5E7194835F068FDD8E794F897
:10BEC000273023B91648BDE8704035F05FBD1548EE
:10BED000BDE8704035F05ABD1348BDE8704035F0FC
:10BEE00055BD00BF68B1012041DE040857DE0408DB
:10BEF000503500205EDE040879DE04088BDE04087D
:10BF000070920408A1DE0408BEDE0408CEDE040838
:10BF1000E9DE04080CDF040883DE0408C5DE04083B
:10BF2000BFDE0408C6DE040811DF04086C4B2DE9EF
:10BF3000F04FDA7891B09846002A00F0A680694860
:10BF400035F024FD0025DFF8B0A1DFF8C4B1A94623
:10BF5000079508A9E8B223F05FF89DF82830002B78
:10BF60006CD0022D0C9C40F09D80002C00F0918044
:10BF700007EE904ADFED5C6AF8EEE77A86EEA77A84
:10BF8000FDEEC77A17EE906A9AF8A244089B012C3E
:10BF900040F281801A460221544896FBF4F434F0B2
:10BFA00044FF0D9A002A00F0918041F288304FF44E
:10BFB0007A7302FB0400B0FBF3F00F9B002B00F040
:10BFC000878041F288314FF47A7C03FB0411B1FB86
:10BFD000FCF1062D03D0079F81440F44079798F882
:10BFE00003C0BCF1000F75D04FF47A7C0E9FB7FBF5
:10BFF000FCFCCDF810C04FF00A0C91FBFCFE0CFBD2
:10C000001E11CDE902E190FBFCF10CFB1100CDE922
:10C0100000102146364835F039F8022D08D19AF83B
:10C02000A234012B04D932460999584635F02EF82E
:10C03000304A342303FB05230022DA620135182D30
:10C0400087D198F80330EBB12B494FF47A73D1F8CC
:10C05000A804D1F8AC24D1F8B0145209B0FBF3F322
:10C06000264835F013F80A22079B079893FBF2F352
:10C0700099FBF2F102FB1307214802FB1192009792
:10C0800035F004F811B0BDE8F08F1E4835F07EFCA5
:10C0900058E7264678E7099A02211B48344634F0CF
:10C0A000C4FE7EE75CB107EE904ADFED0F6AF8EE62
:10C0B000E77A86EEA77AFDEEC77A17EE904A089ADD
:10C0C00029460A48002634F0B0FE6AE7104674E7B5
:10C0D00019467EE721460D4834F0D8FF9DE700BFA2
:10C0E000FCAE01201FDF04080024744974DF04083B
:10C0F00096DF04087822012020280120CADF0408E6
:10C10000EADF04086ADF040883DF0408C6DF0408E6
:10C11000BADF04086B4B6C4819684FF47A732DE949
:10C12000F04790B0B1FBF3F134F0B0FF05A817F081
:10C1300015FE58B1654A05A9002308A8B2F90020E8
:10C1400017F032FE08A9624834F0A0FF614B0024CA
:10C15000614D1B78614A05F5C66905EB83036049AB
:10C16000127805F5CA65D3F81C3609885D4834F0A5
:10C170008DFF5D4B5D4819685D4BDFF8CCA1B1FBCD
:10C18000F3F134F052FE22F061FD4FF47A72594B14
:10C19000B0FBF2F102FB11020A20B3F9003089B2C0
:10C1A00092B2B2FBF0F2544834F03FFE534BD3F856
:10C1B000008059F82470A300D7B10126A64016EAE2
:10C1C000080F13D0F20611D01AF8042039465B5933
:10C1D0004B4853F8222034F028FE022E06D1494B5A
:10C1E00093F8251011B1484834F01FFE0134E0E700
:10C1F00034F0C9FE454A4649464834F047FF464CAC
:10C20000464A3946464B4748D31AB4F8B42434F06A
:10C210003DFF4549D1F88420002A42D007EE902AFC
:10C22000DFED426AB8EEE77AC6EE877AFDEEE77A8E
:10C23000CDED037AB4F8B6345BB107EE903ADFED9A
:10C240003B6AF8EE677A86EEA77AFDEEC77A17EEBC
:10C25000903AC96959B107EE901ADFED346AF8EEE9
:10C26000E77A86EEA77AFDEEC77A17EE901A304885
:10C270000125304E0089304F6428CDE90031014658
:10C28000039BA8BF64212D4834F000FF2C4834F0F4
:10C29000E1FD2C4B1C6834B934F075FE10B0BDE8DC
:10C2A000F0870392C6E794FAA4F33846B3FA83F30F
:10C2B00005FA03F256F8231024EA020434F0B5FD1F
:10C2C000E9E700BF58A1012018E004081E42012040
:10C2D00032E0040828BB012070920408F2520120C9
:10C2E000EC52012043E00408849C012069E004082A
:10C2F00040420F00BE45012079E004082053012090
:10C300009AE00408EC0C0020A2E0040800000120E0
:10C3100000080000A6E00408202801200080000892
:10C3200000400008CAE00408782201200024744973
:10C330000800002044B304089EE5040804E1040852
:10C340004AE1040818BB012004000120F0B58BB0BD
:10C35000054634F039FC00286ED000223749012010
:10C360000BB0BDE8F040FFF7F3BA2D2903D0A1F1DF
:10C370003003092B5BD8052C04DD0BB0BDE8F04081
:10C3800034F080BE284618F083F80AAB621C03EB39
:10C39000440424F80C0C15F8013F303B092BFAD962
:10C3A000144629780029E0D1062CE6D1BDF91C30CD
:10C3B0009AB2072AE1D8BDF91E4040F2DC50A4F23F
:10C3C000EE2292B28242D8D8BDF92050A5F2EE22D8
:10C3D00092B28242D1D8BDF92260B442CDDCB542DE
:10C3E000CBDBBDF9247007F1640292B2C82AC4D82D
:10C3F000BDF926001128C0DCDFF848C00C2240B28D
:10C4000002FB03C2A2F8BC44A2F8BE54A2F8C06466
:10C4100082F8C27482F8C304094A0094CDE903701B
:10C42000CDE90156084634F0A9FE0BB0F0BD202935
:10C43000A3D101352246B3E70446B2E7D82C012048
:10C44000CFDC04082028012038B50446114D2046D1
:10C4500034F0BAFB68B1104B93F909104B1C06D1AC
:10C460000E4B59780E48BDE8384034F00FBEC9B2C3
:10C47000F8E7204618F00CF8052804D8C0B22C467E
:10C480001FF0E2FAE3E705210648BDE8384034F042
:10C49000DBBD00BF222F050800000120FCAE0120FB
:10C4A00060E104086FE10408052838B50D460FD88F
:10C4B000084C6072084835F0EBFB0848FFF7C4FFF2
:10C4C00034F061FD2946102034F062FDFF236372D1
:10C4D00038BD00BF000001208FE10408222F0508AD
:10C4E00038B50446114D204634F06EFB68B1104B50
:10C4F00093F90A104B1C06D10E4B19780E48BDE873
:10C50000384034F0C3BDC9B2F8E7204617F0C0FF89
:10C51000022804D8C0B22C4614F05EFBE3E70221E7
:10C520000648BDE8384034F08FBD00BF222F050813
:10C5300000000120FCAE012064E1040874E104085D
:10C540002DE9F74F3C4B00253C4C1A78A8465B7808
:10C55000DFF8ECB00090A272637235F0BBFB1BF009
:10C560004DFA28F00DFA0D27354B00996F43DE196F
:10C57000D6F80090484617F0C9FE00283DD0B8F123
:10C58000000F01D034F0FFFC49462E485F4434F0E0
:10C590004CFC0021304634F0EBFC34F0F4FC3B79E9
:10C5A00003F01803082B3BD0102B3DD0304634F05D
:10C5B0007CFD0D2303FB05B3B3F809001BF03CFA27
:10C5C0000746C0B1304634F04BFB8246D7E9012123
:10C5D00002440144304634F0CEFB60B90190494634
:10C5E000194834F022FC7968019A3046514434F0FD
:10C5F00041FC34F0C8FC08F10108013540F2691330
:10C600009D42B0D135F050FBFF23A3726372B8F1A5
:10C61000000F0DD10D4803B0BDE8F04F34F014BD4C
:10C620000B48FFF75DFFC1E70948FFF70DFFBDE7C6
:10C6300003B0BDE8F08F00BFFCAE01200000012078
:10C64000FC9D0408D02D05089BE10408ABE104081B
:10C65000222F0508022838B50D460FD8084CA072C5
:10C66000084835F015FB0848FFF73AFF34F08BFC1B
:10C670002946082034F08CFCFF23A37238BD00BF8C
:10C680000000012093E10408222F050838B5044674
:10C6900034F09AFA80B3224BDB680133172B21D890
:10C6A00020490C221C4602FB031295684DB91D4A15
:10C6B0000C210134172C17DD002401FB04208568B0
:10C6C0009DB1174BDC6023F007F82A462146164837
:10C6D00034F0DCFC0C235C43124B185DBDE83840A1
:10C6E00023F016B81C46E2E7E7D99C42E1D10F4897
:10C6F000BDE8384034F0A8BC204617F0C9FE172822
:10C70000044606D8074A0C2303FB00239D68002D2E
:10C71000D7D121460648BDE8384034F0B7BC00BF49
:10C7200000000120D0D10408E2E10408B8E10408C7
:10C73000CCE104082DE9F341054634F045FA0446FE
:10C7400020B134F09FFC02B0BDE8F081284601AA78
:10C750002A4927463BF0BFF826460546DFF89C806D
:10C7600075B9022CEDD1A7F57A73B3F57A7F1FD98D
:10C770004FF4FA624FF47A71214834F07BFCE2E71F
:10C780004CB1012C0FD001AA4146002001343BF0EE
:10C79000A2F80546E4E701212846FFF799FA431C71
:10C7A0000646F0D1CFE7284617F072FE0746EAE7C3
:10C7B000B8B236F0ADF9FF2EBCEEC00A114B0BD16A
:10C7C000114AF8EE407A1278AA4212DC10EE101AE2
:10C7D0000E4834F05BFCB6E7F8EE407A03EB8603D4
:10C7E00010EE102A31460A48C3ED007A34F04EFCB0
:10C7F000A9E7E3EC017A0135E6E700BF8B140508F1
:10C80000FAE60408382D0120E40C002004E20408B4
:10C81000F7E104082DE9F04F014691B0064686483D
:10C8200034F034FC854B864D4024C3F800D00023FF
:10C83000844906222B703046834B09781C700123F3
:10C840001EF01EF80A2014F0B7FC2B78DBB20C2B7C
:10C8500040F2ED809DF80C90B9F1FE0F2ED0B9F1A9
:10C86000FF0F15BF0F241524002601269C4240F01F
:10C87000DE80611E6846C9B212F078F810AB1C4425
:10C8800014F8413C834240F0CE8006F1FF389DF819
:10C890000D40B8F1010F13D904F01F0765094C468C
:10C8A00061376A4834F0D6FA022E71D0013D042D6A
:10C8B0006AD8DFE805F00A5D616965000226D5E700
:10C8C0009DF80E709DF80F50EBE7614835F05EF86B
:10C8D0000025DFF8D4914FF0030ADFF8D0B15D48AE
:10C8E00034F0B8FA1DF805100135484634F09DFAC9
:10C8F0000C2D55D134F047FB022E5BD064223B4611
:10C900005548B4FBF2F102FB1142C9B2D2B234F085
:10C91000BDFB5FFA88F8B8F1010F7BD84F4A504B46
:10C920009DF810104F4800290CBF114619464E4D76
:10C9300034F0ACFB9DF811104C4B4D4800290CBF56
:10C940002946194634F0A2FB022E63D19DF812400D
:10C95000484834F07FFA9CB3FF2C41D00A22464865
:10C96000B4FBF2F102FB1142D2B234F08FFB2AE0A9
:10C97000424835F00BF8ABE7414835F007F8A7E738
:10C98000404835F003F8A3E73F4834F0FFFF9FE746
:10C9900000230DF11F008DF83F3034F0F7FF97E7CB
:10C9A00095FBFAF303EB43039D429BD1584634F0C9
:10C9B00051FA97E73A462146344834F067FBA8E736
:10C9C000284634F0E3FF9DF81340314834F042FA32
:10C9D00054B1FF2C21D021462E4834F057FB06E0FD
:10C9E0002D4834F0D3FFEEE71F4834F0CFFF00248A
:10C9F0001D4D1E4E284F0DEB04031A7D8AB1FF2AF0
:10CA000014BF32463A4621460134244834F03EFBF6
:10CA1000042CF0D111B0BDE8F08F1F4834F0B6FF00
:10CA2000E5E72A46EFE71E4834F00EFBF2E71D4823
:10CA300034F0ACFFEEE700BF33E20408E049012028
:10CA4000EE490120E40C0020EF49012044E20408F3
:10CA50004FE204087DE2040894E204081CE20408A2
:10CA600013E20408CBE2040823E20408D9E704082F
:10CA7000E2E20408E9E20408FDE2040856E20408E0
:10CA80005EE2040866E2040875E20408B0E2040805
:10CA900005E304081C2E050827E2040815E3040832
:10CAA00020E3040830E304088FE20408B614050804
:10CAB0002DE9F74F054634F087F8044618B9374B8F
:10CAC0009B78042B04D834F0DDFA03B0BDE8F08F76
:10CAD00001272646DFF8E08001AADFF8E09028462B
:10CAE000DFF8DCA02E493AF0F6FE40B92D4B2E4A75
:10CAF0001B689B1A2D4A18BF01231370E5E766B91E
:10CB00000121FFF7E5F8421C0446DED001AA2449C2
:10CB1000002001363AF0DFFEE7E717F0B9FC2F28D6
:10CB2000054635D807B31EF011FD062D0CD10520A2
:10CB300014F042FBDAF800301B0125D5FF2C1FD082
:10CB4000E0B2FFF767FE09E0012014F035FB184959
:10CB50000123EAB20978E0B21DF092FE2946484668
:10CB600034F094FA0027D1E70628F0D1E2E7FFF786
:10CB700051FEF8B29BF8003001378342F7D8EDE759
:10CB80000027DFF82CB0F4E70A4834F0FFFEE5E7B1
:10CB90002F21404634F058FAB8E700BF4CB10120CD
:10CBA0008B140508BC2800206981020865B10120AA
:10CBB000E40C002039E3040859E3040848E30408BE
:10CBC0000CB0012013B5204C237C022B2FD1012364
:10CBD0000DF10702F52104F1100015F01FF940B323
:10CBE0009DF80710194834F051FA237C022B22D10A
:10CBF00001230DF107029A21154815F00FF9E0B154
:10CC00009DF80710134834F041FA237C022B16D10B
:10CC100001230DF107029B210D4815F0FFF880B1AB
:10CC20009DF807100C4834F031FA02B010BD002115
:10CC3000D8E70146D6E70021E4E70146E2E7002114
:10CC4000F0E70146EEE700BFC820002079E30408C2
:10CC5000D82000208CE304089FE30408024BD3F89B
:10CC60009C0409F019BF00BF202801200A4C05468A
:10CC70000A4808B534F0EEF8D4F8980415F03EFAF6
:10CC8000D4F89C0422F07AFB38F094FC0DB129F022
:10CC90005DFF29F06DFF00BF2028012063DC040840
:10CCA000094C0A4808B534F0F3FF94F838250AB166
:10CCB00014F01CF894F839350BB113F0F7FF15F0A8
:10CCC000CFFD0020FFF7D2FF20280120B2E30408A7
:10CCD0000A4D00240A4808B534F0DAFFD5F8980464
:10CCE00015F00CFA074B85F83A45C5F83C461C7020
:10CCF00038F0EEFD2046FFF7B9FF00BF20280120E5
:10CD0000B9E30408D85C0120034808B534F0C0FF3B
:10CD10000120FFF7ABFF00BFE0E304084A402DE924
:10CD2000F04F984685B0D34306460D4600241B4F6E
:10CD30000393204622F0BEFC0E9B184228D0039B92
:10CD4000174A0342DFF85CA014BF4FF001094FF00F
:10CD5000000910EA05033046494602934FF00C03E0
:10CD600003FB042314BF3A465246D3F808B04346A7
:10CD7000CDF800B034F0EAF9029ACDF800B043469D
:10CD8000002A14BF52463A464946304634F0F6F976
:10CD90000134172CCDD105B0BDE8F08F6A2E0508FF
:10CDA000D0D10408FEE30408F8B54D1E064601F193
:10CDB0001F04054F15F8012F30463946023616F08C
:10CDC00053FFA542F6D1F8BD8FE204082DE9F041EA
:10CDD0009AB0074639F064FB064601AD20220021D7
:10CDE00028463CF0FFF816B3402E07D040223146CB
:10CDF0002D4834F029F91AB0BDE8F0810024A0468E
:10CE0000022207EB440168463CF0E2F900231022BD
:10CE100009A968468DF8028017F0B0FA099B0DF158
:10CE2000020293421FD128550134202CE8D141221F
:10CE3000002109A81D4C3CF0D5F846B394F84036C3
:10CE4000B3B1202204F2416128463CF0A3F878B146
:10CE500004F2416109A8FFF7A7FF09AA1449154880
:10CE600034F0F2F8C7E71978134834F0EDF8C2E768
:10CE7000284613F0CDFE0123104909A884F839355E
:10CE8000FFF792FF09A90E4834F000F9B3E794F8D0
:10CE900039351BB994F84036002BF3D0074909A85F
:10CEA000FFF782FFEEE700BF05E404082028012019
:10CEB00043E404084DE4040827E40408612E01203B
:10CEC00077E4040870B5054639F0EAFA064600B37F
:10CED000134C94F861369BB104F2626039F0E0FAC9
:10CEE000B042024605D1294604F262603CF05EF988
:10CEF00060B10C4A0C490D48BDE8704034F0A4B84C
:10CF00000422294604F262603CF062F9012384F8AD
:10CF1000383504490648BDE8704034F0B7B800BF62
:10CF200020280120822E012084E404084DE4040816
:10CF300094E4040870B5054639F0B2FA064600B329
:10CF4000134C94F861369BB104F2676039F0A8FA8B
:10CF5000B042024605D1294604F267603CF026F94A
:10CF600060B10C4A0C490D48BDE8704034F06CB813
:10CF70001422294604F267603CF02AF9012384F860
:10CF8000383504490648BDE8704034F07FB800BF2A
:10CF900020280120872E0120A7E404084DE404087E
:10CFA000B2E4040870B50646124C39F079FA054629
:10CFB00090B11122002120463CF014F82A460E4977
:10CFC00030463CF0F3F838B1102D2A463146204661
:10CFD00028BF10223CF0FCF823780120054A002BE2
:10CFE000054B0EBF012113460021044ABDE87040E5
:10CFF00034F0C4B8A0450120B6140508B8E404080C
:10D000002DE9F04F8BB0834633F0DEFD044638B196
:10D0100000224B490120FEF7DDFB0BB0BDE8F08F8D
:10D02000584617F035FA0928054600F38380DFF8E3
:10D030001CA186008DF81F4037180AF27C680BF19E
:10D040000100544633F0C8FD08EB07098346C24689
:10D0500058B117F01DFA0D2807D8E31983F87C069C
:10D060009DF81F3001338DF81F30584633F0B4FD62
:10D07000834660B117F00CFA052808D873192344C9
:10D0800083F87D069DF81F3001338DF81F30584618
:10D0900033F0A2FD834660B117F0FAF9082808D8EA
:10D0A0007319234483F87E069DF81F3001338DF8F1
:10D0B0001F30F91C0DF11F025846514433F098FD02
:10D0C0009DF81F20052A2DD1002308A94846089362
:10D0D0008DF824303BF05EFF7319234493F87D16DE
:10D0E00018B1F9B193F87E36E3B12E444FF4617074
:10D0F0001923344494F8802613FB0202049294F816
:10D100007F2613FB02030F4A039394F87E36CDE982
:10D110000113002194F87C36084600932B4634F026
:10D120002DF87AE7002348F8073089F8043033F007
:10D13000A9FF72E709222146034833F09BFF6CE701
:10D140009C2E01209CDC0408C0E404082028012057
:10D15000F8B528F01BF858B3164D00241648174FA1
:10D1600034F014FCD5F8980414F0C8FF27F0D0FC74
:10D1700028F014F8064648B1132022F0C9FA33F01B
:10D1800002FF0F48BDE8F84034F000BC384633F0E9
:10D190004CFE782C08D80134D5F8980414F0AEFF72
:10D1A000642014F009F8E3E733F0EDFE3446F3E7CA
:10D1B000F8BD00BF20280120C6E404082613050896
:10D1C000E0E404081FB527F0B9FC044627F072FC20
:10D1D000A38921880290A268044801926288009283
:10D1E000626833F053FF04B010BD00BFE6E40408EA
:10D1F0007FB5054633F0E8FC044630B100221849FB
:10D200000120FEF735FC04B070BD2846154E01AD77
:10D210006A4614493AF05FFB78B1032C02D133F02F
:10D2200031FFF0E717F034F96A4645F8240031463B
:10D23000002001343AF04FFBEEE7032CEFD1039EC0
:10D24000DDE9014532462946E0B208F003F900283D
:10D25000E5D033462A462146034833F017FFD2E78C
:10D26000583601208B140508FCDC04087FB50646FF
:10D2700033F0AAFC054638B100221B49012004B056
:10D28000BDE87040FEF772BC304617F001F90F2878
:10D29000044620DC304633F09FFC0146204608F06F
:10D2A00003F998B104F12002104B03EB8201C87816
:10D2B0000290284689780191294633F822300C4A99
:10D2C0000093234633F05AFF04B070BD04B0BDE8AC
:10D2D000704033F0D7BE0F222946064804B0BDE89F
:10D2E000704033F0C7BE00BFD83601205836012049
:10D2F00010DD0408C0E404082DE9F04F8FB00746A4
:10D300008A46164600240DF12409DFF85C805AF89D
:10D310002430494602A8029331F096FF16B356F81E
:10D3200024300DF1100B029D03A803935946EB1A0C
:10D330005D425D4131F088FFCDF800B023464246A2
:10D340002946384633F002FF23460134CDF80090D9
:10D3500042462946384633F011FF202CD7D10FB072
:10D36000BDE8F08F3546EFE741E5040870B588B0B9
:10D37000064633F029FC054630B10022154901204C
:10D38000FFF7BAFF08B070BD304617F081F81F28CC
:10D39000044619DC304633F01FFC0146204608F0F5
:10D3A000B7F970B103AE0B48314600EB840031F0A1
:10D3B0004BFF00962346084A2946284633F0DEFEF6
:10D3C000E0E733F05FFEDDE71F222946034833F034
:10D3D00051FED7E75836012041E50408C0E40408AF
:10D3E000154B9B78012B04D0144B0146186814F0A0
:10D3F00003B8134910B40A78124C531CA054DBB282
:10D400001A060B7013D41A460F490978994205D8A9
:10D41000521A3F2A07D85DF8044B7047C1F18001CA
:10D420000A443F2AF7D95DF8044B27F075BE002364
:10D430001A460B70E8E700BF903D01200845012027
:10D4400090450120104501200D450120F8B500212F
:10D450000446021F064600F1080752F8043F03F194
:10D46000200003F1080502333F283DD80F2D18D8BE
:10D47000032B02D9002908BF01219742EDD10129D0
:10D4800021D002290FD1206800F03F0040F0800039
:10D49000FFF7A6FF2079FFF7A3FF207ABDE8F84049
:10D4A0009EE70221E9E7D4E90032A0681B0192005F
:10D4B00000F0030003F0300302F00C0213431843A2
:10D4C000BDE8F8408CE7206800F00F0040F0400015
:10D4D000FFF786FFD4E9013000F00F0040EA0310A7
:10D4E000BDE8F840C0B27BE704F10C0700253A46DE
:10D4F00052F8043DAD0003F1800103F50040FF291F
:10D5000006D9B0F5803F03F5000319D245F00105B7
:10D51000A242EDD165F03F00C0B2FFF761FF05F018
:10D5200003033278022B27D0032B104616D0012B91
:10D530000ED0FFF755FF0436AD10B742EFD1F8BD5E
:10D54000B3F1807F34BF45F0020545F00305DFE706
:10D55000FFF746FF7078FFF743FFECE7FFF740FF68
:10D560007078FFF73DFFB6F90200C0B2FFF738FF51
:10D5700096F90300C0B2DCE71046FFF731FF707880
:10D58000FFF72EFFB6F90200C0B2FFF729FFD2E77E
:10D59000084625E77F2810B5044607D964F07F00C8
:10D5A000E409C0B2FFF71CFF7F2CF7D8E0B2BDE85A
:10D5B000104015E738B5044600EB410534F9023B4D
:10D5C000D81780EA4300FFF7E5FFA542F6D138BD42
:10D5D000C31783EA4000DDE7F8B50F4BD3F8B05628
:10D5E000D3F8B476D3F8B866A9B1831E00EB410135
:10D5F0003C181E440F441D4434F9022B36F9023FF7
:10D6000035F9020F9B1848BF0133A0EB6300FFF709
:10D61000DFFFA742F0D1F8BD2028012038B5194D11
:10D6200004464720FFF7DCFED5F8BC361B0305D5C2
:10D63000D5F8B4361868201AFFF7ACFF124CA07C5E
:10D64000FFF7A8FFD5F8C0362068C01AFFF7C0FF63
:10D65000D5F8C4366068C01AFFF7BAFFA068FFF7B4
:10D6600099FFA089FFF796FFE089FFF793FFA17C60
:10D67000D4E9002385F8D016C5F8C826C5F8CC36FD
:10D6800038BD00BF20280120E45E0120F0B52B4CFE
:10D6900085B02B4ED4F8E076D4F8E45629492A48D0
:10D6A000AF42D4F8D43694F8DC263678097890F86E
:10D6B000200027DB01ADC4F8E83684F8EC6684F876
:10D6C000ED0684F8EE1684F8EF265320FFF788FE67
:10D6D000D4F8E806FFF75EFF94F8EC06FFF75AFF70
:10D6E00094F8EF3694F8ED16284694F8EE26039356
:10D6F000CDE90112FFF7AAFE00230120C4F8E036AD
:10D7000005B0F0BDD4F8E87601AD8DF8086004F5F9
:10D71000DD66BB4201938DF809008DF80A108DF883
:10D720000B2004D095E8030086E80300CDE76A6883
:10D7300073689A42F6D10020E2E700BF202801205A
:10D74000E15E0120D5370120C45201200EB470B52E
:10D7500083B00646482007AC54F8045BFFF740FE50
:10D760002020FFF73DFE30460AF08CFA3A20FFF702
:10D7700037FE2A46234609490020019416F0A2F9F3
:10D7800004460A20FFF72CFE054A033413681B1BCE
:10D79000136003B0BDE8704003B0704791D5000836
:10D7A000044501201E4900221E4B0968C3F8F026DB
:10D7B0001F29A3F8F426A3F8F626A3F8F826C3F841
:10D7C000E02623D03F291CD04FF4FA42B2FBF1F1FE
:10D7D000A3F8FA161448B3F9FA26018829B11F2ACA
:10D7E00001DD914217DC92FBF1F1A3F8FC16817880
:10D7F00012020E480031C3F8E42618BF012101705F
:10D8000070474FF40072A3F8FA26E3E74FF4806202
:10D81000A3F8FA26DEE70121A3F8FC16E7E700BF2C
:10D82000F835002020280120903D01208E3D012068
:10D83000194BB3F8F426D3F8E0060132D3F8F0160A
:10D84000013092B2013110B4B3F9FA46C3F8E006E0
:10D85000A242C3F8F016A3F8F4260FDAB3F8F826BC
:10D86000B3F9FC16013292B28A42A3F8F82602DB21
:10D870000022A3F8F8265DF8044B7047B3F8F626AB
:10D8800000215DF8044B0132A3F8F416A3F8F81652
:10D89000A3F8F626704700BF202801202DE9F04F9D
:10D8A0005E4D85B0904600290CBF042206220193EC
:10D8B000D5F80437DDF838905C1C02920F9F67D0D2
:10D8C000994544DDDFF868A157B1109AD5F8BC1628
:10D8D000D01B012203FB00F0385C82400A422FD0AB
:10D8E000019AA2EB0804D5F8002703FB04F408EB27
:10D8F0000406002A37D158F8040038F0D1FD00F1B1
:10D90000050B58460AF05EF9A0BBDAF8000095F85E
:10D910000827A0EB0B00CAF80000002A34D101232D
:10D9200085F80837D5F8003743BB58F804000AF0EB
:10D93000A9F996F904104B1C02D03948FCF760FB9A
:10D94000D5F80447631C4B45C5F80437BCDB994543
:10D950004ED0D5F80007029B834294BF00200120DF
:10D9600005B0BDE8F08F4FF0030B58460AF02AF9D6
:10D970000028CAD0012005B0BDE8F08F1E44294818
:10D980003179FCF73DFBDBE72C20FFF729FDC9E7E8
:10D99000D5F80037934203D3002005B0BDE8F08FDF
:10D9A000214C0646039104EB8303D3F8640638F058
:10D9B00077FD0B300AF006F9039982460028D9D189
:10D9C000D5F80037194804EB8304032B98BF314680
:10D9D000D4F86426FCF714FB1549D5F804370A6817
:10D9E000013385F808A7121AC5F804370A6067E7FB
:10D9F00001200AF0E7F80028ABD10D4A0A2013688D
:10DA0000013B1360FFF7ECFCD5F800074FF0FF3344
:10DA10000130C5F80437C5F800079CE7202801202D
:10DA2000A4E804081C2E05087092040894E8040871
:10DA3000044501202DE9F04F984E87B0B378012BB3
:10DA400033D0032B01D00323B370802021F0B0FD2D
:10DA5000074620B38021924D21F0A0FD7C79914AA8
:10DA6000002397F90270022152F824200C3C85F81B
:10DA700009073846B2F5613F14BF1F460F46CDE98E
:10DA8000002102971A46802121F098FC864B032C36
:10DA9000186000F2E480854B40221A7088B9844BEC
:10DAA00000221A7007B0BDE8F08F27F06FFB002846
:10DAB000F5D0B3787A4D012B00F0E4807B4B402207
:10DAC0001A70002395F866807A4AB8EB030896F836
:10DAD00003C017681C46DFF8F4E118BF4FF00108D7
:10DAE000BCEB030C74499EF806B01A4618BF4FF001
:10DAF000010C17F0020FDFF8D89101F1500A14BFA2
:10DB0000604618469EF805E01BF0FD0FB6F800C011
:10DB100001F1CC06B9F802B008BF9946674F18BFAB
:10DB20004FF00109BEEB030EC5F8B4663F7801F56E
:10DB3000A47618BF4FF0010E1CF1FF3CC5F8B86683
:10DB400018BF4FF0010C95F88868FF1AC5F8C03669
:10DB5000C5F8B0A618BF0127DFF878A1012E18BFBD
:10DB6000192EC5F8BC36A5F884B808BF0126DAF826
:10DB700000B018BF00260590C1E90133C1E90333A5
:10DB80004F4B93F800A0D3B2591E15290ED8DFE8E9
:10DB900001F01A1A1A1A1A1A1A1A24101038161022
:10DBA00034282828400B3C10059931B101219140BF
:10DBB0000C430133DBB2162B2FD80132E3E7494681
:10DBC0000029F3D1F9E79A4534BF0021012100294A
:10DBD000EFD0012191400C43EBE731460029E5D11C
:10DBE000EBE702EB42010BEB410111F8561C00314F
:10DBF00018BF01210029ECD1DBE741460029D5D12E
:10DC0000DBE771460029D1D1D7E739460029CDD1CC
:10DC1000D3E761460029C9D1CFE71620C5F8BC4635
:10DC200038F03CF80023D5F890680221D5F8D446A6
:10DC30001F4A85F88B08C5F8F036A5F8F436A5F824
:10DC4000F636A5F8F836C5F8E03685F89838C5F800
:10DC50008C68C5F89448117007B0BDE8F08F194B77
:10DC6000194A1B6803EB4303A2FB03235B0912D091
:10DC7000402BA8BF4023DBB20C4A137000287FF46E
:10DC800020AF0CE726F05AFFD5F80C3782689A428D
:10DC90003FF614AF03E70123EEE700BF903D0120FC
:10DCA00020280120FCB00408084501200C45012073
:10DCB0008E3D012020530120E02E01206D9C01208B
:10DCC000E40C0020F8350020D34D621004530120ED
:10DCD000EC520120FC5E012008B5084B9B78032B19
:10DCE00006D0FFF7A7FE064B012283F8992808BD4E
:10DCF00030F0B6FC0028F4D008BD00BF903D0120F4
:10DD00002028012038B5FCF703FA054618B1094B65
:10DD10001868FCF789F909242AF0DCFB0028FBD1FC
:10DD20002AF0D8FB18B1013CF6D1284638BD20F0C6
:10DD300097FEF8E7EC27002000B5ADF2946D40F2B5
:10DD40008C62094901A839F091FD039B1BB10DF1CB
:10DD50005E0101A89847BDF85E20044B1A800DF2C1
:10DD6000946D5DF804FB00BFC8200020E80C002083
:10DD7000924B93491B88934A896AA2F8023400297E
:10DD800000F0098107EE903A9FED8F7A9FED8F3A70
:10DD9000F7EE004AB8EE676A07EE901AF0EE432AF3
:10DDA00002F20443F8EE677A02F58E62DFED881A1C
:10DDB0009FED882A26EE276ADFED870A9FED870A06
:10DDC0009FED871A26EE076A9FED865A2DED048B8C
:10DDD000FDEEC67A36EE033A17EE900AFDEEC37AF0
:10DDE000203017EE901A2031402800F2A180B4EEC6
:10DDF000E16AF1EE10FA40F3D880B0EE467ADFED3A
:10DE00007A5ADFED7A6AB4EEE67A77EE657AF1EE69
:10DE100010FAB0EE677AF6DCF4EEC27AF1EE10FAA0
:10DE200040F1BA80DFED705ADFED716AF4EEE67A08
:10DE300037EEA57AF1EE10FAF0EE477AF6D4B4EEAA
:10DE4000E27AF1EE10FA00F3A080DFED6A7AB4EE28
:10DE5000E77AF1EE10FA48BF32EE477A67EE077ABA
:10DE6000DFED656AB0EE404A4029F0EE413A67EED8
:10DE7000275AA7EEA04AE7EE843AB0EE644AF0EEE5
:10DE8000647AA5EEA37AA7EE264AE7EE667AC7EE95
:10DE9000843A53D8B4EEE26AF1EE10FA40F3888087
:10DEA000B0EE437ADFED505ADFED506AB4EEE67A19
:10DEB00077EE657AF1EE10FAB0EE677AF6DCF4EE02
:10DEC000C27AF1EE10FA76D5DFED475ADFED486AF7
:10DED000F4EEE67A37EEA57AF1EE10FAF0EE477A34
:10DEE000F6D4B4EEE27AF1EE10FA51DCDFED417ACD
:10DEF000B4EEE77AF1EE10FA48BF32EE477A67EEF9
:10DF0000077AF0EE408AB0EE419A67EE275AE7EEC4
:10DF1000A08AB8EE008AF6EE006AA7EEA89AA5EEEF
:10DF2000897A74EEC75A27EE087A65EEA66A0BE086
:10DF3000F7EE003A4029B0EE634AABD9F6EE006A3C
:10DF4000B0EE457AF7EE005AC4EE847AC3ED043A97
:10DF500083ED065A243303ED045A03ED015A03ED11
:10DF6000025A67EEA66A67EEA55A27EE877A43ED56
:10DF7000096A43ED076A43ED085A03ED067A9A42AF
:10DF80007FF432AFBDEC048B704731EEC77A65E7A2
:10DF900031EEC77AB3E77047B0EE677AB4EEE27A53
:10DFA000F1EE10FA7FF751AFEFE7F0EE467A33E784
:10DFB000F0EE437A83E7B0EE677A92E704BB012084
:10DFC000EC0C00202028012027D4D236DB0FC93FDB
:10DFD000DB0F4940DB0F49C092E741B99730083C5D
:10DFE00015A82ABE00000000DB0FC940E4CB164193
:10DFF000E4CB16C1DB0FC9BFF304353F154B6422D8
:10E000001549187C93F9243007EE100ADFED135AF6
:10E0100007EE903AB1F88C30F8EEC76A9FED106ABF
:10E0200007EE103AF8EEE77A0E4BB8EEC77A67EED5
:10E03000A57A26EE877AE7EE067AFCEEE77A17EE07
:10E04000901A88B202FB00F283FB02301044C0F346
:10E050004720704768B10120202801200AD72341BA
:10E060000AD7233C03082080114B124A197C93F9EC
:10E07000243007EE101ADFED105A07EE903AB2F88E
:10E080008C30F8EEC76A9FED0D6A07EE103AF8EE95
:10E09000E77AB8EEC77A67EEA57A26EE877AE7EEDA
:10E0A000067AFCEEE77A17EE903A98B2704700BF16
:10E0B00068B10120202801200AD723410AD7233C38
:10E0C0002DE9F84F3A4B3B4CD3F8B06604F13C0ACB
:10E0D000394F06F13C0B3546DFF8F890D84645F845
:10E0E000040BD4ED007A143454ED046AFDEEE77AA3
:10E0F00014ED037AFDEEE66AB7EC010ABDEEC77ACD
:10E1000017EE902A54ED027AFDEEE77A45F8042BDB
:10E11000C5ED026A85ED057AC5ED087A39F040FC57
:10E12000B9EC010A28F8020B39F03AFC5445A8F87A
:10E130000400D6D1214A06F13403F2EC017AFDEE57
:10E14000E77A17EE901A23F8021B5B45F5D11C4BBA
:10E150001C491A885888A6F8482009789A88DB88CC
:10E16000A6F84A00A6F84C20A6F84E3071B106F188
:10E170005003154A03EB4101F2EC017AFDEEE77A18
:10E1800017EE900A23F8020B9942F5D10F4A104B73
:10E1900052885B68A6F870207367FFF765FF044B31
:10E1A000A6F87800B3F8CA38A6F86A30BDE8F88F48
:10E1B00020280120A8360020F0270020F45201205A
:10E1C000709C0120E40C002014000020EC5201207F
:10E1D00014530120180D00202DE9F04F7A4C8DB01A
:10E1E0008046B4F8F436002B40F0FE80774F3B8831
:10E1F000002B00F0A2804046FFF762FFD4F8B05633
:10E2000049202E46FFF7ECF8D4F8F006FFF7C2F9E4
:10E2100056F8040BFFF7BEF9304630F097FA05F1D7
:10E22000100030F093FAD4F8BC36DB0300F1A18083
:10E23000D4F8BC369E0300F19380D4F8BC36580362
:10E2400000F1BD8005F1280030F080FA032105F1CE
:10E250003400FFF7AFF95E4BB5F93A001B8AC01ADC
:10E26000FFF798F9D4F8BC36D90400F199809A04E4
:10E2700000F18D801E0400F1858005F13C00032132
:10E28000FFF798F9D4F8BC36D8025FD4990257D476
:10E29000B5F9503007EE903A4E4BF8EEE77A93ED31
:10E2A0000B7A77EEC77AFCEEE77A17EE900AFFF763
:10E2B00071F9494B1B78012B0ED905F1500805F176
:10E2C000520608EB430836F9020BB5F95030C01A74
:10E2D000FFF77EF9B045F6D1D4F8BC369A0525D4BF
:10E2E000D4F8B02601253D493D4B501AC4F8B42658
:10E2F000C4F8B82680103B4A84F8985803FB00F312
:10E300002B4482FB0302A2EBE37202EB42029B1A54
:10E31000C3EB431301EB8303C4F8B036BB78012B86
:10E3200001D126F0F9FE0DB0BDE8F08FB5F96A0015
:10E33000A0F2DC50FFF74CF9D2E7FFF7A7F95AE754
:10E34000042105F14800FFF735F9A1E7032105F1A4
:10E350004200FFF72FF9D4F8BC36990298D5EFE7C1
:10E36000286AFFF735F9D4F8BC3658037FF56AAF51
:10E3700025E0E869FFF72CF9D4F8BC369E037FF559
:10E380005CAFEDE7B5F87800FFF704F975E7686F63
:10E39000FFF71EF9D4F8BC361E047FF56EAFF1E727
:10E3A000B5F87030B4F88408C01AC0F30D00FFF758
:10E3B000F1F8D4F8BC369A047FF55CAFE7E7686AF9
:10E3C000FFF706F93EE700BF20280120903D01201D
:10E3D0004CB1012008000020E40C0020302F012067
:10E3E000DF7BEFBD56555555D4F89058D4F88C388E
:10E3F000AB4207D0CE4BC4F88C581B78093B012B9D
:10E4000040F2B981D4F89468D4F8D456AE4207D01B
:10E41000C74BC4F894581B78093B012B40F29E81EE
:10E42000B4F8F836C34F002B40F0DD803B88002B5A
:10E4300000F0D980FFF72AF94046FFF741FE50204F
:10E44000D4F8B0A604AED4F8B4B6FEF7C9FFD4F839
:10E45000B8261025D4F8B0364FF0010910681B68B3
:10E46000D4F8B42603441068A3EB4000FFF7B0F8DB
:10E470000BF104020AF10401304630F079F830461D
:10E4800030F064F930460BEB05020AEB050130F081
:10E490006FF83046FEF7DAFF09FA05F3D4F8BC2628
:10E4A000134240F0F1800135132DF5D10BF1280214
:10E4B0000AF128013046B14630F05AF8304630F0C3
:10E4C00045F90AF134020BF134000AF13C0C3146F3
:10E4D00032F9023B30F9025B9445A3EB050341F8A6
:10E4E000043BF5D108AA0025AD0052F8043DEDB279
:10E4F00003F1080133B10F2903F1800300F2BD805D
:10E5000045F001059642EFD1002228460192FEF720
:10E5100067FF019A1346114605F00300022800F038
:10E520009E80032800F0878001287AD00133AD084F
:10E53000042BF1D1002940F07D81D4F8BC3603F4DE
:10E54000005103F40042DB0400F1CA80002940F0CE
:10E550001C815AB1BAF87830BBF878209B1A049322
:10E56000049BD81780EA4300FFF714F803213C20EE
:10E57000FFF732F8D4F8BC36DD0200F1548198027E
:10E5800000F14C816C4B50201978FFF725F8D4F836
:10E59000BC36990506D5BAF96A00BBF96A30C01ACB
:10E5A000FFF716F8D4F8B06601226449644B751A77
:10E5B000D4F8B40684F8982802F15532AD10C4F8A6
:10E5C000B806C4F8B46603FB05F3013382FB03020B
:10E5D000A2EBE37202EB42029B1AC3EB431301EB83
:10E5E0008303C4F8B036574B1B681A067FF596AE06
:10E5F000554DD4F8C0362A689A4251D04820FEF7CB
:10E60000EFFE2868FEF7E4FF6868FEF7E1FF40468A
:10E61000D5E90023C4F8C026C4F8C436FEF7FEFFCF
:10E620007CE656F823C0002940F0EB804FEA0C123C
:10E630000146D2B27AE756F82300002963D1C0F32D
:10E6400007200193CDE90212FEF7CAFE019B16F8DE
:10E650002300FEF7C5FE039ADDE9013166E756F8AF
:10E660002300002974D1C0B20193CDE90212FEF754
:10E67000B7FE039ADDE9013158E7FF2B94BF45F05F
:10E68000020545F003053DE7AB000AEB03025B44DE
:10E6900052F8240C53F8243CC01AFEF799FF02E705
:10E6A0006A68D4F8C4369A42A8D1B4F9FA36B4F8F4
:10E6B000F826002BB8BF0133B2EB630F00F0C58022
:10E6C000224B94F8D026997C914205D11968D4F850
:10E6D000C826914200F0B2804046FEF79FFF1DE63B
:10E6E000BAF87030BBF870001B1A049300297ED171
:10E6F000002A3FF436AFBAF878300221BBF8782010
:10E700009B1A059356E0C0F303301043CDE9013165
:10E71000FEF766FE019B56F82300C0F30710FEF7D4
:10E720005FFE019B029956F823201201D2B2FDE64A
:10E730008E3D0120903D0120E40C0020302F01206F
:10E74000DF7BEFBD0CB00120543E0120E45E0120D0
:10E75000C0F30310CDE901311043E0E74520FEF797
:10E760003FFE1E20FEF73CFE2846FEF713FF304614
:10E77000FEF710FF54E64520FEF732FE0020FEF7BC
:10E780002FFE2846FEF706FF3CE6DAF87430DBF889
:10E7900074105B1A0493002A3FF4E2AE0121BAF828
:10E7A00078300CAABBF8780002EB810201311B1A09
:10E7B00042F8203C890000207318400053F8042DD3
:10E7C000C0B20AB140F001009E42F6D10E44FEF7FD
:10E7D00007FE02E04E453FF4C9AE59F8043B002B5A
:10E7E000F8D0D81780EA4300FEF7D4FEF2E7DBF852
:10E7F0007410DAF874305B1A02210593002AD9D01C
:10E80000CDE70CF00F000021039310430291019219
:10E81000FEF7E6FD039BDDE9012187E604214820A0
:10E82000FEF7DAFEAEE603214220FEF7D5FED4F86D
:10E83000BC36A4E61046FEF7D3FD7EE65A68D4F84F
:10E84000CC369A427FF448AF68E5B4F8F6365B06FA
:10E850003FF4D4AE34E700BF2DE9F8438946017890
:10E86000A9B1DFF83C800546044608F10807464692
:10E8700030463AF086FCB8420BD2621BA0EB08038C
:10E8800038B109F8032014F8011F0029F0D1BDE8C0
:10E89000F88314F8011F0029EAD1BDE8F88300BF0E
:10E8A000EC9804082B4B42F201021B681A4200D17B
:10E8B0007047294B5B68C3F3080330B4CBB9EFF35F
:10E8C0001183B3B9254A264D264C1368A0681168F8
:10E8D0008B42FAD129688842F7D823494FF47A74D9
:10E8E0000D6804FB05F1081AB0FBF5F004FB030307
:10E8F0001DE0EFF31180102383F3128803F1E0236E
:10E900001A499D681A68D2031FD4144AC0B2146809
:10E910000B6880F3118814494FF47A7023440C6813
:10E9200000FB04F1491BB1FBF4F100FB0313156874
:10E9300001240F4902200F4A8D6081F8214082F89E
:10E94000D408C2F8D03830BC704701220A609D68F4
:10E95000DBE700BF0CB0012000ED00E058A1012072
:10E9600060A1012010E000E05CA1012054A1012081
:10E97000C4520120202801202C4B42F201021B68C6
:10E980001A4200D170472A4B5B68C3F3080330B4C6
:10E99000CBB9EFF31183B3B9264A274D274C13683F
:10E9A000A06811688B42FAD129688842F7D8244AB6
:10E9B0004FF47A71146801FB04F2101AB0FBF4F002
:10E9C00001FB03031EE0EFF31181102383F3128890
:10E9D00003F1E0239C681A6812F4803F194A20D1A1
:10E9E000144BC9B21868136881F31188144A4FF4A4
:10E9F0007A710344106801FB00F2121BB2FBF0F2C3
:10EA000001FB032310480224104982681944104B6B
:10EA100002F2DC5283F8D448C3F8D018826030BCCC
:10EA20007047012010609C68DAE700BF0CB001203D
:10EA300000ED00E058A1012060A1012010E000E0FD
:10EA40005CA1012054A10120C452012060E3160002
:10EA5000202801202DE9F047924D4FF0000C924CF8
:10EA600084B0924F688A04F6D401914A914B0FFA10
:10EA700080F9914E02F1240EC4F8CC7284F8D5C806
:10EA80008E4FDFF868C2C4F8A432C4F8C462C4F878
:10EA9000C872DCF8003022F8029F964503F59673A1
:10EAA00041F8043FF5D1DFF84882854BD8F800C023
:10EAB000DFF840E203F178011CF4805F08BFB5F98C
:10EAC0001E90AEF806900FE00AEB8A0A0AEB8A0A5B
:10EAD0000AF5617292B293F8019009F104092EF8D7
:10EAE00019200633994214D01A78002AF9D193F8E4
:10EAF0000290DA789145F4D209F1FF3A0132B9F186
:10EB0000000FE1D102EB820202EB820202F5617298
:10EB1000E1E71CF0080F32D11CF4804F41D11CF00A
:10EB2000010F0CF4005315D103BB1CF4004F22D18C
:10EB3000EB7B13B1022384F8663095F8222094F819
:10EB4000C012131D8B42A8BF0B4684F8083A04B0CC
:10EB5000BDE8F08744F62062A4F8C22293B30822ED
:10EB6000584B84F8C022C4F8C432DEE744F6206370
:10EB7000A4F8C232F3E7012384F86630DDE72B7A8C
:10EB80000C2B26D8DFE813F0BA00BA009702660211
:10EB9000ED02320132017A01BA01FA01BA00250010
:10EBA0002F00122244F62063474984F8C022A4F8BB
:10EBB000C232464A464BC4F8C412C4F8C822C4F84C
:10EBC000A432ACE70C22434B84F8C022C4F8C43210
:10EBD000ABE7082013F06AFBD8F800C0C4F8C462A1
:10EBE000C4F8C87298E703010A203B49002293FB4E
:10EBF000F0F3A3F5B0633948C4F8D0129BB2C4F85F
:10EC0000C40221F812300132122AFAD142F6F82356
:10EC10003349402084F8C022A4F8C232314BC4F8F2
:10EC2000C812C4F8CC3220F0C3FC0028D1D095F82B
:10EC30000AC0032390F902004FF4E131BCF1000F48
:10EC400001934FF000036A7A18BF4FF0080C00914F
:10EC500008BF9C4640219A4218BF4CF0010C224A42
:10EC6000CDF808C020F0AAFBC4F8F80378B1DFF8AB
:10EC7000889099F80030002B00F02083002394F84E
:10EC8000662084F8943012B9032384F86630D4F8EF
:10EC9000F833003318BF0123002B9AD0D8F800C0F6
:10ECA0003AE700BF68B1012020280120299B000815
:10ECB00052410120A0860100219B0008259B0008ED
:10ECC00040310120C99C00082D9B00083D9B000895
:10ECD000400D0300B99C0008043201204D94000847
:10ECE00031800008FDAB00084D84000858A10120C8
:10ECF0000CB0012054410120F3410120BB4B4020C6
:10ED0000C4F8083220F054FC814600283FF461AF7B
:10ED10004FF0000A84F8DEA106F042F92A7A034691
:10ED2000012A0ED0C0F0B6820A2A1FD1D8F80020DE
:10ED300082F48062C2F38022024382F0010284F8EE
:10ED4000DE21032107224FF0010C4FF4006084F80C
:10ED500004120C2184F80C2242F6F82284F8DCC15B
:10ED6000C4F8F40184F8C012A4F8C222697ADFF86A
:10ED7000D0C200319E48DFF8CCE218BF0121C4F8B0
:10ED8000C8C2C4F8C4E2C4F8CC024AB294F8DEC1E6
:10ED900099F90200002B40F04382BCF1000F40F0D3
:10EDA000778295F80AC0BCF1000F00F0C082012301
:10EDB00042F008024FF4E131CDE901320023009125
:10EDC00040218C4A20F0FAFA8B4B1860EB7B94F8C8
:10EDD000C022013BDBB29A4284F8F03102D8002312
:10EDE00084F8F031031C18BF012355E7062B4FF0C0
:10EDF0000C0240F0E28184F8FA3021210023DFF890
:10EE0000489284F8C02284F8F02084F8C83084F84E
:10EE1000F93084F8F83084F8EF1042F6F821774A98
:10EE2000774B4020A4F8C212C4F8C422C4F8C832F8
:10EE300020F0BEFB824600283FF4CBAE06F0B0F8CF
:10EE4000697A9AF902C00031AB7A18BF01214AB23F
:10EE5000002800F01082002B00F0B48242F008027B
:10EE60000321CDF8009060460292002301914021D9
:10EE7000644A20F0A3FA644B1860B3E744F62063B9
:10EE80000E21624A4FF00009A4F8C2324020604BC4
:10EE900084F8AC9384F8C012C4F8C422C4F8C83211
:10EEA00020F086FB824600283FF493AE4FF4805258
:10EEB000402120F069FB697A844684F8A993B1EB7C
:10EEC00009019AF9020018BF01214AB2BCF1000FF2
:10EED00000F0878142F0080203214FF4E13C4B46E9
:10EEE0000292019140214B4ACDF800C020F066FA11
:10EEF000494A4A4B106083F8009073E71023484A50
:10EF000041F27C514FF0000984F8C0322823C4F844
:10EF1000C4224020434AA4F8C21284F89893C4F84B
:10EF2000C82284F8993320F043FB00283FF451AE07
:10EF3000A97A032290F902004B464945019295F8BF
:10EF400009C04FF040010CBF4A460822CC4518BF0B
:10EF500042F00102DFF8F4C00292CDF800C0324A5C
:10EF600020F02CFA0121C4F8E00912F031FAD4F8AB
:10EF7000E039B3EB090318BF01238DE602010A2033
:10EF800000232A4992FBF0F2A2F5B06241F8232057
:10EF90000133102BFAD141F60B21254A84F8C032F7
:10EFA0004020244BA4F8C212C4F8C422C4F8C832CA
:10EFB00020F0FEFA00283FF40CAE00236A7A032109
:10EFC000DFF88CC0D21A90F90200CDF800C018BF4B
:10EFD0000122CDE90112184A402120F0EFF9174A29
:10EFE000031C106018BF012356E600BFE02A012071
:10EFF0007D8E00085993000800450120B185000866
:10F00000CD85000811890008EC410120559B0008BE
:10F01000A1AF00087D9D0008205D0120F85C012063
:10F02000659B0008D99C0008819B0008382A0120B4
:10F0300081970008B59700080DAD000888440120AD
:10F04000058F0008D58E000890D0030048E8010025
:10F05000A068060042F6F8231021C04A4020A4F818
:10F06000C232BF4B84F8C012C4F8C422C4F8C832FC
:10F0700020F09EFA814600283FF4ABAD05F090FFEA
:10F08000697A99F902C00031AB7A18BF01214AB2FE
:10F09000002800F0DE80002B40F084814FF0030E4A
:10F0A0004FF4E132029160464021CDE9002EAD4A95
:10F0B00020F084F9DFE602010A20DFF8B8C200235D
:10F0C000C4F8D012C4F8D4C292FBF0F2A2F5B06238
:10F0D000A54892B2C4F8C40221F813200133122BC0
:10F0E000FAD142F6F821A14A402084F8C032A4F8AF
:10F0F000C212C4F8C82220F05BFA814600283FF40F
:10F1000068AD05F04DFF6B7A00280CBF012103218B
:10F1100095F80AE0002B99F902208146944B14BF20
:10F120004FF0060C4FF0070CBEF1000F1046019196
:10F130004FF040010CBF0022082200934CEA020C61
:10F140008C4B8D4ACDF808C020F038F995F8233063
:10F1500013B1052384F86630B9F1000F3FF442AED5
:10F1600089E642F6F8230821844A4020A4F8C232F6
:10F17000834B84F8C012C4F8C422C4F8C83220F00B
:10F1800017FA814600283FF424AD05F009FF6A7A9A
:10F1900099F902100346003218BF012298B30323E5
:10F1A0004FF4E13C02920846019340210023CDF840
:10F1B00000C0744A20F002F95DE600231B200521FF
:10F1C00084F8C02284F8F0204FF4E13984F8C83084
:10F1D00084F8F93084F8F83084F8EF0084F8FA10F5
:10F1E0001BE6AB7A002B73D042F0080201214FF4EA
:10F1F000E13E6346CDE90112CDF800E04021624ACC
:10F2000020F0DCF8EEE54FF0010E4FF4E13C029205
:10F2100008465C4A4021CDE900CE20F0CFF8E1E578
:10F22000BCF1000F6ED1AB7A002B5DD042F0080E1E
:10F2300003214FF4E1326346CDF808E0019140210B
:10F240000092524A20F0BAF8514B1860514B1860A6
:10F25000BCE5002B5ED042F0080201214FF4E13EF4
:10F2600003460292604601914021CDF800E03D4AFC
:10F2700020F0A4F8B6E5002B61D101220291CDF86F
:10F280000090604601924021434A20F097F8A9E59A
:10F2900003238DE5022103224FF4806084F8DCA172
:10F2A00084F80412072184F80C2245F2F052C4F8C5
:10F2B000F40184F8C012A4F8C22257E5374B384A4B
:10F2C0001A6010F039FB0222012389F80020D6E4ED
:10F2D0004FF0010C4FF4E132CDE901C10092402121
:10F2E000294A20F06BF87DE54FF0030C4FF4E13232
:10F2F000CDE901C100924021244A20F05FF8244B5F
:10F300001860A3E742F0080303214FF4E1320293AF
:10F31000002393E74FF0010E4FF4E1320291604673
:10F320004021CDE9002E0F4A20F048F85AE54FF071
:10F33000010C4FF4E132CDE901C1009240E542F009
:10F34000080201210346CDF8009002926046019127
:10F350004021114A20F032F844E500BF558B0008E7
:10F36000698B0008398D00084D94000861940008ED
:10F37000A0860100DC310120759600087D8A000816
:10F38000958A0008098B00087D9D000859930008A4
:10F3900000450120EC410120118900088C4A012020
:10F3A0005D9F000842F0080203214FF4E13E6046F1
:10F3B0000292002301914021CDF800E0074A1FF09E
:10F3C000FDFF58E503220291CDF8009060460192BE
:10F3D0004021034A1FF0F2FF4DE500BF398D0008C0
:10F3E00011890008C9B1013930B40546441E002016
:10F3F00055FA81F514F8011F020A4840A54280EA37
:10F400000010C0B24FEAC00342EA002183EA1010A4
:10F4100080EA0100EED130BC7047084670470023F7
:10F42000F7B5494C07468DF803306023474EC4F8C2
:10F4300088343378152B0ED0122B0CD0012B0CBF37
:10F4400002258C25FBF778FF002807DA013DF9D16A
:10F45000002003B0F0BD44F62065F3E70A25FBF772
:10F460006BFF0130F4D0013D15F0FF05F7D1D4F862
:10F470008424930803EB5203C4F88834FBF75CFF41
:10F48000431CE5D00028F9DC00230DF1030084F8CB
:10F490008C34FBF7A5FF0028DAD09DF803301B2B36
:10F4A000D6D10DF10300FBF79BFF0028D0D09DF8CB
:10F4B000032094F8093A9A42CAD10DF10500FBF7EE
:10F4C0008FFF9DF80530012BC2D801A8FBF788FFFC
:10F4D0009DF80430002BBBD00DF10300FBF780FF3B
:10F4E0000028B5D09DF803300E2BB1D10DF10300EB
:10F4F000FBF776FF0028ABD09DF8032033789A42C3
:10F50000A6D10DF10300FBF76BFF0028A0D09DF8FA
:10F510000330002B9CD13D46EA1BBDF8043092B26B
:10F52000023B9A4209DB0DF10300FBF759FF94F807
:10F530008C04B0FA80F040098BE72846FBF750FFB7
:10F54000002885D00135E7E720280120B8BB01203D
:10F5500070B5264C0646082594F80A3A434084F8CC
:10F560000A3A94F8F43304EB8303D3F8D403F30793
:10F5700015D512F05BFA402011F0C0FD94F8F43379
:10F5800004EB8303D3F8D40312F04AFA402011F0BD
:10F59000B5FD013D760815F0FF05E2D170BD12F012
:10F5A00045FA202011F0AAFD94F8F43304EB83030C
:10F5B000D3F8D40312F034FA202011F09FFD94F810
:10F5C000F43304EB8303D3F8D40312F02FFA202092
:10F5D00011F094FD94F8F43304EB8303D3F8D403CF
:10F5E00012F01EFA202011F089FDD2E72028012018
:10F5F00010B50D4C94F80A0AFFF7AAFF94F8F433FB
:10F6000004EB8303D3F8D40312F010FA202011F096
:10F6100075FD94F8F433202104EB8304D4F8D4036B
:10F62000BDE8104012F04EB92028012010B5104C52
:10F6300094F8F43304EB8303D3F8D40329F08AFF5E
:10F64000FF20FFF785FFFF20FFF782FF7F20FFF7F6
:10F650007FFF00231B2084F80A3AFFF779FF94F814
:10F66000090A0130C0B284F8090ABDE810406FE70A
:10F670002028012010B50B4B01241C70FFF7D6FF8A
:10F680000020FFF765FF2046FFF762FF0E20FFF71F
:10F690005FFF2046FFF75CFFFFF7AAFF0248BDE8C7
:10F6A0001040BCE6B8BB0120B9BB0120F8B5047816
:10F6B0000546002C3ED004F10A060027FFF7B6FFEE
:10F6C000300AFFF745FFF0B2FFF742FF0E20FFF7C9
:10F6D0003FFF1A4B1878FFF73BFF3846FFF738FF1C
:10F6E0002046FFF735FF0020FFF732FF0020FFF72D
:10F6F0002FFF0020FFF72CFF0020FFF729FF00203D
:10F70000FFF726FF0020FFF723FF0020FFF720FF71
:10F710006B68013C1878FFF71BFF6B6814F0FF045F
:10F7200003F101036B60F3D1FFF762FF0448BDE80A
:10F73000F84074E64FF485760127BFE7B8BB012097
:10F74000B9BB012038B505460478FFF76FFF0020EC
:10F75000FFF7FEFE0420FFF7FBFEB4FA84F40E2050
:10F76000FFF7F6FE094B64091878FFF7F1FE204613
:10F77000FFF7EEFE2878FFF7EBFEA020FFF7E8FE8C
:10F78000FFF736FF6868BDE8384048E6B8BB01209F
:10F7900038B5154B04460268934322D0134B062517
:10F7A0001D70FFF743FF0020FFF7D2FE0520FFF793
:10F7B000CFFE0E20FFF7CCFE2846FFF7C9FE002043
:10F7C000FFF7C6FE0020FFF7C3FE6078FFF7C0FE1C
:10F7D000A078FFF7BDFEFFF70BFF0548BDE83840F6
:10F7E0001DE6012038BD00BF00FFFF00B8BB0120AF
:10F7F000B9BB01202DE9F04FDFF8DC82D1B0B04C6D
:10F8000008F11409C4F8FC031FF066FF002584F812
:10F81000935484F89454FBF761FF2F28F7D101210A
:10F82000002012F011F90027ADF80850FBF756FF41
:10F8300010AD0190FBF752FF8DF81500FBF74EFF5E
:10F840008DF81600FBF74AFF0646FBF747FFE85521
:10F850000137FBB29E42F8D1FBF730FF8DF80D0067
:10F86000FBF72CFFB4F893348DF80C000121BDF8A0
:10F870000C7000209F4214BF0327002712F0E4F809
:10F88000002F40F08E80019B0695303B102B00F23C
:10F890004382DFE813F06E009900E3029D0011003F
:10F8A000B2004102DB00B401EA0112025A02410235
:10F8B00038028502A600B902012602ADB246002137
:10F8C000084684F8001484F8011412F0BDF8D4F846
:10F8D000FC0311F057FD2E20FAF774FB0198FAF79C
:10F8E00071FB9DF81500FAF76DFB9DF81600FAF70D
:10F8F00069FB50460AF1FF3AFAF764FB5FFA8AFAAD
:10F900000AF1010AAA44D4F8FC0311F06DFD0028A5
:10F91000F9D015F8010BFAF755FB5545F3D13846E8
:10F92000FAF750FB94F80114D4F8FC0311F064FDCD
:10F9300094F80014D4F8FC0311F05EFDD4F8FC0335
:10F9400011F01AFD0021084612F07EF8002E3FF457
:10F950005DAF94F80C3A002B40F08B82594B5A4A19
:10F960001B689B1A594A18BF0123137051B0BDE898
:10F97000F08F94F88F34A3B194F80B3A013B032B2A
:10F9800018D8DFE803F002021302FD2302210AA8BF
:10F99000ADF82830FBF7E4FD0120FBF787FDC12817
:10F9A00008D1002602AD4FF0010A88E7FFF762FE9A
:10F9B0000028F6D1002602AD4FF0010A0F2784F887
:10F9C0008F6484F890647AE76B238DF80830E8E759
:10F9D0004FF43273002602AD4FF0020AADF8083042
:10F9E0006DE72B785A1E032A00F23D8284F80B3A09
:10F9F000002602AD4FF0010A61E72B7894F80C2A3B
:10FA00009A4205D8002602AD4FF0010A082756E7B2
:10FA100084F8F43394F80B3A042B0ED8012202FA3E
:10FA200003F313F0160F08D0002302210AA884F86C
:10FA30008F24ADF82830FBF793FD002602AD4FF080
:10FA4000010A84F88F6484F8906438E72B7894F87E
:10FA50000C2A84F88F749A4284F89074D2D90326C1
:10FA600084F8F43394F80B3A042B37D0FFF702FEF6
:10FA7000A0B3012116482FF035FC78B302211548B8
:10FA80002FF030FC50B3B4F88F3449F2073223F032
:10FA90000801914207D049F20A32934203D049F259
:10FAA0000B4293421AD1032384F80B3A94F80B3A91
:10FAB0000026084D4FF0040A84F89234FFE600BF98
:10FAC00020280120BC2800206981020865B101209E
:10FAD000B02C0120AF2C012001990408B8F80020B7
:10FAE00098F80230ADF810208DF812300AABC24AF7
:10FAF0001068083252F8041C1D464A4503C52B46BF
:10FB0000F6D1D9F80000152199F8042028600AA838
:10FB10002A71FBF725FD082107A8FBF7D8FC002870
:10FB20005FD09DF810209DF81C309A4259D19DF865
:10FB300011209DF81D309A4253D19DF81E209DF84A
:10FB400012309A424DD19DF81F304FF2103284F896
:10FB500091349DF8203084F890349DF8213084F859
:10FB60008F34B4F88F3423F02001914211D04FF23A
:10FB7000104293420DD04FF29032934209D04FF68B
:10FB80005002934205D003F5BA520F3292B2012AC5
:10FB900003D8012384F80B3A88E723F0080249F2DE
:10FBA00007318A4207D049F20A32934203D049F220
:10FBB0000B42934203D1022384F80B3A76E741F6D5
:10FBC0000672934209D043F20632934205D023F4E1
:10FBD000807343F20642934203D1042384F80B3A24
:10FBE00064E7013E16F0FF067FF43CAF84F88F64B3
:10FBF0004FF0040A84F890640F27804D5FE694F874
:10FC00000B3A032B40F088807D4B12251D70FFF7C7
:10FC10000DFD0020FFF79CFC0720FFF799FC0E204C
:10FC2000FFF796FC2846FFF793FC1420FFF790FCA3
:10FC30000020FFF78DFCAC20FFF78AFC8820FFF73F
:10FC400087FC1320FFF784FC7620FFF781FCFFF789
:10FC5000CFFC6C48FFF7E3FB00287FF4A2AE002640
:10FC600002AD4FF0010A0F2729E694F80B2A012A6A
:10FC700001D0042A50D12B78042A05A88DF8083029
:10FC80000CBF9B005B00DBB28DF8153000238DF8B4
:10FC90001630FBF7DCFC0028E1D04FF48173022121
:10FCA0000AA8ADF82830FBF75BFC4FF42F70FBF788
:10FCB000FDFB30283FF475AED1E72B788DF814307A
:10FCC00094F80B3A5A1E032A26D8DFE802F0020203
:10FCD0000F02022B05A90CBF07200320FBF7D8FC5D
:10FCE0000028BCD09DF814A00026E8E505A8FFF781
:10FCF0004FFD0028B3D01422414B0DEB02001A70C7
:10FD0000FFF720FDECE72B788DF8143094F80B3AD0
:10FD1000022B07D0032B0AD0002602AD4FF0010AB8
:10FD20000227CCE505A90420FBF7B2FCD8E705A81B
:10FD3000FFF72EFD002892D0314B162205A81A702D
:10FD4000FFF700FD0028CDD189E794F80B3A8DF834
:10FD50001460013B032B3FF624AEDFE803F0020200
:10FD6000110205A8FBF773FC00283FF478AFFA22D4
:10FD700005A90120FBF752FC00287FF412AE6EE7C4
:10FD800005A8FFF705FD00283FF469AF1C4B1322BF
:10FD900005A81A70FFF78AFC00287FF402AE5EE720
:10FDA00094F80B3A8DF81460022B05D0032B13D076
:10FDB000012B7FF454AFAFE705A8FBF748FC002800
:10FDC0003FF44DAF40F2DC5205A90520FBF726FCBD
:10FDD00000287FF4E6AD42E705A8FFF7D9FC00282C
:10FDE0003FF43DAF064B152205A81A70FFF75EFCE5
:10FDF00000287FF4D6AD32E705990408AF2C012026
:10FE0000B8BB0120B9BB012094F80BBABBF1040FB9
:10FE100082D105A88DF81460FBF719FC00283FF487
:10FE20001EAF05A8FBF7D2FB00283FF418AF4FF434
:10FE3000827302210AA8ADF82830FBF791FB142049
:10FE4000FBF734FB30283FF4ACADC0287FF407AF9C
:10FE5000002602AD4FF0010A5F4630E500260F4D47
:10FE60004FF0090A2BE5002602AD4FF0010A0927E1
:10FE700025E5013B0221DBB284F80C3A04EB830355
:10FE8000D3F8D40311F01EFD94F80C3A04EB83036D
:10FE9000D3F8D40311F0C4FD5BE500BF4BE50408C3
:10FEA00038B5054630F090FE044628B906220849C8
:10FEB000284614F007FA50B9064831F0E9FE17F069
:10FEC0009DFD24F05DFD14B10020FCF7E9FE38BD76
:10FED00063E7040855E504082DE9F0470546214F7E
:10FEE000DFF8A080DFF88090DFF89CA0284636F08D
:10FEF000D7FA064660B91C4B1C4893F888281C4B5F
:10FF000003EB8203BDE8F047D3F8A81631F0BEB882
:10FF100002463946284614F0D5F978B9154C164DE5
:10FF2000164830F097FF54F8041F19B1284630F0F6
:10FF30007CFFF8E7BDE8F04731F025B8002458F819
:10FF4000241021B90E48BDE8F04731F07DB83246A3
:10FF5000284614F0B7F901340028F0D189F8884810
:10FF60005546C3E76FDF0408202801206BE504082D
:10FF700070920408189904089EE5040875E50408C1
:10FF8000ABE104081C990408222F05082DE9F3476A
:10FF9000054630F019FE044610B131F073F822E046
:10FFA000284601AA2749264637F095FC27460546EC
:10FFB000DFF89C80DFF89C90DFF89CA03DB9224BD5
:10FFC0003246A1B2D3F89C0407F08FF90BE06FB171
:10FFD000012FE2D1B31E284659425941FBF778FE62
:10FFE000421C044622D102B0BDE8F087284636F014
:10FFF00057FA414606460246284614F063F9A0B176
:020000040801F1
:1000000032464946284614F05DF9B8B132465146A9
:10001000284614F057F998B132460C49284614F096
:1000200051F90028B9D1032600E03E4601AA05494E
:100030000020013737F04FFC0546BFE70126F5E702
:100040000226F3E78B1405082028012089E504081F
:1000500080E5040883E5040886E504082DE9F84FE7
:1000600080460E46174636F01BFA0446F0B90C25BA
:10007000404FDFF82481404830F0D7FE20461FF083
:1000800019FB3368184205D005FB04734046996894
:1000900030F0CBFE0134172CF0D1336813B9374858
:1000A00030F0D8FEBDE8F84F30F06DBF024634495D
:1000B000404614F007F90546B0B92C462D4E0C25E4
:1000C000DFF8C8802F4830F0C5FE20461FF0F2FA56
:1000D000384205D005FB04634046996830F0A5FE20
:1000E0000134182CF1D1DDE798F800302D2B29D1FF
:1000F00008F10108013C01254FF0000A47F4000B0C
:100100000C221C4B404602FB0A32D2F808902246D1
:10011000494614F0D7F810BB50461FF0CBFA1BEA43
:10012000000F1CD085B1BAF1170F01D03768074313
:100130003760154830F08EFE49461448BDE8F84F48
:1001400030F0A4BF0025D7E7BAF1170F02D0356809
:1001500025EA000535600E4830F07CFEECE70AF138
:10016000010ABAF1180FCBD10A48BDE8F84F30F0B8
:100170006BBF00BFD0D104088CE5040896E50408E5
:100180006FDF040875E50408A2E504089EE504088D
:10019000ABE50408ABE104089DE50408014A024907
:1001A0005CE700BFFFFF7F001CBB012040F2022282
:1001B000004953E724BB01202DE9F84F384F05468D
:1001C00036F06EF90446D7F80090B0B9354D0126E7
:1001D000354F364830F03EFE55F8241049B106FA46
:1001E00004F313EA090F02D0384630F01EFE013442
:1001F000F2E7BDE8F84F30F0C6BE02462C4928466B
:1002000014F060F878B92B4C2B4D2C4830F022FEBE
:1002100054F8041F0029ECD00B78002BF8D02846A6
:1002200030F003FEF4E72B782D2B10D10135013C83
:100230004FF0010A0026DFF86CB05BF82680B8F1B9
:10024000000F07D11E48BDE8F84F30F0FDBE4FF05B
:10025000000AEFE722464146284614F033F8E8B991
:100260000120B040830504D51648BDE8F84F31F0B1
:100270008DBBBAF1000F0AD012F018F8124830F016
:10028000E9FD41460C48BDE8F84F30F0FFBE40EABA
:10029000090038600D4830F0DDFDF2E70136CCE7AB
:1002A0008041012088990408BDE50408B3E50408ED
:1002B0006FDF0408849904089EE5040875E50408C6
:1002C000ABE10408C1E50408A2E50408ABE50408B5
:1002D0002DE9F0478AB0054636F0E2F8024630B91B
:1002E0008E490120FBF7C6FA0AB0BDE8F087052267
:1002F0008B49284613F0E6FF0446B8B9894D0146FC
:10030000702205F60D2038F06DFEC5F8B844C5F82A
:10031000C444C5F8D044C5F8DC44C5F8E844C5F881
:10032000F444C5F80045C5F80C45DDE704227E49D4
:10033000284613F0C7FF044620BB284630F04CFC8B
:1003400007460028D0D036F0ABF8DFF80482064626
:1003500058F824501DB9754830F076FEC4E732468F
:100360002946384613F0AEFF50B9204631F0E4FC80
:1003700029466F4830F08AFE6E48FFF7A9FFB3E7C1
:100380000134E5E707226C49284613F09BFF044639
:10039000002873D12846202138F0F3FE054678BBAB
:1003A0002C46664D664830F040FD21460134284613
:1003B00030F03BFD0E2CF8D1624E0024DFF8949112
:1003C00030F0E1FD604FDFF890810025DFF88CA16F
:1003D0002146484630F029FD012332685046AB40A3
:1003E0000135134214BF3946414630F01EFD0E2D33
:1003F000F2D1013430F0C7FD0C36082CE5D173E79B
:1004000002AD524E01AA514937F065FA002840D09A
:10041000022C18D1029B072B3BD803990D2938D801
:100420000278722A1AD06E2A33D13E4A0C2000FB81
:100430000323012202FA01F1D3F8B82422EA0102CF
:10044000C3F8B82416E014F023F801AA45F82400F4
:1004500031460020013437F03EFAD7E70C20314A0C
:1004600000FB0323012000FA01F1D3F8B80408438C
:10047000C3F8B8043048FFF72BFF35E728460024BF
:1004800002AD324E01AA314937F025FA78B1082C75
:1004900002D130F0F7FD27E713F0FAFF01AA45F883
:1004A000240031460020013437F015FAEEE7082C1D
:1004B000EFD1029B0F2BECD8DDF80CC0BCF1070F7D
:1004C000E7D8049F0D2FE4D8059E06F16402C82AE0
:1004D000DFD8069DFF2DDCD807986428D9D8089965
:1004E0006429D6D88842D4DA099C032CD1D8C3EB2E
:1004F000C3020C4B134483F8110A83F80DCA83F826
:100500000E7A83F80F6A83F8105A83F8121A83F868
:10051000134A0848FFF7DCFEE6E600BF2D32012053
:10052000CDE5040820280120D3E50408ABE1040848
:10053000D8E50408222F0508E2E50408EAE50408E6
:1005400041DC0408D82C0120FADC04088B140508CF
:100550001C9904081C2E0508DAE70408EFE50408D6
:100560002DE9F04F87B0044635F09AFF064628B9CA
:100570004120FBF7D3FB07B0BDE8F08F02468B4963
:10058000204613F09FFE002836D11424884D894858
:1005900031F0FCF92D21D5F8980411F0BDFD013C96
:1005A000F8D1854C30F0EFFC844E04F5C475844FCF
:1005B000DFF8408221683846A28801F13F41A379E3
:1005C000B2FA82F201F57E0106EB8303C2F11F024B
:1005D000890AD3F84C31413130F027FCE17911B16F
:1005E000404630F022FC083430F0CDFCA542E1D189
:1005F000744831F0CBF9BEE7DFF8C081204605AA88
:10060000714908F50A7737F066F900248246B94641
:1006100017F8343032465046E50008EB8303D3F830
:100620004C1113F04FFE30B101341A2CF0D1674851
:1006300030F00AFD9FE705AA6349A84437F04BF95B
:10064000074613F025FF98F82E220646002A40F0B0
:100650009980002800F39F80A944B9F8020017F0A0
:10066000EBF93D78002D00F08A80F3B299F8046030
:10067000D0F8048038460193019A99F8053054491E
:1006800002FB063613F05AFE60B908F8060018F8A7
:100690000680B8F1000F16D14E4831F077F96AE7BD
:1006A000012273E0602D8CBF613D413D072D66D86E
:1006B000781C13F0EDFE0F2861D8013540EA0515CE
:1006C00008F80650E3E7404610F076FF8146002820
:1006D00055D04FEA1813404F00264033029308F0DC
:1006E0000F03039300252EE0788817F0A5F97A7997
:1006F0003B7905FB03234268D15C414522D1B442DA
:1007000004D101998D421DD00021D1545FFA85FB9F
:1007100032485FFA86FADDE9021230F086FB59466C
:100720005046FAF7F5FFB44209D12D4830F07DFB71
:1007300050465946FAF7ECFF2A4830F076FB2A4833
:1007400031F024F90135BB79002B08BF01239D420C
:10075000CADB013608371A2EC4D1D9F80010B9F80F
:10076000042001F13F412148B2FA82F201F57E01F5
:10077000C2F11F02890A413130F088FCFBE630F0FB
:1007800081FCF8E6002801DD964206DD01211848CB
:1007900030F070FCEFE6012882D105AA0A4900205A
:1007A000013E37F098F8074656E700BF6FDF0408B0
:1007B00020280120F5E50408889C01207092040897
:1007C00033E604083EE604088B14050870E60408C6
:1007D0003CDE040878E60408989404088AE60408D5
:1007E000DDE40408AEE6040826130508B8E60408AC
:1007F000C0E404081B2E05082DE9F74F814635F0AB
:100800004FFE054628B1012822D199F800302A2B45
:100810001ED10024DFF8E4814FF00D09714F7248BA
:1008200031F0B4F809FB048638460134316830F001
:10083000FCFA291C304618BF012130F099FB30F03A
:10084000A2FB40F269139C42ECD103B0BDE8F08FEB
:100850003D21484638F095FC002800F0BC80074652
:1008600017F8013C7A1E202B32D0A7EB0907013084
:10087000054601302B78202BFAD0DFF880A14FF00D
:100880000008FFB2D3460D2303FB08A426683046B8
:1008900035F006FE314602460190484613F012FD3F
:1008A0000646002840F08A80019BBB4240F08680CB
:1008B000237903F06003202B3ED00BD8F3B14B48D3
:1008C00030F0C2FB204603B0BDE8F04F30F0EDBB86
:1008D0001746C5E7402B45D0602BF0D1444A00278E
:1008E00002EBC606B9463B4696F898A7574502D292
:1008F000B9F1000F22D0002BE1D00EE0284613F012
:10090000C7FDB4F9053001B28B42D8DCB4F9073029
:100910008B42D4DB204630F0EFF90D23354803FB42
:1009200008B8D8F8001030F080FA0021204603B053
:10093000BDE8F04F30F01CBB6679CFE7D6F89427BE
:1009400052F8270060B12946019313F0F7FC019B90
:1009500030B94FF0010939B2204630F0CDF94B469D
:100960000137C3E74FF00D0994F805A009FB08B95A
:100970005645D2DA002DD0D02F4601353B78202BBA
:10098000FAD0204630F0A2F999F80430054603F079
:100990000703022B0CD0032B0AD0384613F078FD46
:1009A000A8552C21384638F0ECFB0136451CDFE712
:1009B000384613F06DFD25F81600F2E708F101083E
:1009C00040F2691398457FF45EAF0B4803B0BDE871
:1009D000F04F30F039BB484603B0BDE8F04FFBF7AD
:1009E000AFBD00BFD02D0508D4E60408F2E6040828
:1009F00070920408E7E60408ABE10408FC9D0408D3
:100A0000F7B5044630F0E0F8064638B10022324926
:100A1000012003B0BDE8F04030F0C4BB2F492046B0
:100A200013F08CFCB0B92E4B4FF47A714FF4FA628C
:100A3000A3F87E1AA3F8802AA3F8821AA3F8842ABE
:100A4000A3F8861AA3F8882AA3F88A1AA3F88C2A8E
:100A500003B0F0BD204613F01BFD0328054633D834
:100A6000204630F0B9F8074660B113F011FD0126B9
:100A70000446384630F0B0F840B903B0BDE8F04065
:100A800030F000BB40F2EE240646F2E713F000FD22
:100A9000002EF2D0A4F2EE2240F2DC539A42ECD8BF
:100AA000A0F2EE229A42E8D80D4B00210D4A03EB4A
:100AB0008503A3F87E4AA3F8800A2B46CDE90040BF
:100AC000084630F05BFBC3E703223146064803B01B
:100AD000BDE8F04030F0CEBA9E320120CDE50408EA
:100AE0002028012000E7040811E7040870B5044637
:100AF0000E46084635F0D4FC3146054602462046EF
:100B000013F0E0FB68B9665D304613F027FC00B9CE
:100B100036B901352C44204601340378202BFAD015
:100B200070BD0020FCE72DE9F04F0F468DB0C449A1
:100B30000646FFF7DBFF0546002840F07182C149F9
:100B40003046FFF7D3FF0546002840F06B82BE49D0
:100B50003046FFF7CBFF0546002840F06582BB49D1
:100B60003046FFF7C3FF002805460ABF01240824CA
:100B700035460FB144F0100431F0ACF816F03EFFEA
:100B800023F0FEFEB2492846FFF7B0FF08B144F05B
:100B9000200414F0090F00F03082AE4831F078F8EC
:100BA0000020FBF71BF830F0EEF9AB48FCF7C2F978
:100BB000A948FCF787F914F00803039305D0002037
:100BC000FBF732F8A448FCF701F904F01803182BDE
:100BD00007D1A24831F05CF8A14830F03BF930F081
:100BE000D2F9A04831F054F89F4B20469F4D1A7817
:100BF0009F4E002A9F4ADFF828B306BF1346012103
:100C000000219D4A30F0BAFA9C4831F041F8204664
:100C1000FBF784F89A4831F03BF895F8883895F856
:100C20008E7A984AF81A06EB83034742D3F8A8361F
:100C300047412046394630F089FA95F88E3A3946D0
:100C4000914F06EB83038F4A204606F5E366D3F8FF
:100C5000A83630F093FAD7ED007A8C4A2046F5EEAC
:100C6000407AF1EE10FA0CBF0121002130F086FA33
:100C70003A468749204630F0CBFA864831F008F8EA
:100C800005F5976205F694212046FAF761FE824841
:100C900030F0FEFF95F90F1A804A2046B1FA81F133
:100CA0000027490930F06AFA05F60D2205F6F4210D
:100CB0002046FAF7DFFD7A4830F0EAFF794BD3F8A7
:100CC0000080794BD3F8009056F82750002D40F063
:100CD000AD812E4669EA080BDFF848A2734B53F842
:100CE0002650002D40F0C281714830F0D1FF714B89
:100CF000714F2046714E00933A6831686C4BFCF797
:100D00000DF86F4830F0C4FF40F2022320460093F4
:100D1000BA68B16801266A4BFCF700F8694830F000
:100D2000B7FF694F6948DFF800C22B5C0CA9EA5D88
:100D30000DF1300E194401F8202C15F80C108E44DA
:100D40000EF8102C16B1591A4E424E410135082D9D
:100D5000EBD10025314608AB5D4A20468DF818508E
:100D60008DF8285030F0F2F904AB3146584A20464D
:100D700030F004FA574830F08BFF574A5749204665
:100D800030F0F0FB564830F083FF564A5649204673
:100D9000FCF7B2FA554830F07BFF554A55492046DA
:100DA000FAF7E4FE544830F073FF4E4A4E492046AD
:100DB000FAF75EFE514830F06BFF514A204601269B
:100DC00002F51171DFF864A130F0C8FC4D4830F035
:100DD0005FFF4D4A2046DFF898B002F1960130F0EF
:100DE000A3FA4A4830F054FF494A204602F28A21C9
:100DF00030F0D8F9474830F04BFF474A204602F21E
:100E00009C61FAF7E7FC454830F042FFDFF82081AB
:100E1000022208F1230308F1FF309919304438F019
:100E2000B9F81AF81530B0FA80F75B447F0993F8E7
:100E3000D42818F81530022B40F039817AE000BF31
:100E400019E7040893E1040820E7040826E70408EA
:100E500062E504082AE70408222F050832E704089F
:100E60005AE70408B3E10408C848012020280120FB
:100E700070920408B6140508B8E404086AE7040888
:100E800074E704087AE7040838BB012083E7040804
:100E90000CBD012092E7040898E70408A2E70408C3
:100EA000AFE704086C4701208041012088990408BD
:100EB000CEE70408FFFF7F001CBB01208CBD012092
:100EC000D5E70408DCE70408EC9804085CBE0120C0
:100ED000E0E70408E7E7040864BA0120ECBD01205C
:100EE000AFE5040858360120D0470120F3E7040895
:100EF000D836012050480120EEE70408F9E704083D
:100F000040310120FDE70408FC33012006E8040815
:100F10009E3201200EE804089C2E012012E80408ED
:100F2000B7E70408C3E7040868B101208F35012042
:100F30006B35012016F80A304FF0190940F2EE2106
:100F4000204619FB03133946CDE900232B46664A98
:100F500030F0FCF816F8083040F2EE21624A2046E4
:100F600019FB03133946019318F815305B4493F8C5
:100F7000D43800932B4630F001F901350236122D9A
:100F80007FF444AF594830F083FE21460020584E8C
:100F90002FF0FEFF039B2146002B00F09C800020D9
:100FA000544DFBF757FB214601200027FBF752FB6E
:100FB00021460220FBF74EFB4F4830F069FE3378A4
:100FC0004E48AB72FBF78CFAFF23AB72F8B20137D5
:100FD0002146FBF769FA062FF8D1494830F058FE50
:100FE000737846486B72FBF72FFAFF2345486B7204
:100FF00030F04EFE44482FF02DFFA20704D53C4BA5
:1010000021461878FBF726FB630704D5384B2146A9
:101010005878FBF749FA30F047FE0DB0BDE8F08F85
:101020000124A6E50224A4E50424A2E52B78DBB183
:101030004FF0010A69EA08035A4620460AFA07FAFD
:1010400013EA0A0F2B4614BF0121002130F07EF86D
:1010500068EA09035A46204613EA0A0F2B4614BFD2
:101060000121002130F08AF801372DE62B78E3B119
:101070000127B74019EA070F0AD068EA0903524668
:1010800020463B422B4614BF0121002130F05EF880
:1010900018EA070F09D01BEA070F2B4652462046D5
:1010A00014BF0121002130F069F8013616E60092E4
:1010B0002B463946154A204630F048F818F81530C6
:1010C000124A39465B44204693F8D43800932B46A5
:1010D00030F054F851E73078FBF7BCFA21467078CD
:1010E000FBF7E2F989E700BF19E8040819E70408EB
:1010F000ECBE01200000012036E80408222F05087C
:1011000059E8040880E8040865E7040829E80408A9
:10111000012108E5002106E52DE9FF41074635F0EC
:10112000BFF908283CD1002401AE385D13F00AF95C
:1011300030550134082CF8D10024DFF870808DF888
:101140000C40385D13F0FEF83055C5B240462946D4
:1011500038F017F828B101342946301938F011F861
:1011600020B12FF08FFF04B0BDE8F081082CE8D14A
:101170000D493046FDF770FB00230B4C0B481A5D00
:1011800004A90A44195C013302F80C1C082BF6D19F
:10119000002301A906488DF80C302FF077FFE2E715
:1011A0000028E9D0DDE700BF68B10120EC98040811
:1011B000E0E70408000000004FF416734FF480715C
:1011C000152203810023818082710380438030B423
:1011D00040F2D93540F2C5344581848130BC704736
:1011E000034B93F85B30002B0CBF46204320704725
:1011F000E0350120054B93F85B302BB94FF4A47315
:101200005843642390FBF3F0704700BFE0350120A2
:101210000E4B1B78022B17D00D4A5378127803EB34
:10122000830302EB82025B00C01AC3EB4203C0EBF4
:10123000C00090FBF3F00628A8BF062020EAE0706B
:10124000C0F19600C0B270479720704728BB0120BC
:1012500004530120034B93F85B30002B0CBF0F208D
:101260000C207047E035012070B41C4CB4F870308D
:10127000E8B903F00103C3B994F87450ADB1184A4A
:1012800002F1F40602E00133AB420ED052F8041B27
:101290004904F8D594F8601104EB8101D1F8F80005
:1012A00046F823000133AB42F0D170BC70475A08B6
:1012B000012A08D90D6802F001030A48A4F8702039
:1012C00028440860D7E70A6848F20500054BA4F8EF
:1012D0007000134470BC0B60704700BFE035012004
:1012E00058360120A08601002DE9F04300283BD1AB
:1012F0002D4A92F8740068B32C4A00242C4B1678BF
:1013000092F901E003EB8000C6F1FF0CA6F17F0724
:1013100092F9028003F1F4025FFA8CFCFFB203E061
:10132000834202F1040215D053F8041B8904F7D557
:10133000E1B20825A1EB0E0181EAE179A9EBE1799F
:10134000B9F1010F08DD8342D57004F1010402F107
:101350000402E9D1BDE8F08335460029F3D04145C8
:1013600014BF65463D46EEE7104B1A78F02A09D8BF
:1013700002F10F000C4A1870086844F21A13034473
:101380000B60B6E7084A7F2093F9014092F8765047
:101390001870AC42987801DA002C02DA4042C0B2F0
:1013A000987020445870E7E7E035012014000120D0
:1013B000583601202DE9F0412D4EE0B196F8EC3180
:1013C000002B51D196F87720013AD2B2D6F8F031FD
:1013D000284C03EB4303284886F8EC21C3EB0313A6
:1013E0000A6884FB0354DB17C3EB6413053390FBDB
:1013F000F3F31A440A6096F874409CB31F48002324
:101400001F4F00F1F40C1D4602E00133A34229D026
:1014100050F8041BC1F30322062AF6D197F800E026
:10142000EA431EF0010F02F001020DD096F8EC2104
:1014300096F8778002EB050E9EFBF8F208FB12E2AD
:10144000012ACCBF002201220135002ADDD0C1F3E0
:10145000834106EB8101D1F8F8204CF823200133B9
:10146000A342D5D1BDE8F081013BDAB2AEE700BFBF
:10147000E03501201F85EB5140420F005836012016
:10148000C0520120F0B54D4C94F8F42100285BD1F6
:10149000002A58D04A4BB3EE097AD3ED007AF4EE25
:1014A000C77AF1EE10FA78DCBBEE097AF4EEC77A6F
:1014B000F1EE10FA4CBF08270027B3EE097AD3EDFE
:1014C000017AF4EEC77AF1EE10FA68DD47F0010711
:1014D00094F87450BDB33B480022DFF8F8E000F107
:1014E000F40C14E094F9F761B142ACBF0221002181
:1014F00094F9F861B3421BDA94F9F961B342D8BFA9
:1015000041F008010F4217D1013295421BD050F82B
:10151000043BD903F8D503F00F0194F9F661C3F346
:101520000313B142DEDC94F9F8610121B342E3DB3D
:1015300041F004010F42E7D0DEF80C304CF82230C5
:1015400001329542E3D1F0BD94F8F5010D6880B306
:101550001B4B82F001021C4ED3ED007A93ED017A11
:10156000F0EEE77A1948B0EEC77A84F8F421C7FEA6
:10157000877AFDEEE77A17EE903A193B03EB4303C7
:10158000C3EB031386FB0376DB17C3EBE6130533CC
:1015900090FBF3F32B440B607AE704278DE7BBEE57
:1015A000097AF4EEC77AF1EE10FA48BF47F0020765
:1015B0008EE7074B2B440B606AE700BFE035012044
:1015C000F452012058360120353AFC4440420F00C5
:1015D000400D030060B0040870B40D4E96F87440DE
:1015E000A4B106F17802054606F5B676002302E0BE
:1015F0000133A3420AD052F8040B35EA0000F7D1B8
:10160000086846F823000133A342F4D170BC704748
:10161000E035012030B4294B60B9294A927CBAB92F
:1016200093F861312749203301EB83014FF4A06027
:1016300030BCD1E793F8FA01E0B10138204A83F8D1
:10164000FA010C68204820440860927C002AE7D008
:101650001E4A12689106E3D51D4A93F8FA111278D2
:1016600092071AD511BB93F863311649203301EB69
:101670008301DBE7124A93F8FB41957CA54205D82C
:10168000042483F8FB0183F8FA41DAE701340120EE
:1016900083F8FB4183F8FA01D3E70029C0D193F81E
:1016A00062310849203301EB8301BFE793F85F31D2
:1016B0000449203301EB8301B8E700BFE035012086
:1016C000E45E012058360120801A060020530120D4
:1016D000E15E012010B4A8B91B481C4C90F8FC2115
:1016E0000B6823440B6012B15DF8044B704790F80F
:1016F0005F314FF44070164920335DF8044B01EB25
:10170000830169E7134B1B789BB1012B08D10E486D
:10171000114C90F8FC2182F0010280F8FC21DFE7F7
:1017200009480E4C90F8FC2182F0010280F8FC215F
:10173000D6E70C680120054B034A23445DF8044BAF
:1017400082F8FC010B607047E035012040420F0039
:101750005836012028BB012020A1070048E80100DD
:1017600010B4354A08BB92F8FD31C3B192F8FE11AE
:101770008A081341DB0715D5012A01F0010153D076
:1017800041D3022A0ED12D4BA3F11802002914BF18
:10179000194611464FF400305DF8044B1CE792F8EF
:1017A000FF3153BB5DF8044B704792F8FE310133B3
:1017B00003F00F0382F8FE3133B192F8FD310C686B
:1017C0001F4820440860D0E71E4882F8FD31407968
:1017D00008BB1D48C07818B143F0040382F8FD31FE
:1017E0001A480078C007EAD4194800680028E6D0F3
:1017F00043F0010382F8FD31E1E716494FF4003070
:101800005DF8044BE8E6144B03F11802002914BFFD
:1018100019461146BEE7114800780028D9D00220A9
:10182000034682F8FD01D4E70B4B03F108020029BF
:1018300014BF19461146ADE7E035012088B0040811
:10184000A086010004530120C4520120C05201208F
:1018500018BB01206CB0040860B0040828BB01204C
:1018600090F8603043B942690121072082F8443082
:10187000A2F8460082F84810704700BF4FF0FF30D2
:10188000704700BF4FF0FF30704700BF034B93F825
:101890002923027293F82A3343727047E0350120FE
:1018A00000207047002070470120704701207047DA
:1018B0000020704700207047027A407A02FB00F057
:1018C000704700BF027A407A02FB00F0704700BF09
:1018D00000207047012383731846704701238373E8
:1018E000184670474FF0FF30704700BF704700BF89
:1018F000002070470120704700207047027A407A2C
:1019000002FB00F0704700BF0020704700207047C6
:101910000020704730B41E25044C002005FB021146
:101920000C4484F82C3330BC704700BFE0350120F4
:10193000014B9888704700BF14000120094B0A49E9
:10194000D3F8382530B4D3F83455002422F02802D7
:1019500029402046C3F83C45C3F83415C3F8382560
:1019600030BC7047E03501209C2F9FEF00230222FE
:101970000370027143708370C3707047037913F072
:10198000020308D00369D0E90920013B101A18406E
:10199000C0B2181A704718467047017170477047F7
:1019A00003799B070AD5436A8269D154436A016966
:1019B0000133B3FBF1F201FB123343627047037949
:1019C00013F0010306D0D0E90732C0689B1A013832
:1019D000184070471846704710B50379014613F058
:1019E00001030ED0FFF7EBFF50B10B6A4A69CC68D8
:1019F000D05C0133B3FBF4F2C0B204FB12330B62D0
:101A000010BD1846FCE790F8533830B53BB990F854
:101A10005118012490F85238DAB2914200D830BD02
:101A200004FA03F2B0F85A5801332A43A0F85A28AE
:101A3000F2E7D0E90920131A584258417047034B86
:101A40009A790AB901229A71002070471400012086
:101A5000074BDA7952B11B7A43B103EBC203054A53
:101A6000093B32F81320044BA3F84025704700BF10
:101A70001400012038B60408E035012008B5174BE2
:101A80001B780BB1164AD371164B1B780BB1144A55
:101A90001372FFF7DDFF144B144A1B78013382F8F1
:101AA0004235134B1B887BB1192B0FD9642B0FD9EF
:101AB000C82B0FD9B3F5C87F0ED9B3F5167F03D85D
:101AC00004230133064A9371002008BD0023F8E780
:101AD0000123F6E70223F4E70323F2E79949012003
:101AE000140001209A49012094490120E035012089
:101AF0009649012008B5054B1A7A1AB901221A72C3
:101B0000002008BDFFF7A4FFFAE700BF1400012082
:101B100008B5054BDA791AB90122DA71002008BD3F
:101B2000FFF796FFFAE700BF14000120064B1A7872
:101B3000064B1B7803EBC203054A093B32F813201E
:101B4000044B1A80704700BFCA5C0120CB5C0120A7
:101B500038B60408CC5C01200A4B93F843250A4BA5
:101B60005AB10A4A127822B903F118025A610020C8
:101B7000704703F1E0025A61F9E703F5C0725A6158
:101B8000F5E700BFE035012014000120D25C012000
:101B9000034B4FF0FF30B3F84425024B1A807047D7
:101BA000E0350120D05C0120034B00201A88034B54
:101BB000A3F84425704700BFD05C0120E035012028
:101BC000074B93F90030012B06D0064B0020B3F8E9
:101BD0004825A3F8462570474FF0FF30704700BFF7
:101BE0009C1E0120E035012008B5064B1A782AB169
:101BF000054A1278012A01D000221A70FFF7ACFFC3
:101C0000002008BDD25C0120C85C0120064B93F97E
:101C10000020064B12B91A70002070471A78002A6B
:101C2000FAD10122F7E700BF9C1E0120CE5C012003
:101C3000104B0020104A93F84A15517193F84B1538
:101C4000917193F84C15117093F8502583F84D2538
:101C5000B3F85625A3F85225B3F85825A3F8542510
:101C6000B3F85E25A3F85A25B3F86025A3F85C25E0
:101C7000704700BFE035012004530120104A0020C6
:101C8000104B517983F84A159179127883F84B15E6
:101C900083F84C2593F84D2583F85025B3F8522549
:101CA000A3F85625B3F85425A3F85825B3F85A25B8
:101CB000A3F85E25B3F85C25A3F86025704700BF44
:101CC00004530120E0350120074B002093F86725DD
:101CD00083F8642593F8682583F8652593F86925CA
:101CE00083F86625704700BFE0350120074B0020D0
:101CF00093F8642583F8672593F8652583F86825AC
:101D000093F8662583F86925704700BFE035012008
:101D1000104B002093F86A2593F86C1502F00F021F
:101D200042EA012293F86E150901C9B20A4393F8F9
:101D30006D15A3F85C2093F86B2502F00F0242EAC0
:101D4000012293F86F150901C9B20A43A3F85E2076
:101D5000704700BFE03501200E4B0020B3F85C2037
:101D600002F00F0183F86A15C2F30311120A83F817
:101D70006E1583F86C25B3F85E2002F00F0183F82E
:101D80006B15C2F30311120A83F86F1583F86D25E2
:101D9000704700BFE0350120074B002093F8702505
:101DA00083F85A20B3F87225A3F85620B3F87425A7
:101DB000A3F85820704700BFE0350120074B0020F2
:101DC00093F85A2083F87025B3F85620A3F87225AB
:101DD000B3F85820A3F87425704700BFE035012000
:101DE0000448562208B500F2765135F03FFD002038
:101DF00008BD00BFE03501200449562208B501F2B4
:101E0000765035F033FD002008BD00BFE0350120DD
:101E1000084A00200849B2F8CC350B8292F8CE353A
:101E200092F8CF2503EB83035B00CB81034B9A70C1
:101E3000704700BFE03501204CB10120FCAE01200D
:101E4000084A0020084B118AD289A3F8CC150A2130
:101E5000B2FBF1F283F8CE25044A927883F8CF25BD
:101E6000704700BF4CB10120E0350120FCAE0120DD
:101E700030B1007910F1FF3018BF4FF0FF307047DC
:101E80004FF0FF307047074B93F8D02542B9064A10
:101E9000528802F0010283F8D125012283F8D0256F
:101EA00000207047E03501200CB00120034B0020DA
:101EB00083F8D20583F8D305704700BFE0350120D1
:101EC0000A4A00200A4BB2F8D4151B685980B2F8B0
:101ED000D615A3F84C10B2F8D8159980B2F8DA15D7
:101EE000B2F8DC25D9801A80704700BFE0350120A8
:101EF000FC5E01200D4B6021002093F8DE2501FBE4
:101F00000232B2F8E215A3F8D415B2F82C16A3F8F1
:101F1000D615B2F8E415A3F8D815B2F8E615B2F85C
:101F2000E025A3F8DA15A3F8DC257047E035012099
:101F30000A4A00200A4BB2F800171981B2F80217BA
:101F40005981B2F804179981B2F80617D981B2F80D
:101F50000817B2F80A2719825A827047E035012023
:101F6000D89801200A4A00200A4B1189A3F80017CB
:101F70005189A3F802179189A3F80417D189A3F80E
:101F80000617118A528AA3F80817A3F80A27704780
:101F9000D8980120E0350120144B0020144993F813
:101FA0000C27303281F8E521602193F8DE2501FB12
:101FB000023292F8271683F80D1792F8FA1583F873
:101FC0000E1792F8FB1583F80F1792F8FC1583F89B
:101FD0001017B2F81416A3F81217B2F8121692F8E6
:101FE0002F26A3F8141783F816277047E035012031
:101FF00014000120104B114993F80C27303281F85E
:10200000E82193F81727303281F8EA21122193F85A
:10201000962701FB023203F5E36302F22A7102F212
:102020003A7251F8040B914243F8040BF9D10A8833
:1020300000201A80704700BFE03501201400012005
:102040000A4A122192F8963701FB032302F5E36155
:1020500002F5E56203F22A7351F8040B914243F84A
:10206000040BF9D10A8800201A807047E03501205E
:10207000134A0020134910B592F80C37303381F819
:10208000E53102F5BC6392F8DE1501EB410103EB8B
:10209000411302F2977102F5F4621C7A03310633A0
:1020A00001F8034CDC7801F8024C1C7901F8014C72
:1020B000DC8822F8104001300328EED1002010BD4A
:1020C000E03501201400012007490020074B0A7861
:1020D00083F8DE25013283F80C274A7883F89627A7
:1020E000013283F817277047FCAE0120E03501204C
:1020F0000A49002230B501F2A670094C135DA3F124
:102100006105052D01D8203BDBB283540132072A3B
:10211000F4D1002081F8AD0730BD00BFE0350120CB
:1021200067DD0408094B93F8AE27012A08D893F815
:10213000AF27012A02D0032A18BF032283F8B2274F
:10214000B3F8B6270020A3F8B0277047E035012088
:1021500010B5044623790E2B00D110BD032B03D1FB
:10216000E3689868FFF7F4FF1434F3E70B49D1F8FC
:10217000B8379A68134618790E280CD19B1A9A1012
:10218000074B534391F8C127013B93FBF2F3013313
:1021900081F8C03770471433EDE700BFE035012008
:1021A000CDCCCCCC094BD3F8C40710B568B1084CE2
:1021B000D4F8EC11013191FBF0F200FB121003EBAB
:1021C0008003C4F8EC01D3F8C80710BDE035012046
:1021D0001400012008B5A0F101030228B3FA83F32B
:1021E0004FEA531301D0184608BD122033F056FDB4
:1021F00028B9054B1B7803F00103184608BD1220CF
:10220000BDE8084033F02AB8C052012010B50C4C8C
:102210004FF49072202104F5007036F0E3FE094B74
:1022200001201A68002384F82B032D32C4F82033D0
:10223000C4F824331846C4F8D82784F8283310BDCE
:10224000E035012058A1012000228273DEE7154A03
:1022500070B492F9C04792F8C157214491FBF4F34E
:1022600004FB1311D2F8B847CBB282F8BC17A168AF
:1022700014246B4304FB03130021C2F8DC3782F8FB
:10228000E0171E79CCB201310E2E09D1AC422346A3
:1022900028BF2B46013B82F8E03770BC0FF092BD9F
:1022A0001433EEE7E035012038B5164B0546D3F878
:1022B000B8271C465268BAB994F8E10798B10138BA
:1022C000114BC0B284F8E10704EBC00000F2E470E7
:1022D00003C883E80300FFF749FF284694F9BC17B9
:1022E000FFF7B5FF002038BD93F9BD07D3F8DC3701
:1022F00000EB800003EB800090470028DCDA4FF011
:10230000FF30F0E7E0350120983D012038B5054663
:102310000C4631B31C4BD3F8B8278A4223D093F82C
:10232000E127511C03EBC20283F8E11703F5F761C3
:1023300002F2E47203C9C3F8B84782E8030000223E
:1023400083F8BD27236833B19847013003D128466D
:10235000BDE83840A8E7FFF709FF00212846FFF74E
:1023600076FF002038BD93F9BD1793F8C12791FB84
:10237000F2F402FB141283F8BD27FFF7F7FE2146A3
:102380002846FFF764FFECE7E035012010B50C4666
:10239000A0B9184A184892F83418236803442360F7
:1023A00001B110BD92F85F314FF4806013492033C2
:1023B000BDE8104001EB8301FFF70EB9FBF71EFEED
:1023C00032280ADC0B4A142892F8341881F00101F3
:1023D0000CDD82F834180A48DFE720680121064B3B
:1023E000044A034482F83418236010BD054882F87B
:1023F0003418D2E7E035012040420F005836012062
:1024000020A1070048E801000C4B10B5044600F875
:10241000011B92FBF3F103FB11230A460849002B31
:10242000B8BF5B4211F020FC202301300C2802DDF4
:102430000023637310BD23540130F7E780969800A2
:10244000C912050810B504460846FEF7D3FE01463A
:10245000FEF700FF0A220346204691FBF2F20449F0
:1024600011F002FC237963712E23237110BD00BF8C
:10247000D112050810B5044B044C1A8804492046B3
:1024800011F0F2FB204610BDD05C0120153E01206A
:10249000D8120508054B0649B3F8482510B503F6D0
:1024A0003A04204611F0E0FB204610BDE035012043
:1024B000D812050870B50D4C054616460B46024667
:1024C0000221D4F840080FF059FC2A46084B142189
:1024D000D4F840080FF052FC33462A46D4F840089E
:1024E0001621BDE870400FF049BC00BFE035012067
:1024F000B4DD040870B51B4D95F8B237012B27D118
:1025000022F044FE0446D8B1174905F6440011F004
:10251000ABFB164D22F012FB044622F0CBFAA46866
:10252000820AC2EB94242B461149124811F09CFBFD
:102530002B4622460E491048BDE8704011F094BB6E
:1025400005F644000D4911F08FFB084D2246EAE7DD
:10255000002405F644000A4911F086FB094D224685
:10256000E1E700BFE0350120DF120508DC120508B5
:10257000EB1205082C3E0120343E0120E51205082F
:10258000B41405089713050808B5FFF7B3FF054B0A
:10259000002093F8B22783F8AF27B3F8B027A3F849
:1025A000B62708BDE0350120012806D003D3022854
:1025B00007D0002070470EF057BD044BD3F85C08DD
:1025C0007047024BD3F86008704700BFE035012028
:1025D00037B504461C4800EB4303B3F85C5005F0E4
:1025E0000F0039B1611CD8B102288CBF20239C2375
:1025F00023700C46B2B1C5F30315FFF7D5FF13499D
:102600003C23012DB0FBF1F191FBF3F203FB12131C
:102610000AD00F49204603B0BDE8304011F024BB7A
:102620009B23E5E71546E8E742F210716425B0FB0D
:10263000F1F0B0FBF5F105FB1100064900902046D2
:1026400011F012FB03B030BDE035012040420F0015
:10265000F1120508FB120508084B07EE900A93F8E3
:102660005B304BB9F8EEE77A9FED057A9FED050AEE
:10267000A7EE870A35F094B9704700BFE035012016
:102680006766E63F0000004238B5044600790D4613
:1026900060B10EF091FF18B1032383710023C37161
:1026A000227A2946BDE838400FF052B838BD00BF45
:1026B00010B504468022002136F094FC382204F143
:1026C0008000002136F08EFC224600230F4850F88F
:1026D0002310013304320E2BD167F8D124220C4988
:1026E00004F1C00035F0C2F80B220A4904F1E400FD
:1026F00035F0BCF800210323102084F8EF1084F893
:10270000F0300EF015FB84F8F10010BD60B0040845
:1027100098B00408BCB0040808B50E4B9FED0E0A33
:10272000D3E900210D4B07EE902AC3F87818F8EE94
:10273000E77AC3F87428F0EEE77A27EE800A10F003
:1027400005FD074A0749137881ED7C0A43F0010330
:10275000137008BDE45E012050E0EF30E035012049
:10276000E15E0120140001202DE9F043B64C85B054
:1027700094F87C38ABB1012B04D00023184605B087
:10278000BDE8F08394F81839082BF6D8DFE813F089
:102790009F00A900B000B900CB00D500F6001701DA
:1027A0002901A0F10A030546222B65D8DFE803F0D2
:1027B0003B64643B6464646464646464646464642B
:1027C00064646464646464646464326464646464FB
:1027D000126412009D4A002094F8823894F88168AF
:1027E000D054002E5FD094F88438022B00F0698119
:1027F000032B00F0A781012B5BD1B31E072B58D808
:10280000DFE813F056014C0147013D0132012A0176
:1028100014010901002284F88128134684F88228D3
:1028200084F88328AAE794F8F038002B4DD0884923
:1028300001F1140313F8012D8B425A70FAD1834A27
:102840001378402B40F23981373B1B01DBB25278C1
:10285000402A8CBF373A303AD2B2134494F88328D6
:10286000DBB29A4200F0AB813F22002384F8F428C7
:10287000002284F8F02881E794F882380E2B04D8DF
:10288000591C724A84F88218D05494F8F038002BFE
:102890007FF473AF94F88308684084F8830818467F
:1028A00005B0BDE8F083137884F88468472B00F006
:1028B000ED81013600232A2D84F8816884F882385E
:1028C000E8D1012284F8F02858E70023D0E7B528A2
:1028D0007FF453AF0023012284F8193984F81829B2
:1028E0004CE7622800F0F681002384F8183945E7A8
:1028F000032284F81A0984F81B09002384F8182994
:102900003CE794F81A29042594F81B190023024483
:1029100084F81C09D2B284F81859114484F81A2991
:1029200084F81B192AE794F81A29052594F81B192D
:1029300000230244A4F81E09ECE7B4F81E3906256A
:1029400094F81A2994F81B19024403EB002084F828
:102950001859D3B280B25A1884F81A39B0F5AC7F3E
:10296000A4F81E0984F81B2940F2228101230022C9
:1029700084F819391346A4F82029FFE694F81A2997
:1029800094F81B190244B4F82039D2B2B3F5AC7FE5
:10299000114484F81A2984F81B1902D2E21882F82B
:1029A00024090133B4F81E299BB29A42A4F82039B5
:1029B0003FF6E3AE0722002384F81829DEE694F8F8
:1029C0001A390822834284F818293FF4D6AED4F885
:1029D0007C2A012100230A4484F81919C4F87C2AAE
:1029E000CCE61C4B0022A3F1140184F8182913F83B
:1029F000012D8B425A70FAD194F81B39834200F0B2
:102A00005C81D4F87C2A3F210023013284F8F41839
:102A1000C4F87C2AB2E601202CF0AAFC94F8816864
:102A200000EB80004000C4F8940842E701202CF03D
:102A30009FFC94F8816800EB800000EB800083002D
:102A4000A4F89A3835E700BFE0350120BCB1012079
:102A5000D43E0120E83E012000202CF089FC94F8AF
:102A6000816884F8900824E71178AD4A30291378FA
:102A70008CBF43F0020323F00203137019E71378AD
:102A8000572B7FF416AFD4F88C385B42C4F88C38DF
:102A90000FE72BF011FCC4F88C080AE71378532BCE
:102AA0007FF407AFD4F888385B42C4F8883800E771
:102AB0002BF002FCC4F88808FBE61B0103F0F003CE
:102AC000C5E6731E082B3FF6F4AE01A252F823F0C0
:102AD000352B0108B3280108B3280108B3280108E1
:102AE000B3280108B3280108152B0108052B01089C
:102AF000F52A010800202CF03BFC94F88168C4F80A
:102B0000A408D6E601202CF033FC94F88168A4F8E0
:102B10009C08CEE601202CF02BFC41F21843814AA0
:102B200003FB00F394F88168A2FB03239B09A4F83C
:102B30009838BEE602202CF01BFC94F88168C4F89B
:102B4000A008B6E6022E00F0CA80032E05D12CF0B4
:102B50000FFC94F8816884F8A908032E7FF6A9AECB
:102B6000331F94F8A878C3F3870303EB8707FD3777
:102B7000FFB2102F3FF69DAEF21EA2EB830303F0CF
:102B8000FF03012B00F0EA81042B0BD100202CF075
:102B9000EFFB7B1E002294F88168234483F8CC0865
:102BA00083F8DC28D4F8EC380133C4F8EC3880E63C
:102BB0000023A4F8203900283FF4FCAEDDE5D4F86A
:102BC0000C29212194F88438013284F8F418012B5F
:102BD000C4F80C2900F08A80022B7FF476AE7221B3
:102BE000514B524AB4F8980884F8F418B4F89C1879
:102BF0009881D981D2E9002313437FF466AED4F8DB
:102C0000A41800293FF461AED4F8A028002A3FF4AC
:102C10005CAE642342F21075454EB1FBF3FEB1FB8E
:102C2000F5F003FB1E1101F5FA61B2FBF3F7B2FBFD
:102C3000F6F6B2FBF5F5BEFBF3FC1A40ADF8041056
:102C400003FB1CEC02EB82028DF806C05200B0FBC5
:102C5000F3F103FB110101A8ADF80C208DF807106A
:102C6000B7FBF3FCB5FBF3F1B6FBF3F203FB1C7708
:102C700003FB115503FB12638DF80A708DF80830C1
:102C80008DF8095011F058F80023F1E55378502BD6
:102C90007FF40FAE9378472B00F06D81522B7FF4B9
:102CA00008AED3784D2B7FF404AE1379432B7FF419
:102CB00000AE022384F88438FBE5D4F80C3994F88C
:102CC00019290133C4F80C39A2B33E22002384F839
:102CD000F42853E50222002384F818294EE52CF04D
:102CE00047FB94F8816884F8A80836E70C4A672106
:102CF000127884F8F41891077FF5BAAD0A4AD4F82F
:102D00008808D4F88C1894F8905810605160D4F862
:102D10009408B4F89A18957490601182A8E500BFE1
:102D2000E15E0120D34D6210E45E0120F03E0120FF
:102D300040420F0094F81C392121023B84F8F4181A
:102D40002E2B3FF61AAD01A151F823F0252F0108D3
:102D5000FD2E01087B2701087B270108A32E01080F
:102D60007B2701087B2701087B2701087B270108B7
:102D70007B2701087B2701087B2701087B270108A7
:102D80007B2701087B2701087B270108692E0108A2
:102D90007B2701087B2701087B2701087B27010887
:102DA0007B2701087B2701087B2701087B27010877
:102DB0007B2701087B2701087B2701087B27010867
:102DC0007B2701087B2701087B2701087B27010857
:102DD0007B2701087B2701087B2701087B27010847
:102DE0007B2701087B2701087B2701087B27010837
:102DF0007B2701087B2701087B2701087B27010827
:102E00007B270108092E010894F828294923102A54
:102E100084F8F43884F8A92840F2C380102284F89A
:102E2000A9287D4B0021A3F17807A3F16806A3F13F
:102E30004805A3F1580093F808E0013193F809C060
:102E400007F801EB914293F80BE006F801CB13F879
:102E50000CCF05F801EB00F801CBECD3D4F8EC383B
:102E60000133C4F8EC383EE05621D4F83C3942F244
:102E700010706A4A84F8F4180121D4F8385984F89B
:102E80009A1A94F8991A958193FBF0F3D38100294B
:102E90003FF473AC0022012384F8992A84F89A2A1B
:102EA0006CE44F2394F82F0984F8F438C30703D552
:102EB00094F82E39032B7FD059490B7823F0020365
:102EC0000B70564B574994F85369B4F8505984F82D
:102ED000982A9E741D82D1E90023134303D100F088
:102EE0000C000C286AD094F8993A002B3FF445ACBA
:102EF00094F89A3A002B3FF440ACCBE7532294F875
:102F0000293984F8F428DA0703D594F82839032BF3
:102F10004ED0434A0021137884F8981A23F0020314
:102F20001370E0E75020D4F834290A253B4BD4F83D
:102F3000281984F8F408D4F82C0959601860384925
:102F400094F8980A92FBF5F29A600B7868B343F014
:102F5000020301220B7084F8992AC9E707F1FF38B0
:102F60000020A04488F8AC782CF002FA94F881682C
:102F700088F8BC0816E6D378472B0BD0D378532BB0
:102F80007FF497AC1379562B7FF493AC032384F82A
:102F900084388EE41379412BF0D1012384F88438EE
:102FA000ECE7002A7FF43DAF58E703F0FD03D0E7DC
:102FB000012384F8983A96E7012282E7B4F92C7944
:102FC000194D4FEAE778194EA7FB0523D4F82809D5
:102FD000174F05FB0833D4F8245990FBF6F012EB99
:102FE00005083D6843F1000918EB000208A7D7E97E
:102FF000006749EBE07312EB060843EB0709B8EBF7
:10300000050269F10003C1E900236CE7AFF300801A
:10301000B0F5F79049000000043F0120E45E012074
:10302000E15E0120F03E012000840C2440420F00AC
:1030300058A1012090B3002270B540F2551582B01E
:10304000AA2613468DF804206C46ADF80050552290
:103050000DF103058DF802108DF80360534008222E
:1030600002E0013ACBB207D059001B06F9D581F036
:103070003103013ADBB2F7D1AC4202D014F8012F90
:10308000ECE70168AA228DF803304B6A69468DF897
:10309000042005221BB1984702B070BD70470EF0A6
:1030A00055F9F9E72DE9F04190F860309AB044699C
:1030B0007BB942680120537884F84430D178937802
:1030C00084F8480043EA0123A4F846301AB0BDE86A
:1030D000F081064602E020680EF082F920680EF0CA
:1030E00087F905460028F6D1014662220DF1060057
:1030F0001A4C35F077FF1A491A4B40F2FF50D1F8BD
:10310000A02A1B68A778134491F89C1A0392132FE6
:103110000493154B154A029373691791ADF8040097
:10312000CDE9052313D894F80180642201A9013761
:1031300002FB084008F10108043034F097FBB8F1B5
:10314000130F7369D8BF5FFA88F5A77065701868A8
:10315000FF211AB0BDE8F0416CE700BF60A4012078
:10316000E035012058A1012020A4012061180108A8
:1031700038B590F860305BB90278032A0DD0042A84
:1031800019D0022A1C4C0FD0002384F8A43A38BD71
:10319000194B002283F8A42A38BD174C84F8A53AAD
:1031A000002384F8A43AF2E7012384F8A53A002327
:1031B00084F8A43AEBE701254268017E52780E4C70
:1031C000A94202F00F0284F8A55A09D00229DBD1E6
:1031D000002AD9D0162084F8A63A1CF099FAD3E731
:1031E0002AB1152084F8A61A1CF092FACCE7162012
:1031F0001CF08EFAC8E700BFE03501202DE9F04150
:103200001E460023074608468B550C469046751E01
:1032100033F046F9301A2544211840426A1A2B1B14
:10322000002A12DA234420211A1B002A11DA002373
:1032300042463846A355084B93F8A71A2346891BE4
:10324000BDE8F041C9B20EF099BD2B5C05F801391B
:10325000E4E703F80119E7E7E03501202DE9F04143
:10326000144C94F82A5385421BD9064688461046CA
:10327000174633F015F9AA1B04F5007305FB086522
:10328000824239461D444444A8BF02462846164699
:1032900035F080FE002814BF0123002384F820337A
:1032A00001D1BDE8F081324639462846BDE8F041FB
:1032B00034F0DCBAE035012030B583B014460D4659
:1032C0001A46084901A810F0CFFC074B93F82933A0
:1032D000A34204D901AA21462846FFF7BFFF0020D8
:1032E00003B030BD3C150508E0350120074890F8D3
:1032F0002903904207D9084611461A4608B5FFF738
:10330000ADFF002008BD0020704700BFE035012060
:10331000F8B507460026F5B20024E0B201342022B9
:1033200029460CF0BAFC0C2CF7D10136092EF2D14B
:1033300042221B4D0120441C00210CF0AEFC15F86C
:10334000012FE4B22046002AF5D197F90E302BBBAD
:103350001446144D4D22E0B202210CF09EFC15F8EB
:10336000012F0134002AF6D12B220F4D0220441CDC
:1033700003210CF092FC15F8012FE4B22046002A3C
:10338000F5D12B22094D0220441C04210CF085FCB0
:1033900015F8012FE4B22046002AF5D10020F8BD2F
:1033A00018EA0408581505084C15050840150508C5
:1033B00010B500248473FFF7ABFF204610BD00BF9B
:1033C00070B516461A785AB11D460846441C314657
:1033D0000CF063FC15F8012FE4B22046002AF5D169
:1033E000002070BD084611461A460CF056BC00BFBE
:1033F00070B50B4C4FF0FF3504F525762368DC34AF
:10340000184643B193F83430142B04D00DF0ECFF80
:10341000854228BF0546A642F0D1284670BD00BFB0
:1034200058AC01200B4B0C4910B593F8A92A82B077
:1034300093F8A83A04240D3209781E338DF804401D
:103440000272437221B901210DEB040028F0A8FC9F
:1034500002B010BDE0350120D85C01202DE9F0411B
:1034600018468AB01D460F46904633F019F81E28BC
:103470004FF003034FF00004294628BF1E208DF8AB
:1034800004308DF805800246064602A88DF80670C5
:103490008DF8074034F0EAF9064B1B781BB1204643
:1034A0000AB0BDE8F081311D01A828F079FC0AB00E
:1034B000BDE8F081D85C012010B582B000248DF801
:1034C000043001AB8DF80540FFF7C8FF02B010BD16
:1034D000094B042200B583B01B788DF804201BB182
:1034E000002003B05DF804FB01210DEB020028F081
:1034F00057FC03B05DF804FBD85C0120094B0222A5
:1035000000B583B01B788DF804201BB1002003B0F8
:103510005DF804FB012101A828F042FC03B05DF82E
:1035200004FB00BFD85C0120084B012100B583B02B
:103530001B788DF804101BB1002003B05DF804FB6C
:1035400001A828F02DFC03B05DF804FBD85C012035
:10355000074B002000B583B01B788DF804001BB921
:10356000012101A828F01CFC03B05DF804FB00BF9A
:10357000D85C0120ECE700BF70B5104C054694F80C
:10358000AD6A46B9012384F8AD3A22F0F3FB22F08C
:10359000ADF884F8AD6A0A4B94F8631593F8F431EA
:1035A00094F8622513F0400F02F11E0214BF10239D
:1035B0000D236A720B442B7270BD00BFE0350120F1
:1035C0001400012022F02CBD084611461A4608B509
:1035D00022F04CFD002008BD08B5064B93F8AD2A3B
:1035E00012B993F8AE3A0BB1002008BD23F038FFB2
:1035F000002008BDE035012010B50A4C94F86405A0
:1036000022F0DCFD94F8661594F8650522F04CFD77
:1036100004F54B704FF4F072202135F0E3FC0020EC
:1036200010BD00BFE035012010B504460121FFF7B1
:103630002BF800212046BDE8104023F047BB10B511
:1036400004462221FFF720F8204623F011FB2046F4
:103650000121BDE8104023F039BB38B5A0F66C0459
:10366000D4F84C380022354D1B685A62A1F1290369
:10367000302B31D895F8AF3A0133DBB2012B85F806
:10368000AF3A0BD995F8B03A85F8AF2AB4F85A2872
:103690000133520885F8B03AA4F85A2895F8B02AB0
:1036A0000023082AA4F85C3815D185F8B03AB5F89B
:1036B000B23A01339BB2032BA5F8B23A08D9237969
:1036C000DB0705D5E36A94F85A085BB3216B98478A
:1036D0000023A4F85A3838BD5B396C290ED8B4F8E9
:1036E0005A3885F8AF2A5B0843F08003A4F85A38AB
:1036F00095F8B03A013385F8B03ACFE794F85538E9
:10370000002BCBD1012185F8AF3AA5F8B23A80233E
:1037100084F85518A4F85A38206C85F8B01A26F0A9
:10372000B3FBBBE7E3696269D054E369E168013345
:10373000B3FBF1F201FB1233E361C9E7E03501208D
:1037400038B5A0F66C0423796579DB0722D594F8A7
:10375000503803B3D4F848381A68D36A5B08536208
:1037600094F8543823B1B4F85E380133A4F85E38C5
:10377000E943206C01F0010126F086FB012384F867
:103780005338002384F8513884F85238A4F85A3852
:1037900084F8503838BD94F85338012B03D194F88D
:1037A000513884F852382046FEF72DF994F85338F2
:1037B0004BB90123E943206C84F853381940BDE824
:1037C000384026F061BB002305F00101206C84F82D
:1037D0005338BDE8384026F057BB73B590F86338CE
:1037E00005460C46032B2FD10023204E8DF80730C1
:1037F0009DF8073095F864289A4201D802B070BD50
:103800009DF8073006EBC30393F8B83A8BB184F008
:10381000010383B19DF8073006EBC303D3F8B40A64
:103820000EF004F99DF807300133DBB28DF8073054
:10383000DEE72346EDE79DF8073006EBC303D3F838
:10384000B40A0EF0EDF8EDE7036CC06BDB79DB0733
:1038500048BF81F0010424B102B0BDE870400EF011
:10386000E5B802B0BDE870400EF0DAB8E0350120EE
:1038700070B5A0F6680494F8553893B1B4F85C3884
:1038800001339BB2082BA4F85C381CD90021206CB2
:1038900084F85518A4F85C1826F0F6FA94F8553810
:1038A0008BB93D4E96F8F43A1BB901212046FFF73B
:1038B00094FF94F854384BBBD4E909239A4203D1BE
:1038C000002386F8F43A70BD96F8F42A022A12D83A
:1038D00002F1010214BFFF237F2386F8F42AA4F823
:1038E00058380823206C84F85638012384F854385B
:1038F000BDE8704098E65A1CA169A262CB5C2169C0
:10390000DBB28A42EBD30022A262E8E794F9563890
:10391000C3B394F8581896F8F55A11F0010123D062
:10392000012D03D801212046FFF757FFAB1E012BC5
:1039300003D800212046FFF750FF0135EDB2032DDB
:1039400086F8F55ABFD9B4F8583800225B0886F8D3
:10395000F52AA4F8583894F85638013B5BB284F83D
:103960005638002BA8D0AEE715F0FD0304D1012195
:103970002046FFF732FFE0E7012BDED12046FFF7BC
:103980002CFFDAE7D4E9091291429CD184F854382B
:10399000206CBDE8704052E6E035012010B5A0F67D
:1039A000680494F8553823BB94F8542892BBD4E9A2
:1039B000091399421DD0591CA069A162C35C2069FA
:1039C000DBB281424FEA430328BFA26243F4007393
:1039D000A4F858380A2384F85638012384F8543858
:1039E00094F86338012B01D0042B02D1206CFFF72F
:1039F0001BFE94F85038002B6FD194F851380133E6
:103A0000DBB2092B84F8513827D12046BDE810409D
:103A1000FDF7F9BF94F956387BB1B4F85818204631
:103A20004B0801F00101A4F85838FFF7D6FE94F8CE
:103A30005638013B84F85638DBE784F85438D4E92B
:103A400009239A42D5D194F86338012B01D0042B75
:103A5000CFD1206CFFF7F3FDCBE70A2B3DD194F8D3
:103A600053382BB9B4F85A3843F00103A4F85A3844
:103A70002379D9070AD5B4F85A08820501D4C307B7
:103A800018D4B4F860380133A4F860380122002358
:103A900084F8502894F8532884F85138012A1CD10E
:103AA000617984F85338206C01F00101BDE81040C1
:103AB00026F0EAB9E36AC0F3470013B1216B9847D7
:103AC000E4E7E3696269D054E369E1680133B3FB79
:103AD000F1F201FB1233E361D8E710BD2DE9F04F9D
:103AE000A74C85B094F8F63A039003F0FF07002B3B
:103AF00070D1B4F8FC1A4FF03C0994F8F82A04F598
:103B0000B67C0291B4F8FE1A94F8F95A019149462C
:103B100094F8FA3A9CF802609CF803E0C6F1FF06BC
:103B2000B6B2002E00F0AC80BCF80080C6F1FF06F3
:103B3000B8FBF9FA0EFB06F63612BAF1050F0ED8ED
:103B4000DFE80AF0034B5C6B7E8DAEEB0605F3B24B
:103B5000724608FB05F5B5FBF1F51D44EDB203987F
:103B6000012840F091802E0246EA02461E434FF0A3
:103B7000170E07EB0E0B0120ABEB0E0800FA0EFA46
:103B800001981FFA88F81AEA060F8246029808BFC1
:103B900082467C481EF1FF3E40F828A0EBD2183741
:103BA0000CF1040CBFB2B7F5407FB3D184F8FA3AF8
:103BB0002023A4F8007BA4F8023B012384F8F82A10
:103BC00084F8F63A94F8043B84F8F95A002B60D153
:103BD00084F8F63A05B0BDE8F08FB8FBF1F201FBCE
:103BE0001282F3B2AEEB0606754692B2C2F13C0207
:103BF0007243B2FBF1F21A44D2B2B0E7B8FBF1F370
:103C000001FB1383F2B2AEEB060675469BB273431B
:103C1000B3FBF1F31344DBB2A1E7B8FBF1F301FB13
:103C20001388F2B273461FFA88F5C5F13C08AEEB73
:103C3000060505FB08F5B5FBF1F51544EDB28EE779
:103C4000B8FBF1F301FB1382F5B2AEEB0606734647
:103C500092B27243B2FBF1F22A44D2B27FE7B8FBD0
:103C6000F1F301FB1383F5B2AEEB060672469BB28D
:103C7000C3F13C037343B3FBF1F32B44DBB26EE7B8
:103C80007346754672466AE7160246EA05461E43C3
:103C90006DE794F8453B022B01D1002398E794F897
:103CA000452BB4F8483B012A02D1022284F8452B67
:103CB000D4F8082B0C2B14D8DFE803F007131313E8
:103CC00024131313311313133E00D4F82C0B343286
:103CD0002D4B2C49C3632D4BC36440F22A3307F0AC
:103CE0004BFD0022D4F8083B5A62B4F8482B0C2A4A
:103CF00033D8DFE802F02E323232363232323B3203
:103D000032324000D4F8300B38321F4B1D49C363A8
:103D10001E4BC36440F22A3307F02EFDE1E7D4F8CE
:103D2000340B3C32184B1749C363184BC36440F241
:103D30002A3307F021FDD4E7D4F8380B4032124B78
:103D40001049C363114BC36440F22A3307F014FDDA
:103D5000C7E7DA6842F40072DA60012384F8453B71
:103D600038E7DA6842F48062DA60F6E7DA6842F44B
:103D70000062DA60F1E7DA6842F48052DA60ECE778
:103D8000E035012038000020699901087799010881
:103D90002DE9F04FC04D91B095F84A3B13B911B0E1
:103DA000BDE8F08F95F8F63A002BF8D104460F20C5
:103DB00031F054FAE8B195F86731B3B9B74C94F8DB
:103DC000F531002BEBD0B64A0023DFF8F4821268FD
:103DD00048F823200133202BFAD195F86A01FFF728
:103DE0007DFE002384F8F531D9E795F8FF31002BEB
:103DF000E4D001220023A94990461F46B5F84C0B98
:103E0000A84EDFF8C0E2DFF8C0C2DFF8C09281F848
:103E1000F52140FA03F29900D2070DD456F8232079
:103E200008FA03FAA21A02EB0E0BE34504D94A453D
:103E300047EA0A0788BF8C510133092BE9D1002FCB
:103E4000ADD0994B1B7813F00103039340F04881E8
:103E5000039B95F86821C5F8F03105EB420395F80E
:103E60007410B3F9743B0793C5F8983B002900F030
:103E7000D280A3F57A704FF4B473DFF854C24FEADE
:103E8000810A03FB00F395F85F21DFF848B2D146C1
:103E90008CFB031EDB17203295F85C41C3EBAE139D
:103EA00095F85D110BEB82062034069320313BF828
:103EB00022300BF1F4080D900093F3787B480193C6
:103EC0000BEB8403CDF810C00A93B3780026089753
:103ED00002930BEB81030B93038805935BF8063089
:103EE000C3F3032203F48057042A1CD8DFE802F04E
:103EF0002503C7C4AF00402100220598084207D11E
:103F00000132042A0FD06A4931F822100029F5D174
:103F1000C3F38553002143FA01F0C00700F1228169
:103F200001310629F7D1029C4FF4B473DDE9002179
:103F3000002F59D00698034456E0C3F3834303F19E
:103F4000110C03F10F0020330CF00F0C00F00F00E8
:103F50000BEB83013BF823200CF1200C20308C78F4
:103F60000BEB8C033BF82CA00BEB800E3BF820C036
:103F70009878DB78C9780C939EF802309EF803E0BD
:103F80000993002F00F0848040F2DB57079BBB426F
:103F900000F3B480099BA1EB0E010D9FA2EB0C0274
:103FA000E01A049C07FB01F14FF4B47307FB00F027
:103FB00007FB02F24FEAE07A84FB00070C97CF1769
:103FC00084FB01010498D41780FB02020C98C7EB14
:103FD0006111C4EB6212099CCAEB60107144624427
:103FE0002044C9B292B2C4B21344324A4FF4B47CF2
:103FF00008EB060782FB0320DA171844C2EB2022E5
:104000000CFB123228F806200436BC70B145F9705A
:104010007FF464AF089F234E0024DFF8BC804FF08C
:104020000109254B01E058F8043F09FA04F2013474
:10403000314604363A4214BF012000209847092C2B
:10404000F1D195F86A0111B0BDE8F04F46E5F9F7F6
:10405000D5FF00B20022FF2100EB80001446C0EB28
:10406000001043001548A0FB03035B091E3B23EA35
:10407000E37303F5B4735BE71AF0A8FCE9E7039B6D
:1040800063B30B9A94784FF4B473D17812884FE7E6
:104090004FF4B473A8E700BFE035012014000120FD
:1040A00060B0040830410120C0520120F8BA01205C
:1040B000C8B00408B7600BB6691201081F85EB5140
:1040C0004C3701203F4B4C003E4B4C009F8601007B
:1040D000D34D621058360120D8B004080A9AD1E7AF
:1040E000B5F97A1B64232A4AA1F57A7103FB01F31F
:1040F00082FB0312DB17C3EBA213AAE60C9B071B80
:10410000AAEB020A581A079BA3F2DC5C4FF4B473C3
:104110000CFB00F00CFB07F786460CFB0AFAF817BD
:104120000E90049880FB07C704980C977746099077
:104130004FEAEE7E80FB07C74FEAEA7C0F970746FF
:104140000C9887FB0A7A0E9FC7EB60170F98CCEB91
:104150006A1ACEEB60103C4452440144E4B292B27D
:10416000C9B241E70B4B03EB82024FF4B47392F8F0
:104170006A2002EB420205EB4202114491F8382119
:1041800020320BEB82013BF822208C78C978CFE6F5
:10419000D34D621060B0040838B5124C217AE07932
:1041A0000AF01EFAA379104A013B32F813300F4A85
:1041B00013800F4A12889A4202D00E4B02221A70C4
:1041C00009F070FD0C4DE079217AA3796970AB702C
:1041D00028700AF0F1F9A8800EF070FC4FF0FF3063
:1041E00038BD00BF14000120F8B504085E5C012052
:1041F000605C0120625C0120B652012008B5084BCA
:1042000093F8421521B9012283F84225002008BD08
:104210004B1E49205942594109F084FDF6E700BF81
:10422000E035012008B5044BB3F8460540F40040E2
:1042300009F08CFF002008BDE0350120364B70B539
:1042400086B01A7800268DF80C2003AD5A786C469B
:10425000CDF80E608DF80D209A78CDF812608DF8AB
:104260000E209A88ADF810201A7A8DF8142095E85F
:10427000070003C422801C46284A1278022A30D143
:10428000274B1878274B8DF8000019788DF801100E
:104290000AF092F9244BADF8040093F89C3BE3B983
:1042A000052009F0FFFE214B0A22694628461E78A8
:1042B0008DF8026034F06EFE58B19DF80030A670A3
:1042C00023709DF801306370BDF80430A3800EF0B8
:1042D000F5FB4FF0FF3006B070BD062009F0E2FE9E
:1042E000E1E7134B1B7863B90D4B18780D4B8DF834
:1042F000000019788DF801100AF05EF9ADF804009D
:10430000D1E7304609F0CEFE0A4B8DF800601B88DD
:10431000ADF80430C7E700BFB6520120C85C0120E9
:10432000CA5C0120CB5C0120E0350120CE5C01207D
:10433000D25C0120D05C012008B50C4B93F9003011
:10434000012B0B4B04D1002283F89C2B002008BDCD
:1043500093F89C0B18B9012283F89C2BF6E70128EF
:1043600018BF022009F09EFEF0E700BF9C1E01204E
:10437000E035012070B5124C0546124B0E4694F9FB
:1043800000401A78012C05D1012A01D001221A70AF
:10439000002070BD012A03D1002009F083FEF7E759
:1043A000022AF3D10024084B83F89C4BFFF7C4FF8B
:1043B000064B314628461C70FDF716FCE8E700BFA7
:1043C0009C1E0120C85C0120E0350120D25C012048
:1043D00008B5074B93F90020064B12B91A7000205C
:1043E00008BD1A780AB90122F8E7FDF79FFBF6E746
:1043F0009C1E0120CA5C012008B5074B93F90020E0
:10440000064B12B91A70002008BD1A780AB90122A9
:10441000F8E7FDF78BFBF6E79C1E0120CB5C012043
:1044200008B50A4B93F8D02542B193F8D1253AB19B
:10443000D3F8A02B42F48032C3F8A02B002008BD93
:104440004FF480300DF032FFF8E700BFE035012077
:1044500008B5064B93F8D30528B10138044BC0B218
:10446000597817F0CDFA002008BD00BFE0350120D3
:10447000FCAE012008B5064B93F8D20528B10138EF
:10448000044BC0B219782DF055FF002008BD00BFC5
:10449000E0350120FCAE012038B5144D602395F8BD
:1044A000DE4503FB045495F80D3784F82736104B8E
:1044B00018682EF05BF995F80E37002084F8FA356D
:1044C00095F80F3784F8FB3595F8103784F8FC35EC
:1044D000B5F81237A4F81436B5F81437A4F8123624
:1044E00095F8163784F82F3638BD00BFE035012027
:1044F000FC5E012038B50D4B00210D4A186802F111
:10450000090503461478063303329C7012F8024CF6
:10451000DC7012F8014C1C7135F81140013103298F
:10452000DC80EFD12EF022F9002038BDFC5E0120A6
:10453000773D012008B5054B93F817070138C0B245
:1045400083F8960717F080FA002008BDE0350120B7
:1045500008B5054B93F80C070138C0B283F8DE05A7
:104560000CF03AFB002008BDE035012010B5054CE9
:1045700094F8DE050CF030FB94F8960717F064FA17
:10458000002010BDE035012010B5044620F0FEFDEE
:10459000D8B120460DF016FC0F4B03220521204612
:1045A0000DF0ECFB20460DF0D7FB20F0B1FA20F027
:1045B000F5FD60B113201BF0ABF820460DF002FCB6
:1045C00020460DF0C9FBFDF795FF002010BD6420CB
:1045D0000CF0F2FDEBE700BF0A130508F8B54B1E1F
:1045E00004460F461D4E012B0CD81D4BD3F800027C
:1045F000FDF7AEFDD6F8B8375B680BB100209847E1
:104600000EF05CFA0025236820465B6886F8A45B00
:104610009847A37B022FC6F8B85703F1FF33A37363
:1046200014D120460DF0CEFB0E4B0322052120466F
:104630000DF0A4FB20460DF08FFB31F051F830F067
:10464000B9FFC8200CF0B8FD22F092FA064A2846BD
:10465000136823F400531360F8BD00BFE035012058
:10466000140001201B13050818BB0120394B93F8D7
:10467000A42B70B51C46002A41D1D3F8C41711B938
:10468000C3F8A81B70BD344BD3F8EC110029B8BF98
:10469000C3F8EC21D3F8EC3104EB8303D3F8C8372B
:1046A000C4F8A83B002BEDD001234FF4005084F850
:1046B000A43B2A4BC4F8B8370023A4F8BC370CF04D
:1046C00097F9D4F8A80B0DF06FFBD4F8A80B0121D3
:1046D000427A037A112A2DD884F8AC1B02215B0898
:1046E00084F8A72A84F8AD1B002184F8C13784F828
:1046F000AE1BD4F8B817BDE87040FDF707BEFDF754
:1047000051FDD4F8A85B06468542BBD094F8BD277E
:10471000284694F8BC1794F8C13701FB032384F8AA
:10472000BD372B685B689847AB7BC4F8A86B013B2F
:10473000AB73C6E7002584F8AD1B023A0221023BA9
:1047400084F8AC5B84F8AE1B84F8A72A84F8C137E0
:10475000CFE700BFE0350120140001200C0201204A
:104760002DE9F04FBA4D8BB08146D5F8C437002BF8
:104770003BDBD5F8B03B03F543435033984234D389
:1047800095F8A67AC5F8B00B7FBBB24B1B781BB966
:10479000B14B1B78012B28D095F8A43B0393B5F8B7
:1047A0007A3B039AA3F2E3439BB20ABBB3F5F97FCA
:1047B00016D8B5F9782B40F2E1439A4210DCB5F9EE
:1047C000762B40F2D6639A420ADDA44B1B78D807B9
:1047D00006D4FFF74BFFA24B4FF4FA72A3F8042262
:1047E000A04B1A689A4BC3F8B82B0BB0BDE8F08FFA
:1047F000B3F5F97FB5F9762BDFF864A214D8B5F9D3
:10480000781B40F2E14399420EDC40F2D6639A42B3
:104810000EDD924B1B7813F0010F0CBF0624012410
:10482000DAF80C3201331CE040F2D6639A423FDCE6
:1048300040F2E1418A423DDDB5F9743B8B423BDDFC
:1048400040F2D662934239DCB5F8783BA3F2E243FA
:10485000B3F5FA7F34D801230024CAF80832C5F82A
:10486000B44B4FF47A72CAF80C32B9FBF2F20292EE
:10487000BAF90422002A25DDD5F8B83B1344029A80
:104880009B1AAAF80432724ED6F8DC37002B40F09F
:10489000B681D6F8BC3B029A03F5FA739A429FD9C7
:1048A000D6F8A80B0DF05CFA029BC6F8BC3B97E764
:1048B0000124B5E70224B3E70324B1E70424AFE7FA
:1048C0000524ADE7002CDED0DAF808324FF0000BFB
:1048D000621ED5F8A88B01935B46D2B25C4E04925F
:1048E000019A5A4525DC033CAAF80432012CCAD8A7
:1048F000DAF80C22142AC6DDA2F1140193FBF1F3BD
:10490000322BAAF80432BEDCD6F8B43B0BB9C6F899
:10491000B42BD5F8B43B0521D21A514B92FBF1F2DE
:10492000D3F8080202448A42C8BF0A46C3F80822E4
:10493000A9E7D6F8B8370BB9FA2305E0062C06D15B
:10494000FFF794FE4FF4FA730BF1010BC8E7052C47
:1049500005D14046FDF7A8FC4FF4FA73F4E7022CAA
:104960003FD196F9BD3796F8E02793422EDA01330E
:1049700086F8BD37049B012BDED995F9BD37D5F8F4
:10498000DC2703EB830302EB83031A79013A0C2A39
:10499000D2D801A151F822F053490108894A0108EF
:1049A0003B4A0108694A0108A34A0108754B0108FE
:1049B000F74A0108A94B0108D94B010839490108F8
:1049C000F74A0108C54A01083D4B010896F8BC1793
:1049D0004046013149B2FDF73AFC002386F8BD3765
:1049E000C8E7012CC6D196F8BD17D6F8DC274B1EB8
:1049F0005BB203EB830086F8BD3702EB80000079E1
:104A000020B9002B02DD023986F8BD1796F9BD37B3
:104A1000591C06D003EB830302EB83031B79002BA5
:104A20008AD196F8BC174046013949B2FDF70FFC10
:104A300096F8E03786F8BD379CE7042C7FF47CAF0E
:104A4000D9684046FDF762FC4FF4FA737CE700BF7B
:104A5000E0350120F2520120E0A30120C0520120E4
:104A60001400012058A101209A68002A3FF464AF85
:104A7000042C7FF461AFD9684046904701303FF481
:104A800068AF4FF4FA735FE79A68002A3FF454AFB7
:104A9000042C7FF451AFD968404690474FF4FA7325
:104AA00052E7DA68002A3FF447AFA4F1040CDCF1C6
:104AB000000141EB0C0111701A7C42F001021A74E2
:104AC000FA2341E7D86800283FF436AF042C028867
:104AD00008D142F4006202801A7C42F001021A748A
:104AE000FA2331E740F6010192FBF1F101EBC1211C
:104AF000521A92B2EFE7D96800293FF41DAF086857
:104B0000042C027812D191F805C0944502D9897914
:104B10000A4402701A7C42F001021A749A68002A50
:104B20003FF40AAF19464046904705E791F804C0A4
:104B30009445EFD28979521A0270EBE7D868042CB9
:104B400001680A7811D10079904201D901320A70C6
:104B50009A6822B1D968404605939047059B1A7C14
:104B600042F001021A74FA23EEE6002AF0D0013A6C
:104B70000A70EDE7DA68002A3FF4DEAE1068042C14
:104B800001784FFA81FC07D192F905E0E645C1DDD5
:104B9000927911440170BDE792F904E0E645B9DA73
:104BA0009279891A0170B5E7D96800293FF4C4AE3B
:104BB0000868042C028807D1B1F806C09445A9D929
:104BC00009890A440280A5E7B1F804C09445A1D23E
:104BD0000989521A02809DE7D96800293FF4ACAEDA
:104BE0000868042CB0F9002004D1B1F906C094453E
:104BF00090DDE5E7B1F904C094458BDAE8E796F873
:104C0000AC3BD6F8A88B002B40F0BB8096F8E02791
:104C100098F808309B1A022293FBF2F3DBB201935F
:104C2000D5F8C03B03F5C333A033994502D9039FA0
:104C3000C5F8C09BD8F800304046DB6A984798F822
:104C40000C301FFA80F9002B00F0A580D6F8DC3775
:104C50001A790E2A40F09880002388F80C30D6F894
:104C6000DC0796F8BD3759B2013301EB8102DBB2A4
:104C700000EB82021279002AF5D098F90D2086F80F
:104C8000BD17002A0FDB8A4229D096F8AD3B40467B
:104C9000019903FB0212B04B96F8AE1BD2B20DF095
:104CA0006DF8A9EB0009B9F11D0F7FF6F2AD96F989
:104CB000BD2798F90D30934215D096F8AD3B40468C
:104CC000019903FB0212A54B96F8AE1BD2B20DF070
:104CD00055F896F8BD37A9EB000988F80D30B9F101
:104CE0001D0F7FF6D6ADD6F8DC474FF0000B5FFA0C
:104CF0008BF796F8C137BB427FF6CBAD23790E2BED
:104D00003FF4C7AD227C900719D5019896F8AE1BE9
:104D100096F8AD2B002B18BF0131236802FB070268
:104D20004046C9B2D2B20DF029F8237CA9EB0009A4
:104D300023F00203B9F11D0F23747FF6AAAD227C84
:104D4000D10778D595F8AD3B019903FB071795F886
:104D5000AC3BFFB20BB10137FFB223790D2B00F250
:104D6000F680DFE813F0DD00F400F4003A003A00CA
:104D70006C0098008E00A200A2002E00AB00830001
:104D80007700012301934BE71A7C143342F00302AE
:104D900003F8042C5CE7002F3FF461AF95F8E0378F
:104DA000D5F8DC2703EB830302EB83039A423FF63B
:104DB00056AF117C4C0702D541F001011174143239
:104DC000F4E7E168002900F0C2800C2206A834F064
:104DD000FFF90C233A4606A920E00DF1280A4FF00E
:104DE0000001032B0AF8101D09D1A3683BB112077B
:104DF00005D598470C220146504634F0E9F9574949
:104E0000504634F0AFF996F8AC3B0BB1013FFFB21E
:104E1000504631F045FB3A46C3B251464046FEF794
:104E2000EDF9237C23F001032374A9EB0009B9F108
:104E30001D0F7FF62EAD14340BF1010B57E7E06820
:104E40000028F2D00378BBB1454906A834F0A6F992
:104E50000323BFE7E36806A81A689B6811780C2251
:104E600053F8211034F0B4F90C23B3E7E0680028BC
:104E7000DBD003881B05E7D43A4906A834F08EF945
:104E8000E6E7E0680028D0D0036806A9187829F082
:104E90008BFA05239EE7E0680028C6D0036806A9C0
:104EA00093F9000029F080FAF3E7E0680028BCD00D
:104EB000036806A9188829F077FAEAE7E06800286D
:104EC000B3D0036806A900891B78584300F5C330A6
:104ED000A03029F069FA9DF81A209DF819308DF854
:104EE00019202E228DF818308DF81A209DF81D20DB
:104EF000302A01D02E2A0DD14FF000028DF81D204E
:104F00009DF81C20302A01D02E2A03D14FF0000238
:104F10008DF81C20302BBCD120238DF81830B8E739
:104F2000D4F80CA0BAF1000F13D0206831F0B8FA11
:104F300095F8AE1B53463A46013101444046C9B28A
:104F40000CF01CFF237C23F0010323746DE7002089
:104F50006BE7504669E700BF8B1405082813050866
:104F60002A1305082E13050870B50B4C05460B4E89
:104F70002146023C0EF090FE2B6821462C601C1B43
:104F800006F6C4306B60402CA8BF4024224632F0A5
:104F90006DFC86F8044C70BDCE530120E035012035
:104FA00003885A0608D513F4057F05D00A4A127AF9
:104FB000072A01D80120704703F48253B3F5825FBA
:104FC00001D000207047044B187AA0F10700B0FA16
:104FD00080F04009704700BF68B101202DE9F0431F
:104FE000B94C85B094F8053C012B00F0EA8094F8A8
:104FF000110CFDF7EFF894F8123C0546834208D0F7
:10500000002870D1B14E30681AF0C3F9356084F8C9
:10501000125C94F8133C012B00F08C80D4F81C5CDB
:1050200094F8207CADB32846FFF7BAFF88B33FB9A8
:10503000D4F80C3C23B1A64901220B6084F8202C43
:10504000D4F8245C94F8287C002D39D02846FFF74A
:10505000A7FFA8B33FB9D4F80C3C23B10122C4F890
:105060002C3C84F8282C94F8310CFDF7B3F894F814
:10507000323C0546834209D000286DD1D4F8380C63
:105080001AF087F9C4F8385C84F8325C05B0BDE8E2
:10509000F08394F8210CFDF79DF8B8420646CFD076
:1050A000002840F0A5808A4D28681AF072F92E6019
:1050B000D4F8245C84F8206C94F8287C002DC5D1A9
:1050C00094F8300CFDF786F8B8420646CBD000289D
:1050D00040F0B380D4F82C0C1AF05BF9C4F82C6CB7
:1050E00084F8286CBFE77B4B1B68002B91D07A4972
:1050F000032593F90200002349794FF49642019564
:1051000099424FF0080100921A460CBF1D460D4609
:1051100002951AF053F96D4B186000283FF479AFEF
:105120000AF056FD012384F8123C94F8133C012B3D
:105130007FF474AF694D94F8140CFDF74BF82B68AD
:105140000646002840F09E80002B3FF467AF1846CB
:105150001AF01FF92E6061E7614B4FF47A72D4F8B0
:10516000345CC3F8E822002D90D04FF480524021E7
:1051700028461AF009FA0646002887D1564B4FF404
:10518000E13295F90200032719793346009232463D
:10519000002901974FF480510CBF0825092502957D
:1051A0001AF00CF9C4F8380C00283FF46FAF4D49E1
:1051B00001234D4A84F83C6C0860167084F8323C38
:1051C00064E7D4F8086C494D3046FFF7E9FED5F89E
:1051D00000800746002800F08D80B8F1000F7FF4B2
:1051E00006AFD4F80C3C002B3FF401AF2B60FEE679
:1051F000002D3FF425AFAB79002B00F09F803C4A97
:1052000002EB8303D3F89C10334E002395F9020080
:105210000222357900911021ED1A01921A4618BF29
:10522000012502951AF0CAF8294B186000283FF4AE
:1052300007AF012384F8203C02E7002D3FF413AFB1
:10524000AB79002B77D02A4A02EB8303D3F89C106A
:10525000214E002395F902000222357900914FF486
:105260000071ED1A01921A4618BF012502951AF035
:10527000A5F8C4F82C0C00283FF4F5AE012384F8FF
:10528000283CF0E6002B7FF4C9AED4F8182C002A95
:105290003FF4C4AE1049032692F902004F790A790F
:1052A0004FF46141002F019600914FF020010CBF97
:1052B00000260826002A08BF46F001061A46029674
:1052C0001AF07CF82860A9E6E0350120145F01207F
:1052D000D05E0120185F0120904A0120085F012064
:1052E00078220120205D0120F85C0120E852012095
:1052F00060B0040894F8100CFCF76CFF814600B312
:10530000002E3FF474AEB8F1000F7FF470AE124976
:10531000022296F902004FF416530E7904210192ED
:105320003A46B6FA86F600933B46760902961AF09C
:1053300045F828605BE64FF4614189E74FF49641F8
:1053400062E7B8F1000F3FF452AE40461AF021F880
:10535000C5F800904BE600BF904A0120034A0123A4
:1053600003FA00F0536E034353667047E0350120A3
:1053700008B50146831E00F15402EA2023F8020F0B
:105380009342FBD140F6491303204B85224B4B60DF
:10539000CE230B8100234B66FFF7E0FF0520FFF7CC
:1053A000DDFF0820FFF7DAFF0920FFF7D7FF0A200B
:1053B000FFF7D4FF0C20FFF7D1FF0D20FFF7CEFF42
:1053C0000220FFF7CBFF0123144A81F85B30B2F8CB
:1053D00060306FEA53236FEA4323A2F86030104B2A
:1053E000CB65142381F85A3040F69803A1F8563063
:1053F0006423A1F85830802381F868304FF6FF739A
:10540000A1F86A30A1F86C30462381F86E3042F67C
:105410001403A1F8623008BDCD004E00E035012034
:10542000000A010A30B585B0054601A80EF096FCC9
:10543000044618B92870204605B030BD044A01233F
:1054400001A92846B2F93E2C0EF0AEFCF3E700BFEE
:10545000E03501200F2A03D8052803D805290CD9E7
:1054600000207047062815D00029F9D10728F7D168
:105470000C4B012083F86821704710B400EB400307
:10548000084C012004EB4303194481F838215DF8EE
:10549000044B70470A29E3D8024B0120194481F8D4
:1054A0005C217047E03501202DE9F04100F1200832
:1054B0001F4F0D4640F2671607EB8807002412E0E5
:1054C000022C31D187F87B0028462C2133F059FE7D
:1054D0000546C0B1013401350120022C1CDCE0B1CD
:1054E000144B33F8146028460EF0D2FF864214DBCA
:1054F000012CE5D187F87A002C21284633F041FEB3
:1055000005460028E6D1A4F102000134B0FA80F08B
:10551000022C4FEA5010E2DD20B90023064A18465B
:1055200042F82830BDE8F081A7F87800CCE700BF4A
:10553000E03501203CB10408583601202DE9F04344
:10554000704900260846374633460AE0062C03F128
:10555000010308BF0137950448BF0136202B00F036
:10556000BE8050F8042BC2F30324002AEED1664D0E
:10557000FFB285F8743085F8757085F87660002B79
:1055800000F0B68000204FF00F0E8946F046064628
:10559000044659F8042B0134C2F3031C02F00F0235
:1055A0006645B8BF6646E045A8BFE0469042B8BF32
:1055B00010469645A8BF96469C42EADB464540F316
:1055C0008B8046447410013E013446F3470264B2B6
:1055D000704585F8F92185F8F84176DD704444106E
:1055E0000138013440F3470264B2484885F8F62197
:1055F000A0FB070285F8F741920802EB4202A7EBF5
:10560000420212F0FF0F65D0062F3A4608D9FC0778
:1056100006D401E0D00702D45210062AFADCD7B231
:1056200085F87770002B6AD0AE6FC6F30536720727
:105630004ED40C1F0A4604EB830403E052F8040F17
:10564000470445D49442F9D10127B4070CD40C1F68
:105650000A4604EB830403E052F8040F800403D4E9
:105660009442F9D147F0020772090CD10C1F0A4687
:1056700004EB830403E052F8040F800303D4944244
:10568000F9D147F0200730070CD40C1F0A4604EB71
:10569000830403E052F8040F000403D4A242F9D1BA
:1056A00047F04007F2060BD40A1F02EB830303E026
:1056B00051F8042FD60303D49942F9D147F080075B
:1056C000BFB2A5F84C7BBDE8F083062207248CE727
:1056D0000027BAE70627A3E70622072478E70A4D42
:1056E000FFB285F8743085F8757085F8766049E703
:1056F0000622072485F8F92185F8F84175E7E327A4
:10570000DFE700BF58360120E0350120ABAAAAAA86
:1057100000236B4A2DE9F04F0C4689B09A462C21A4
:105720004FF001089B461E461F46DFF8A0910390EC
:1057300042F820300293019323785FFA8AF5A3B1EF
:105740008B4278D0601C0DF1140C00220CF8013B48
:10575000044610F8013B013243B18B426CD00A2A57
:10576000F4D1002009B0BDE8F08F1A4608AB1A4406
:10577000002302F80C3C0029F3D16B1E0134032BEB
:1057800003D8DFE803F05138105F013505A80EF0AB
:105790007FFE8346EDB2042D59D84D440AF1010A2B
:1057A00095F8E410C8E79DF81420002A40D00DF1C8
:1057B000140CDDF804E04321424800238A4206D05D
:1057C0000133072B04D010F8011B8A42F8D19E4602
:1057D000542A5CD04F2A61D0422A63D0562A65D021
:1057E000492A65D0572A67D01CF8012F002AE2D138
:1057F000CDF804E01CE09DF81430CBB105AA0CE014
:10580000452B49D0532B4BD0572B4DD0552B51D036
:10581000442B53D012F8013F53B14E2BF0D100234B
:1058200008FA03F31F43F5E705A80EF031FE0290D6
:105830000135EDB2B1E7002208AB1A44002302F8AB
:105840000C3C9AE705A80EF023FE0F281DDD002171
:10585000029B4FEA0B1B1C4A03F00F035FFA8BFB02
:1058600043EA87530B43039902EB8109019A43EA08
:10587000022343EA063646EA0B06C9F87860FFF7CA
:105880005DFE012009B0BDE8F08F8104E0E7002350
:1058900008FA03F31E43A7E70123C1E70123F7E753
:1058A0000223BDE70223F3E70323B9E70323EFE76E
:1058B0000423EDE70423B3E70523E9E70523AFE776
:1058C00058360120D1D30408E035012060B0040827
:1058D0002DE9F041844C88B0FFF730FE012394F8A5
:1058E000695140F6A8420021804884F84A3B33F0D1
:1058F00079FB95B97E4B0020FF2203F180011880CF
:10590000043303F8022C03F8012C9942F7D101204B
:10591000FEF7E4F808B0BDE8F08128460BF044FA41
:105920004279C36806460168A4F8482B002BE1D0F1
:10593000704B714A1B68C4F8081B934200F2B88090
:105940000022511CC4F80C2B6C4A0320B3FBF1F36A
:10595000B3FBF2F39AB2C4F8143B0021B2FBF0F3AC
:105960005A006748A4F8FC3AA4F8FE2AC4F8181BA9
:10597000C4F8101B08F060F807460028BAD1284682
:105980000BF01AFEC4F8400C10B12923C7718371C3
:10599000327A4E210BF0DCFE5A4A00234020116B74
:1059A0004FF48067C4F84C0C4FF4805541F400115B
:1059B000C4F8503C11634FF48041126B306902F41B
:1059C0000012C4F85C1CF16800924FF40032C4F875
:1059D000480CC4F8642C94F8482B009803200C2A37
:1059E000C4F8603CC4F8683CC4F8703CC4F8743C2B
:1059F000C4F8547CC4F8585CC4F86C0CC4F8441C5B
:105A00005ED8414B03EB4203B3F8EC503F4B05F13A
:105A1000080700222921A3F59E7804EB8707C4F824
:105A20007C8CC7F8083B307D22F0F8FB60222B46C7
:105A30003749307D22F0C8FBD7F8080B05F01CFF72
:105A4000024600287FF456AF06906027F37940465F
:105A5000079201A95D000292DB00059205F00205A4
:105A6000B4F8482B03F008030197CDE9035323F062
:105A7000F5FF00287FF43EAFF279B4F8480B9207A7
:105A8000D4F8083B1ED50422196A824021EA02019B
:105A90001962196A0A431A625A6C42F400425A6443
:105AA0001A6842F001021A60012384F8043B21E7DE
:105AB000184A19491A44B2FBF1F2013A92B240E78E
:105AC0001D46A3E70122196A144D8240AB4221EA28
:105AD00002011962196A42EA01021A62DCD0104A14
:105AE0009342DDD1D8E700BFE03501203800002027
:105AF0004C370120849C0120FF6BDC0200350C0038
:105B0000E84001200038024060B00408244201202F
:105B10007146030800366E01006CDC020000014093
:105B200000040140054B1B789B0703D5044B9B7C6D
:105B3000042B00D87047FCF7EFBD00BFE15E0120E9
:105B4000E45E01202DE9F04FA54C83B0A54994F8FF
:105B5000A42CA54E12F1FF320B68A44D18BF0122F0
:105B600096F800E0D4F8840A43F0200384F8A42CCB
:105B70001EF0020F2A68C4F8880A0B60C4F8842A51
:105B800000F0D5809A4FBB7C042B40F2D080DFF828
:105B9000948298F8003013F00102009200F0CA805D
:105BA0001EF0010E00F00F81CDF800E094F8A5CCB6
:105BB000B7EE007A8F4B0CF1010CD7F800808E4ABB
:105BC000A3FB0C13D7F8049082FB08604FEAE8713E
:105BD0009B088A4EC1EBA05182FB090203EB8303B1
:105BE000DFED876A4FEAE97B06FB0180ACEB03033C
:105BF000CBEBA25BD4F8A82C04EB830A03F1050CD1
:105C000006FB0B96DAF8B07C04EB8C0CCAF8B00CEF
:105C1000A2EB070ADCF8B07CD4F8AC2C5044DFF8D7
:105C200008A2D21B2F682D68324484F8A53C019548
:105C3000D4F8E05CC4F8A80C7F1BCCF8B06C714EB3
:105C400007EE907A8AFB00378AFB023AC317F8EE18
:105C5000677AD017C3EB67036B4FC0EB6A0AC4F8CF
:105C6000AC2C67EEA67A06FB013106FB0BA6019B66
:105C7000C4F8D81CC7FEC77AC4F8DC6CC4F8E03C92
:105C8000C7ED007ABEF1000F59D1604BA4F8E8ECE3
:105C9000A3F800E094F8EA3CDBB3B7EE007AD7ED66
:105CA000007AD4F8EC3CB4F9F42CC7EE276AA8EBE0
:105CB0000303574907EE103AB8EEC77A27EE267A63
:105CC000BDEEC77A17EE103A91ED7C7A02FA83F2B4
:105CD000D4F8F03C66EE876AA9EB0303002A07EECE
:105CE000903AB4F9F63CB8BF0132F8EEE77A42F3E5
:105CF0004F0267EEA67AA4F8F42CFDEEE77A17EED1
:105D0000901A03FA81F3002BB8BF01335B10A4F89B
:105D1000F63C0123C4F8F09CC4F8EC8C84F8EA3C0F
:105D2000009B0BB9FFF7FEFE012384F8F83C03B09B
:105D3000BDE8F08F2EF001039646337036E7D4F8B5
:105D40007838334AA3EB09039FED326AD2ED7C7AAF
:105D500000EE903AD4F87438F8EEE00AA3EB0803AA
:105D600060EEA70A07EE903AB8EEE77A60EEA06A16
:105D7000B1EE470AE7EE076AF1EEE67A67EE867A59
:105D8000FCEEE77A17EE905A0DF082F99FED227A39
:105D9000DFED227AE0EE077AFDEEE77A17EE903A31
:105DA000002B02DA03F50C43A0331D48D917A0FBE2
:105DB000055280FB030315485209C1EB63130280AF
:105DC000A4F8E83C66E7FCF7A7FC98F8003096F8E2
:105DD00000E003F001030EF0010E0093E6E600BFC1
:105DE000E035012020530120E15E012058A101206F
:105DF000E45E0120CDCCCCCC6BCA5F6B806967FFC1
:105E00006F12833A80969800C4420120045F0120FB
:105E1000140001202C7D8E3FA00CB34500A00C4641
:105E20001F85EB51C05201206766666608B5FCF716
:105E30009BFC00B908BDBDE8084083E6F8B5BB4C43
:105E40000546D4F8FC0C2DED028B48B90CE0D4F8D3
:105E5000FC0C0BF0C5FAFCF787FC90B9D4F8FC0CED
:105E60000BF0C6FA0028F2D194F8942A531E042BA2
:105E700000F2FF80DFE813F0B300B300B3000800C6
:105E80000201FFF75FFEE9E7A94840F6C416D4F81F
:105E9000843A0268A749D21A0B68B24200F2908194
:105EA00003F02003002B40F01B8194F80B3D022BE4
:105EB00005D00A202FF0F2FE002800F033819E4B1F
:105EC0001B8813F4006303D094F80C3D13B901232D
:105ED00084F80C3D994A9A4BD2781B6884F8402D7F
:105EE000C4F8143D0BF0C0F894F8F83C0546002BBC
:105EF00066D0D4F8146DD4F8483DD4F8442DF31A84
:105F00009049821ADFED906A07EE903A0B8B07EE0C
:105F1000102A9FED8E8AF8EEE77A03FB03F3B8EEC2
:105F2000476A91ED0C7A8A4F67EEA67A06EE903AB0
:105F300067EE075A91ED0B7AF8EEE66AD7ED074A5D
:105F400087EE865AD1ED0D7ADFED828A824B834A45
:105F5000997C85EEA66A10889A89B4F8E83CA4F882
:105F60001E2DA4F81C3D27EE077AA4F8180D84F81E
:105F7000201DA7EEA77A65EE087A87ED065AE4EEB3
:105F8000A87A36EE077A17EE100AC7ED077A30F0D6
:105F9000F3FB41EC100B31F04FFD51EC100B30F0E6
:105FA0001BFF07EE900A97ED097A27EE888AC4F85E
:105FB000486DC4F8445D3862A7EE288A87ED098AE7
:105FC00094F80C3D072B00F24F81DFE813F0040337
:105FD000080123018902AF02E8029C00A20094F8A4
:105FE0007C68002E00F0C480012E42D1D4F8FC0C55
:105FF0000BF0F2F9E8B394F8943A022B00F05184D4
:10600000032B00F00D84012B33D1494AD4F8903A88
:10601000D2F800C0ACEB0303C72B2AD9D4F88C3AD2
:10602000042B00F2DA8403EB43024D49D4F8FC0C54
:10603000002301EB820201F19C07D0F808E01E4624
:1060400092F80921C4F890CA04E0102B00F0C8842B
:1060500057F8046FB6455FFA83FC03F10103F4D1EE
:10606000624500F0E98401EB8202D2F89C1009F04D
:1060700021FF304B1B6803F0200313E7D4F8803A6C
:1060800094F87F280133C4F8803A62B194F8953AC5
:10609000344A0133DBB2A2FB0312920802EB820204
:1060A0009B1A84F8953A304E002221480127317816
:1060B000204B21F00201C4F88C2A1B68317006685D
:1060C00003F020030168C4F8846AC4F8901A2249D6
:1060D00084F8962A8A7484F8947A002B3FF4E5AE0B
:1060E000D4F8003DEB1A002BFFF6DFAE1A4B9B7C79
:1060F000042B7FF6DAAE1D4B01202B44C4F8003D83
:106100000BF094F9D1E64FF400200AF071FC14F082
:10611000AFF8002384F80C3D002384F80D3D0023E4
:1061200084F8F83CBDEC028BF8BD00BFE0350120DF
:1061300058A1012020530120F8BA0120C4520120A7
:10614000DC5E0120EC0C002000247449CDCC4C3ED8
:10615000EC420120CDCC4C3FE45E0120045F0120E5
:1061600060B00408CDCCCCCCE15E0120F049020047
:10617000012A00F09F82022A7FF47BAFCB4AD4F839
:10618000903A1168CB1AB3F57A7FFFF472AFD4F866
:106190008C3AC4F8901A002B00F0DA83012B40F2FD
:1061A000EF83C34B042112681B68C4F8902AC4F81B
:1061B0008C6A03F0200384F8966A84F8941A71E6D6
:1061C0000568002223F020030520C4F8905A0B60D4
:1061D00084F8940AC4F88C2A84F8962A65E6B4F800
:1061E000883D1BB9B4F8A03DA4F8883DB4F8183D2B
:1061F000632B0CD894F8403D002B40F0F182AD4B5E
:106200001B78DB0740F1EC82032384F80D3D022369
:1062100084F80C3DD4F8343DD4F8142D9B1A002B8F
:10622000B8BF5B42B3F57A7FC0F2E08194F80C1DF1
:10623000B4F88E5D6423D4F8102D4FF4FA7003FB8C
:1062400005F3012502F2DC52C4F8380D40F60A705D
:1062500084F83E5D9342A4F83C0DB8BF1346C4F8E1
:10626000343D00293FF458AF94F80D3D5BB194F8EC
:10627000A93D012B04D0022B05D194F8403D13B168
:10628000062384F80C3D8C4B93F8A83C13B10223F1
:1062900084F80D3D0AF0E8FED4F8AC3D874AC31AF5
:1062A000934294F80C3D14D9032BC4F8AC0D00F0C4
:1062B000B98194F9B12D94F8200D94F8A81D884265
:1062C00038BF0132002A14BF01224FF0FF3284F898
:1062D000B12D002B3FF423AF94F83E3D002B40F04E
:1062E000B08194F8F83C002B3FF419AFB4F81E2DA0
:1062F0006FF06307D4F8383D71489B1A714DB4F8BC
:10630000A66D80FB0312DB17D5ED007AC3EB62119B
:10631000B4F9C43D0AB207EE102A1A44B4F8A43DF9
:10632000642AB8EEC77AA8BF642277EE677A85ED53
:10633000007ABA4294F83C5DB8BF3A46FDEEE77A7F
:1063400005EB850502FB03F3A4F8C42D05EB8505D9
:1063500080FB032017EE902ADB1716FB02F6B4F839
:10636000A22DC3EB601394F83D0D12FB0162D4F82B
:10637000541DAD0013441BB2502BD4BFCB1801F1F8
:106380005003AB4280F245814F4B9FED507AA3FB07
:1063900005234F4EC4F8545DDB0807EE903AF8EE43
:1063A000E77A67EE877A17EE900A30F0E5F941EC6C
:1063B000100B31F095FA51EC100B30F00DFDD4F8C4
:1063C000141DD4F8343D05EE900A3D4A5B1AD6ED13
:1063D000007A82FB0312DB17C3EB621319B207EEDC
:1063E000101A81EAE173B8EEC77AA3EBE173182BB8
:1063F00077EE677AFDEEE77A17EE902A10B240F357
:10640000FA8000221346A4F8CC2DB4F8962DB3EEF2
:10641000046A86ED007A03FB02F32E4EB4F8982D41
:1064200025EE866A86FB0376DB17C3EBA603B4F87A
:10643000946D02FB03F3B4F8882D01FB06F1B4F868
:106440009C6DA2F57A7200FB0313B4F89E0D07EE63
:10645000902AF8EEE76A07EE903AF8EEE77A86EED1
:10646000A57AC7EE866AFDEEC77A17EE903AFDEE82
:10647000E67A17EE902A12B202F57A7101FA83F3E6
:10648000B34203DB9842A8BF18460646124BA4F855
:10649000586D1B78252B7FF442AE104B94F80D1DE0
:1064A0001E805D809A80D98039E600BF58A1012006
:1064B00020530120C0520120380000203F420F002D
:1064C0001F85EB51A0430120CDCCCCCC88C3E43A4E
:1064D000A8430120676666666D9C0120709C0120C0
:1064E000B4F8182DB4F8903D9A4202D2042384F8EF
:1064F0000C3DB4F88E1D6423D4F8102D012003FB4D
:1065000001F3B4F8925D02F2DC520F21C4F8385D59
:10651000934284F83E0D84F83C1DB8BF1346B4F88E
:106520008C2DC4F8343D84F83D2D9DE6B4F8183D1B
:10653000092B07D8D4F8142DB2F57A7F02DC052296
:1065400084F80C2DB4F88E2D6421B4F8900D01FB65
:1065500002F2B4F8925DD4F8346D03FB02F203FB4F
:1065600005F392FBF0F2632A93FBF0F340F3C6804D
:10657000B242A8BF3246632BC4F8342DD4F8382D6C
:1065800040F3BA809342A8BF1346012141F20A4268
:10659000C4F8383D84F83E1DA4F83C2D64E6DB4B7E
:1065A000F7EE086AD3ED097A93ED087A67EEA67ADA
:1065B000B4EEE77AF1EE10FA00F31C81002301211A
:1065C0004FF4706284F83E1DC4F8343DC4F8383D81
:1065D000A4F83C2D48E6CE4B1B7813F0010340F0A5
:1065E0008F80C4F8103DA4F81A3D95E503231946A1
:1065F00084F80C3D1CE6B4F9CC3D6FF0F9020B4475
:10660000FA2BA8BFFA239342B8BF1346A4F8CC3D97
:10661000FBE600EB800000EB800085009D42A8BFF8
:106620001D46B1E694F9B02DB4F81E1D952998BF0A
:106630000132002A0CBF4FF0FF32012284F8B02D46
:1066400037E6B44BB4F91C2DB3F9043007EE902AA9
:106650009FEDB16A07EE103ADFEDB06AF8EEE77A27
:10666000B8EEC77AD7EE067AF4EEE67AF1EE10FAD3
:1066700036D89FEDAB7A77EE877AF2EE006A94F81F
:10668000B83DBFEE007A9FEDA66AF7EE005A002BE8
:1066900067EEA67ADFEDA36AA34B07FE257A67EEC5
:1066A000877AC7FEC67AC7FEA67AF1EE677AC3ED8F
:1066B000007A16E69D4AD4F8903A1168CB1AB3F5E1
:1066C0007A7FFFF4D6ACD4F88C3AC4F8901A002B39
:1066D00000F00A81012B40F24D81954B022162E5C9
:1066E0009FED947AF4EEC77AF1EE10FAC5DD9FEDD6
:1066F0008C7A77EEC77AC0E7642346E70A463AE722
:1067000094F84C3D002B3FF407AD8B4AB6EE007A6F
:10671000D4F8143D0025D2ED037A884AD4F8100D40
:10672000FCEEE77AD2ED086AB4F8181D9842B4F886
:106730001A6DF4EE476AB8BF184617EE903AB142A8
:10674000C4F8545D9BB2C4F8100D38BF3146F1EE69
:1067500010FAA4F8583DA4F81A1DC4F8505D7FF74C
:10676000DBACDFED777AF4EE676AF1EE10FA7FF5D5
:10677000D3ACD4F8801DDFED737A07EE101AB8EEB3
:10678000477AB4EE677AF1EE10FA7FF5C5AC40F2C5
:106790002E4083427FF6C0ACA3F57A73DFED6A7AB0
:1067A0004D1C07EE103AB8EEC77AE7EE267AFCEEFB
:1067B000E77A17EE903A9BB207EE903A002940F044
:1067C0004F81F8EE677A02F12803B0EE670AC3ED55
:1067D000007A31F0E5F8C4F8805DA4F8880D9BE4F8
:1067E00003234FF4002084F80D3D0AF001F913F063
:1067F0003FFD0CE54FF400200AF0FAF813F038FDE5
:106800000023072001214FF47062C4F8343D84F85E
:106810000C0D84F83E1DC4F8383DA4F83C2D23E54A
:1068200094F87E28002A00F0C78094F8962A002A5F
:1068300040F0AA8084F8966AD4F88C2AB22A40F2F2
:10684000EB8000230222C4F88C3A84F8962A3F4A4F
:10685000D4F8FC0C134493F8F8110AF0CDFDD4F8E9
:106860008C3A94F8962A0133C4F88C3A032A00F043
:10687000BB802F49032A0B6803F020037FF612AB7D
:106880002A4E00220B680420316803F0200384F8AC
:10689000940AC4F8901AC4F88C2A84F8962AFFF750
:1068A00001BB94F8953A294A03EB4303D4F8FC0C56
:1068B00002EB830393F8093102EB8302D2F89C10B8
:1068C00009F0F8FA194A1A4B0321106800221B68D4
:1068D000C4F8900A03F0200384F8941AC4F88C2AB0
:1068E00084F8962AFFF7DEBA4FF49651D4F8FC0CE0
:1068F00009F0E0FAD4F88C3A0D4A01331268C4F872
:106900008C3A02F02003FFF7CDBA00BFEC42012021
:10691000C0520120FCBA0120CDCCCC3D000034C3D4
:106920000000B4430000B4C39C43012058A10120DF
:106930002053012000003443F45201203C43012045
:106940008FC2753F0024744900007A4460B0040887
:1069500094F8953A4B4A03EB4303D4F8FC0C02EB52
:10696000830393F8093102EB8302D2F89C1009F0FB
:10697000A1FABFE74449D4F8FC0C0AF047FDB9E797
:106980004249D4F8FC0CF8E7012A3FF455AF022A3B
:106990007FF46CAFD4F88C3A092B7FF658AF0F2BED
:1069A00052D90023032194F88028C4F88C3A84F843
:1069B000961A0ABB364963E736480421344B00680F
:1069C0001B68C4F88C2A84F8962A03F02003C4F8C4
:1069D000900A84F8941AFFF765BA2D4B022174E7E8
:1069E0004FF0000CFFF73CBB94F88038002BE1D04F
:1069F000D4F88C3A432BDDD8224AD4F8FC0C13444B
:106A000093F828120AF0F8FCD4F88C3A94F8962AF5
:106A10000133C4F88C3A2CE71A4BD4F8FC0C13441D
:106A200093F844110AF0E8FCD4F88C3A94F8962ACA
:106A30000133C4F88C3AAAE794F8953A0C2202FB89
:106A40000311D1F80C1198E794F87D180D4AC1EBA9
:106A5000C101D4F8FC0C0A44134493F8FB11FCE682
:106A6000F8EEE77A92ED0A6A07EE105A134677EECF
:106A7000C67A2833F8EE476A87EEA67A77EE067A6A
:106A8000A3E600BF60B0040868150508881505086E
:106A90002053012058A101200C4C054608B5D4F81C
:106AA000FC0C18F06BFC284618F068FCD4F8FC0CC1
:106AB00001798B0705D441F002010AF089FCD4F872
:106AC000FC0C2946024A27F0F3FD00BFE035012007
:106AD0002D5E0108F0B5324D0023324C85B02E6892
:106AE00002202968C4F8906AC4F8841AC4F8F838F7
:106AF000C4F8FC38C4F80039C4F8043984F80839FB
:106B000084F8953AC4F87C3AC4F8803AC4F8F4386A
:106B100084F8943AC4F88C3A84F8963A18F048FD10
:106B2000B8B3077994F8952A1F4E02E0CAB2042A36
:106B300031D802EB4203511C06EB830393F8093171
:106B4000BB42F3D184F8952A94F8953A00270322A2
:106B500090F9020003EB430306EB83013B4691F8F7
:106B600009C1022106EB8C06D6F89C60CDE901270D
